:020000040800F2
:10000000005000207D720108197301084DEE0008B0
:100010001973010819730108197301080000000021
:10002000000000000000000000000000197301083B
:100030001973010800000000197301085317010823
:10004000197301081973010819730108197301085C
:100050001973010819730108D91A0108ED1A01086A
:10006000E91A0108E51A0108E11A010811940008CB
:1000700001940008F1930008E1930008D19300086F
:10008000BD930008AB9300081973010819730108A8
:10009000197301081973010819730108DD1A0108A1
:1000A0001973010899F700081973010889F7000806
:1000B00079F7000869F7000859F70008FD380108CA
:1000C00001390108F5380108F938010819730108E8
:1000D00019730108911701088517010819730108A0
:1000E000D51A0108197301081973010800000000EE
:1000F0000000000000000000000000000000000000
:0C01000000000000000000005FF808F1A3
:100110002DE9F04F0B4B0C4D0C4AC5F8B8340023B9
:1001200010680B499FB08842C5F8BC3416D11360E3
:1001300062B6084B18680AF033FB074B1B689847F8
:10014000FEE700BF8BC1000820060020F04F002012
:10015000EFBEADDE00F0FF1F04F0FF1F0893099310
:100160000A934FF4E013BD4C0B93236843F48033A0
:100170002360A36943F01003A361236803F40033F1
:100180000993089B01330893099B1BB9089BB3F59E
:10019000A06FF2D1236813F4003300F0A58202238C
:1001A0000A93AF4BAF4F1A6842F010021A601A68F8
:1001B00022F003021A601A6842F002021A606368B1
:1001C000636063686360636843F480636360A64B45
:1001D0001A68043B22F070425A60A44A3A6062688E
:1001E00022F47C1262605A6842F000425A60DA6877
:1001F00022F40042DA609B681E0449BF9C4B4FF416
:10020000E0133B604FF480130B930A9B012B00F02B
:100210008382022B05D10B9B6268134343F4803326
:100220006360236843F08073236023689801FCD5E2
:10023000636823F003036360636843F00203636051
:10024000636803F00C03082BFAD16368DFF8688257
:1002500003F00C03042B00F06382082B00F0628291
:10026000824BC8F800306368DFF85092C3F3031381
:1002700019F80320D8F80030DFF844B2D340C8F8AA
:1002800000307C4B4FF6FF72CBF80C30A3690DF1B8
:10029000780A43F00103A361636A636A764E43F010
:1002A00080736362A369304643F01C03A3614FF07F
:1002B00000032AF82C2D51468DF84E3009F03AF8FB
:1002C00051466E4809F036F851466D4809F032F84B
:1002D00010228DF83E2002228DF83F204FF400724C
:1002E0001EA921F83C2D3046326109F023F86549FA
:1002F00050464A6842F000724A600AF0B5F8139B13
:10030000614A3046B3FBF2F34FF47A72C5F8C03459
:10031000D8F800304FF0010CB3FBF2F35B4A013B1D
:100320005360F0238BF82330002393600723DFF81A
:1003300094E11360564A09F10E01002331F8026F6F
:1003400046FA03F818F0010F18BF0CFA03F803F18E
:1003500001031EBF1060A2F804800832102BEFD1F9
:1003600000F580607045E8D13B68404A934240F018
:10037000EB81012385F8C4340CF064FB18B90FF04D
:10038000B1F80EF0B1FD0EF0DBFE95F8C534414F2B
:1003900043F0010385F8C5343F4BDFF82C819A7890
:1003A0003E4B08F1050A1A703D4B1B683B6095F8FF
:1003B000CA3485F8C634002313F808004FEA830BCB
:1003C0005E1C002800F0C681029311F055FA029BD2
:1003D0004AF8230010B10523C671837112215AF81F
:1003E0000B0011F06FFA032E3346E5D100210846C9
:1003F00011F00CFB0021012011F008FB002102206C
:1004000011F004FB0121022011F000FBA36900217F
:1004100043F00103A3614022224819F0F4FD4FF09C
:10042000FF33214AC5F818356420C2F8033011F0B3
:1004300086F9A02200211D4819F0E5FD00241C4D7D
:100440001C4E0023605956F83310DA00884240F001
:10045000848109EB0203187F38E000BF00100240DE
:1004600000200240D80000200410014000127A0051
:10047000001BB7000005FA0500080140000C014010
:10048000001001400000014040420F0010E000E079
:10049000341600200C3600200816002014250020F9
:1004A00068180020F80A0020380B0020F81B0020F4
:1004B00008BE010878A101081000002060A1010811
:1004C00000ED00E000140140E70A0020103414F0B1
:1004D00037FEE02CB5D1B44AB44C0021A046914679
:1004E000B34E00250B5D01F10F00204406EB030A1B
:1004F00010F801CFBCF1000F05D09AF80CE0E645EA
:1005000008BF82F858E090F803C0BCF1000F05D096
:1005100016F803E0E64508BF82F859E00135032DDF
:10052000E6D1B2F8580040B108EB010009EB8303B3
:100530005065C3F8202502F517721C313829D0D137
:100540000424994E302200219A483D6886F82C45B3
:1005500019F059FD964B224693F80BC093F80A9078
:100560000023944C1846A2464FF0FF0BDFF89CE2A4
:1005700005F040081EF9011F1E29195540F0F380AF
:10058000B8F1000F00F0F980B9F1000F00F0F5802C
:100590000C33302BEED108B186F82C25864B874CD6
:1005A00093F800B0864E874B15F4805214BFA08894
:1005B000B08A83F800B00292994616F015FADFF877
:1005C0005082DFF850A2C8F80000308A16F008FA0E
:1005D0007D4B1860708A16F003FA7C4B18606088B7
:1005E00016F0FEF97A4B1860208816F0F9F9794B6D
:1005F000BAF81A101860C1F5FA60039116F0F4F910
:10060000754A03991060BAF81820B4F806A0501A79
:10061000A0EB0A00039216F0E7F9039A6F4908600D
:10062000C2F5FA60A0EB0A0016F0DEF96C4B6D4AD9
:1006300018606D4B2B40002B40F0A5806B4B03EBFB
:10064000CB0B9BF80130136040F2DC510023684A69
:1006500022F813100133082BFAD1029BB6F814B01C
:100660000BB1B4F804B0B378042B05D14FF480502B
:100670000BF064FF4FF0000B002599F800205D4C53
:10068000A2F11703022B257000F2C880DFF88891D1
:10069000002155F8090005EB090A16F08DFB00282A
:1006A00073D03B68DA0400F1DA800023D8F8001038
:1006B000514A42F823100133082BFAD12378C02283
:1006C00000214E48049319F09EFC3779B378003727
:1006D00018BF0127042B00F2E780DFE813F0900138
:1006E000E5009201E8008A01226842F001022260DE
:1006F0000893236803F002030993089B01330893CE
:10070000099B1BB9089BB3F5A06FF2D123689F0723
:1007100001D5012344E5FEE7636843F460137FE5F8
:100720003B689EE563686268C3F38343D10303F1CA
:10073000020302D4324A534393E5626812F4003F45
:100740003A6818BF5208F6E72E4A93427FF414AE77
:1007500002230FE64AF8230045E60133042B7FF419
:1007600072AE0020B2E61F297FF412AFB8F1000F7D
:1007700003D0BCF1000F7FF40BAF013A0AF803B0CD
:10078000D2B2012004E701235DE71F4B05EB030E06
:100790009AE80F008EE80F00237810350133802D82
:1007A00023707FF475AF7CE72006002098A1010834
:1007B0006C210020584100201C250020A42D002081
:1007C0006823002094110020802300203411002091
:1007D000BC110020B0110020C8110020B811002069
:1007E000C4110020541200202000100088AB010822
:1007F00044230020F42200205825002080250020DA
:1008000000093D00001BB700D0110020CFA1010856
:10081000C82600203836002064170020B44B13F897
:10082000321003EBC2030829217088BF0821D3F8D6
:1008300004C088BF2170BCF1000F3FF432AF002527
:10084000DFF8109323789D42BFF62BAF2B0103EB0B
:10085000090E63440FCB01358EE80F00F2E72378D1
:10086000012B7FF622AF4FF07C59A24D05EB03130D
:1008700003F110071035BD423FF417AF494655F854
:100880000C0C16F005F9494645F80C0C55F8100CFF
:1008900016F0FEF8494645F8100C55F8080C16F00D
:1008A000F7F845F8080CE5E7934CA04602E0934CB6
:1008B000DFF8A482924A934B21461A60924A934BE6
:1008C0004046002F18BF1346914A0025136015F0CB
:1008D000D7FF01464FF07A5016F08EF98D490390FC
:1008E000204616F0D5F88C4CDFF870A20590049BDA
:1008F000AB4240F3E58005EB0A035E790021304608
:100900000EF010FF029000287DD1844A7D4B1A60C2
:100910007D4A7F4B1A60824C82482368002B40F04E
:100920001F81037803F0EF02082A7F4A40F03A81E2
:100930001178182B41F01001117001D10FF046FE13
:100940002368002B40F03781784A794C136806926F
:1009500013F0010640F078819B0440F1C28194F8C5
:100960001826744B04F5A8651A7004F5C26816F8C9
:100970000890002148460EF0D5FE074698B30022A5
:100980004FF0010A5FFA86FB05F80FBC45F8040C2E
:1009900005F80E2C05F8062C05F810AC484610F0AA
:1009A0006BFFD3445FFA8BFB18B180F806A080F888
:1009B00007B04FF0000B2A2110F084FF5E4A00219F
:1009C000384610F0C1FD5D4B2A1D2B605C4B29465B
:1009D00038466B60C5F808B010F00AFE5A467979BF
:1009E00038680AF003FE0136082E05F11C05BED159
:1009F00077E10024A04601274FF0000B5AE7454C51
:100A0000F8E7504C51E7304610F036FF6B1C606140
:100A1000DBB210B10322C37182711A2110F052FFB0
:100A2000002F51D0BAF8000015F0DEFF16F032FAB0
:100A3000454B4FF6FF791E68B6FBF0F34B441B0C99
:100A4000B6FBF3F60FB1B6FBF0F99AF80230042BBF
:100A50003ED1484615F0C4FF2E4916F019F8A060A3
:100A60000790304615F0BCFF414616F011F8079B81
:100A700006903649184616F00BF8069A01461046BD
:100A800015F0FCFE9AF80330E060324601930299BB
:100A90001FFA89F3CDF800B0204615F041F9002384
:100AA00018221D49AB4218D1002383F0010323749F
:100AB00001231D44082D637404F118047FF417AF5B
:100AC0000122234B1A7026E7039816F047FFADE783
:100AD000304615F085FF0599BFE702FB0310466815
:100AE0006068864201D00133DCE70123DDE700BF07
:100AF00088AB0108D41100206F120339ACC5A737A9
:100B000019B100083831002099AE000845B100083D
:100B10003C3100206F12833A802500209BAE0008F4
:100B20005412002094110020ED2600200C360020E5
:100B3000200600209021002040420F0029B6000826
:100B40000FAD0008282930381000002000007A443A
:100B500058120020D0110020ACC5A7366823002011
:100B60000278334B334913F8325003EBC2035E680B
:100B70000D70002E3FF4D5AE00232F4FAB42BFF6D1
:100B8000D0AEC3EBC3017218D2F800C001EB070E60
:100B900041F807C091880133AEF8041092798EF8BD
:100BA0000620EBE70E2B3FF4C3AE1178192B21F092
:100BB00010011170C1E600254FF0040B1F4F204EAD
:100BC000DFF880A0A7F1030917F8018FB8F1000F33
:100BD0003FF4BAAE404610F04FFE01350446706156
:100BE000EDB210B180F806B0C571002140460EF09C
:100BF00099FD80461A21204610F064FEB8F1000FDE
:100C00003FF4A2AE0022B9F8023001929AFBF3F34E
:100C1000B9F800209BB2009230460A4A414615F0CE
:100C20007FF80123082D737406F11806CCD18BE6EA
:100C3000D4A90108152B0020162B00207D2C0020A4
:100C40009421002040420F000025FF2294F82D75CA
:100C5000CF4B294638461D705D609D60DD601D6488
:100C600083F8442083F8452083F8465083F84750A2
:100C700083F848500EF056FD064690B30368C54908
:100C80006A18507C18B15268934200F03F841835BE
:100C9000C02DF5D10025C4F83C6584F830553846A0
:100CA00010F0EAFD10B10223C571837100252A21DD
:100CB00010F008FEB84A0021304610F045FCB74B52
:100CC000B74AC4F84035B74B111F3046C4F8443515
:100CD000C4F8485510F08CFC2A46717930680AF047
:100CE00085FC94F8C534B4F81E6643F0040384F818
:100CF000C534A4F8206694F81A06002E40F011843A
:100D000010F0BAFD94F81B26C4F82406003218BF70
:100D1000012284F8282650B1242294F81C368271CE
:100D2000002BC6710CBF1221162110F0CBFD002044
:100D300010F040FE4FF000089B4B0020C4F84836EE
:100D400008F0DAFA012008F0D7FA984A02F1200CEC
:100D500052F8055CA5B312F9093CE11891F84C660C
:100D600091F84E7691F850E604EB0310911E11F8BD
:100D7000019FB14591F8029008BF80F85866B945C7
:100D800091F8049008BF80F85976F14508BF80F8C3
:100D90005AE68A42EBD104EB031393F8581679B163
:100DA00093F8591661B193F85A1649B15179C3F8BD
:100DB000545683F85B16917983F8608683F85C1645
:100DC00010326245C4D114F007FB14F005FB94F80F
:100DD0006C0614F0B5F9012394F86C2602F01F019B
:100DE0005209022A03FA01F300F0CA83032A00F031
:100DF000CC8394F8680610F03FFD054618B1122325
:100E000083710223C37194F8690610F035FD18B19F
:100E1000132383710223C37194F86A0610F02CFD2A
:100E200018B1142383710223C3711B21284610F0CB
:100E300049FD94F8690610F01FFD072110F042FDEE
:100E400094F86A0610F018FD1B2110F03BFDD4F851
:100E50006426574B9A4240F09D8303F56043D9685E
:100E600041F48051D960D96821F48051D96094F857
:100E70007036002B00F0AA8300231846118801F475
:100E8000415141F445710B4303431380938B23F489
:100E900000631B041B0C93830723138213889BB2EC
:100EA00043F04003138094F8C434032B11D11F2066
:100EB00007F037FC00233F4A02EBC30191F902100F
:100EC000022901F016820133042BF5D1022007F02C
:100ED00028FC0BF014FA012012F0A2FB2C2010F0D9
:100EE000CBFC9F238DF83C300023C4F874063220DD
:100EF0008DF83D308DF83E308DF83F3010F01FFCFE
:100F0000D4F8740610F042FD04230FAA13A92A484E
:100F10000BF07FF9D4F8740610F03DFD9DF84E30CB
:100F20009DF84D201B0243EA02439DF84F201343D6
:100F3000224A93421FD0322010F001FCD4F87406EC
:100F400010F024FDF5211C480BF091F9FF211A48FF
:100F50000BF08DF98DF84C00D4F8740610F01BFDE1
:100F60009DF84C30702B06D194F8C434022B02D17A
:100F7000032384F8C434124B00211E791148751ED6
:100F80006A426A415D7984F878266F1E1CE000BFD2
:100F9000AC1B00208025002040420F0035AD00082A
:100FA000640B002069AE00086C210020DDA101085F
:100FB0000030014032410020003800401520200060
:100FC000FE350020A00C00207B427B4184F87C365B
:100FD000069B14221B6803F40047C3F3C03384F854
:100FE0007A3619F010F8012E04BF94F8793684F897
:100FF00080361FB194F87B3684F88F3694F87E36AD
:101000001BB194F87F3684F88A36012D08BF94F816
:101010007D36C14D08BF84F8853600232E464FF03B
:10102000070B1F469946DFF83C8308F1940A307895
:10103000E8B110F021FC18B180F806B080F80790F4
:10104000002110F03FFC002331781AF813005A00F9
:10105000884240F0BE8208EB020393F8953073702B
:101060000723337101237A1CB770F370D7B20BF1E9
:10107000010B5FFA8BFBBBF10B0F06F10506D6D116
:10108000002B00F0BB80A54E4920736843F4404319
:10109000736014F055F8A24AA24900234FF01C0EC9
:1010A000104688460EFB032CDCF804C08C4540F04B
:1010B0009682DBB21C2101FB0303726919694FF0B0
:1010C00000090A437261062283F819901A7695483E
:1010D00009F051F913A809F023F9934B022F139348
:1010E00034BF4B46802318934FF4807319934FF409
:1010F00080631A9320231B934FF400538B4E13A944
:10110000884816971C931496CDF85490CDF85C90AF
:10111000CDF8749009F011F9012F94BF002201223B
:10112000D8F80030824943F00103C8F800304B681A
:101130004FF0070E23F4702323F4807343EA022355
:101140004B608A687B4B134043F4602343F00203F7
:101150008B60CA6A7B1E22F47002DBB242EA035340
:10116000CB621F270123EA784AB395F80180581C07
:10117000B8F1090FC0B295F804C040F23682A8F168
:101180000A02D1F80C9002EB42020EFA02FA29EAA6
:101190000A090CFA02F242EA0902CA60062B00F2BE
:1011A000318203F1FF3C4A6B0CEB8C0C07FA0CF319
:1011B00022EA030308FA0CF21A434A630346053590
:1011C000AE42D0D15A4B9A6842F480729A609A68C3
:1011D00042F001029A609A6842F008029A609A68A6
:1011E0001007FCD49A6842F004029A60504B9A6847
:1011F0005107FCD49A6842F4A0029A60D4F89C0685
:10120000002841F0BD80D4F8A036002B41F0B88012
:10121000D4F8A436002B41F0B3800DF05DF930B95D
:101220000120022110F030FC012014F065FE0121A4
:1012300094F8C534084643F0020384F8C53410F02E
:10124000E5FB0021084610F0E1FB0021022010F030
:10125000DDFB0A25384E012010F0FFFA002010F0C7
:10126000FCFA192010F06BFA3368DA0302D401207B
:1012700010F0A0FB192010F062FA002010F09AFB89
:10128000013DE8D12946284610F0C0FB294601203F
:1012900010F0BCFB294B2A4F18680FF0DBF9BA8914
:1012A000002A40F0F981274B0DF14C08587A15F0CF
:1012B0009BFB254915F0ECFB244915F0E1FA0BF0F6
:1012C0000EFC234B1860234B188A15F08DFB01464A
:1012D000214815F091FCC4F8A80611F043FB012346
:1012E0001393069B1A68530201D41C4B1393D70027
:1012F0005EBF139B43F010031393194B19680293BD
:1013000011F0020F1EBF139B43F0C60313934E0749
:1013100048BF139B28E000BFA00C00200010024033
:1013200014000020080002404C240140B40C0020AE
:1013300000240140FDF7F1FF741800201025002063
:101340007A2C00207431002035FA8E3CDB0FC93F27
:1013500094310020A8220020A889803A01000010C2
:101360001825002060A1010844BF43F0080313932F
:10137000D40542BF139B43F000631393B04B19781D
:10138000039301F0EF00082801D00E2903D1139B2D
:1013900043F480531393139BD00354BF43F400537F
:1013A00043F420431393139BD7044CBF43F064438F
:1013B00043F044431393960642BF139B43F4807358
:1013C0001393540742BF139B43F400331393139BAF
:1013D00043F400201390500505D59A4A127912B1B2
:1013E00043F4C0131393182908BF139B4FF0010651
:1013F00004BF43F0607313930723149329464046B8
:10140000ECB20BF0E8FF70B120460DF0E7FC50B9EC
:101410006A0958F8223004F01F0406FA04F423EA9B
:10142000040448F822400135242DE7D1864D98E880
:10143000030005F2AC6383E803004FF41972002146
:1014400005F2B46018F0DFFD07F08AFB00227F4F41
:101450007F4C049767607F4F7F4BBE461A809A701F
:101460007E497F4B7F4E80481960338BDFF824A282
:10147000A06085F8182919B2059005F61C1CDAF849
:10148000000027F8121000F596704CF82200013287
:10149000122AF4D1754FDFF8BCC13868C20458BFB6
:1014A000B6F92610AEF80610714901F1500E0A780F
:1014B000AAB98A7891F803A0524510D2002A00F008
:1014C000FF80013A02EB820202EB820202F56172B6
:1014D00091F801A092B20AF1040A2CF81A20043102
:1014E0008E45E4D1020740F16D81307A0A2800F27E
:1014F0006281DFE810F0F300F300D50351047504B6
:1015000095049504D90460011605F3001B8D594A12
:101510009BB212680133B2FBF3F3574A1370FFF723
:10152000B9BB10F0A9F94021C4F82406C4F840065C
:1015300005461C200EF0F6F80746CDB1C0B12423B5
:10154000AB7101231A21EB71284610F0BBF9002181
:10155000A4F8446601914949494A91FBF6F192FB8E
:10156000F6F389B200919BB23946464814F0D8FB95
:101570000023D4F82C26138084F83D36FFF7DABB1D
:10158000414AD1680B43D36033E43F4A11690B43AE
:1015900013612EE43D4B9A420AD103F5EC331969ED
:1015A00041F480411961196921F4804119615EE4B7
:1015B000374B9A427FF45BAC03F5EA33196941F487
:1015C00000411961196921F40041EFE7012302206C
:1015D00054E401330A2B7FF438AD00233FE5013397
:1015E000072B7FF45FAD002364E50A6908EB480A26
:1015F0000EFA0AF922EA09090CFA0AF242EA090289
:101600000A61CBE50C2B0DD8DA1FD1F830C002EB04
:10161000820207FA02F32CEA030308FA02F21A43E1
:101620000A63CBE50D3BCA6A03EB830307FA03FCAD
:1016300022EA0C0208FA03F31343CB62BEE500BFB3
:101640001C250020261A002020060020F1FD00089D
:10165000D8290020CC35002010360020A0860100BB
:10166000B829002038360020EDFD00080C36002097
:101670007C180020100000201C04002020A107007E
:1016800040420F004C0C0020001002400038004087
:10169000003C0040801B00202E46DFF83890DFF829
:1016A0003880B88915F09CF9D9F80020014608EB7C
:1016B00006002C360BF04AFEB6F5B07FF1D1F2E50C
:1016C0000AF1010A0AEB8A0A0AEB8A0A0AF5617230
:1016D000FEE600BFF82400207C120020B64B40201C
:1016E0001C6007F01BFA8346002864D04FF0000905
:1016F000B24A82F80090069213F05AF9317A824683
:101700000129069A0CD0C0F0B9820A2916D1AC4B37
:101710001B6813F480631CBF80F00103DBB21370FD
:101720000322A84B1A700722A74B1A700122A74B5D
:101730001A700C23237042F6F8236380A44B9F4A4F
:101740006360A44BA3609BF90200BAF1000F40F064
:10175000A3821378002B0CBF012303231278002AE5
:1017600040F09C82B27A002A0CBF0022082201922B
:101770000093994A4FF4E133402107F019F8974B51
:101780001860BAF1000F01D0954B1860737D217875
:10179000013BDBB2934A994213709CBF0023137044
:1017A00028B1864B1B7813B1012385F864390030CA
:1017B00018BF012030B908200AF0C0FE049B636006
:1017C000059BA3607E4B1B6858040BD51222227028
:1017D00044F620626280844A84496260844AA2603E
:1017E000844A116042F20102134209D044F6206299
:1017F0009904628040F1C083082222707E4A6260B0
:101800004FF0000A7D4CDB0384F800A040F18D818D
:1018100013F07CF901232370794B40F22A3293F8BC
:10182000F1B05146774818F0EEFBBBF1000F00F025
:101830006F81514658460DF075FF734B02680446A0
:101840001A6082689946002A00F06281584610F0BA
:1018500013F8C5F8680918B1282380F807A0837128
:101860001B2110F02FF80023684AD9F8001002F16C
:10187000180E5EF833004FEAC30C814240F08383B8
:101880006244107F13F05CFCD9F80000604A0388C2
:101890004FF0000A23F001031B041B0C03805D4B77
:1018A000DFF880E11B68ADF836A0934281BF03F1F9
:1018B000B772594902F55852B2FBF1F292BF0022B9
:1018C00002F1FF3292B2511CB3FBF1F35349ADF870
:1018D00032A0B3FBF1F303219BB2B3FBF1F14FEA6A
:1018E000410CAEF800C0DFF840E18DF838A0AEF84A
:1018F00000101EA921F8482DADF8343013F025FD55
:101900006023ADF83EA0ADF840A0ADF842A0ADF820
:1019100044A0ADF848A0ADF846A0ADF84AA0ADF897
:101920003C30E3794FF0000B580757BF01220422E7
:10193000ADF83E204FF4807203F002034CBFADF8C7
:101940004020ADF84820ADF84430ADF842B00FAAC1
:101950006179D9F800000DF0F1FD6179D9F8000046
:1019600013F0C6FCD9F800200121B2F84430DFF8AA
:10197000BCA06FEA43436FEA53439BB2A2F84430E2
:1019800013889BB243F0800313806379108C01FAB3
:1019900003F39BB280B220EA03001084108C80B263
:1019A00003431C20138413889BB20B431380237BB7
:1019B0001B4A00FB03233BE0802A0020852A0020ED
:1019C0000C3600207F2A0020842A0020B328002023
:1019D00069F90008B5000108D5010108E42A0020D2
:1019E0006C1B00207E2A002069FE0008400D0300C9
:1019F00051FE0008B829002041FE0008AB35002048
:101A0000243400209C370020CC3A002060A101083B
:101A1000FF6BDC0210000020006CDC0200350C00C3
:101A2000140000209A37002098370020C83A002080
:101A3000BB4A1869D2F814E040EA0E0EC2F814E06E
:101A40004FF0280E83F819B083F818E0D2F814E0AC
:101A500040EA0E005061B34AC3F814B09A605B7B51
:101A600013A88DF84D108DF84F108DF84C308DF86F
:101A70004EB013F083FBA068CAF8000008F07BFCAE
:101A8000DAF80000036823F001031B041B0C036059
:101A900008F071FC13A808F043FCD9F80030627913
:101AA00034331344139340F22A331693802318934C
:101AB0009D4B13A91493102315934FF4007319939E
:101AC0004FF40053DAF800001C93CDF85CB0CDF869
:101AD00068B0CDF874B0CDF86CB008F02EFC627927
:101AE000D9F800100C2A8EBF5B46904B03EB4203E3
:101AF0008A8998BFB3F8A83092B21343DAF800206D
:101B00008B81136843F0020313600122884B1A7023
:101B10000023FF211C4687481A181C520433802BCF
:101B20009170D170F8D113F061F8834B1B6859059F
:101B30003FD5042006F0F2FF804B0421186006F028
:101B4000E3FF7F4B1870082006F0E8FF7D4B08216B
:101B5000186006F0D9FF7C4B2C22187000217B48BE
:101B600018F051FA7C2385F86C398E2385F86D398D
:101B7000E02385F86F397D23202085F8973906F01A
:101B8000CDFF734B2021186006F0BEFF714B18701B
:101B90004FF4805006F0C2FF6F4B4FF48051186035
:101BA00006F0B2FF00226D4B18706D4B1A7008F0F2
:101BB00059FF6C4CB4F80090B9F1000F40F044822A
:101BC00095F89809002800F03F820FF055FEC5F8FF
:101BD0009C0918B11A2380F80790837113210FF024
:101BE00071FED5F89C090FF0D6FE00BF02215E48B9
:101BF0000AF0F0FA4FF000099F2332208DF83C30B4
:101C00008DF83D908DF83E908DF83F900FF097FD48
:101C10008DF84D9000BFD5F89C090FF0B7FE042356
:101C20000FAA414650480AF0F4FAD5F89C090FF083
:101C3000B2FE00BF9DF84E309DF84D201B0243EAD6
:101C400002439DF84F201343484A934200F04283D9
:101C500000F39F81464A934200F0A48101329342EF
:101C600000F0E581A2F51A42033A934200F02D8379
:101C7000002323806380A360E360E5E102213D4A05
:101C80000723117003213C4A237011703B4A45F22F
:101C9000F05382F8009050E503235FE5082266E5E3
:101CA0000A221B0193FBF2F300223549A3F5B0632E
:101CB00041F822300132122AFAD142F6F823638029
:101CC000304B40206360304B2270A36006F026FF4B
:101CD000824600283FF46FAD12F06AFE737AB17A43
:101CE00000280CBF01220322002B0CBF0623072370
:101CF00000290CBF002108219AF902E082460B431B
:101D00008DE80C00214B224A4021704606F050FD20
:101D1000BAF1000F3FF44BAD1E4B186047E500BF12
:101D200000100240DF8C00089C37002060A10108F1
:101D3000C63A0020183500200C360020641B002015
:101D4000701B0020601B0020711B00208C0F0020E6
:101D5000781B0020731B0020881B0020841B0020A0
:101D6000851B002038040020003800401620C200E7
:101D700017BA20007F2A0020842A0020B3280020E0
:101D8000E428002091F90008ADF90008A0860100C0
:101D9000210201086C1B00201023237042F6F82357
:101DA0006380814B40206360804BA36006F0B6FEE9
:101DB000824600283FF4FFAC12F0FAFDB27A002808
:101DC0000CBF01230323002A0CBF002208229AF92A
:101DD00002E00192009382464FF4E133744A93E7A4
:101DE0000823237042F6F8236380724B402063601F
:101DF000714BA36006F092FE824600283FF4DBACF4
:101E000012F0D6FD002200280CBF012303239AF90B
:101E100002E00192009382464FF4E133674A73E790
:101E200000234FF00C0E664A66491370664A062876
:101E300084F800E00B7013702BD01B22634B4FF41F
:101E4000E13B1A700522624B83F800E0614B1A7087
:101E500042F6F8236380604B402063605F4BA360D1
:101E600006F05CFE824600283FF4A5AC12F0A0FD0F
:101E7000B27A00280CBF01230323002A0CBF0022E2
:101E800008229AF902E00192009382465B46544A86
:101E90003AE721224D4BDFF884B11A704C4B83F89E
:101EA00000E04C4B1870D3E74FF0000B4D4B402037
:101EB00083F800B00E23237044F6206363804A4BFE
:101EC00063604A4BA36006F029FE00283FF473AC20
:101ED000B0F800A0464B0AF4825A83F800B0B37AF7
:101EE000BAF5825F90F9020014BF01220322B3B950
:101EF000BAF5825F14BF5B4608238DE80C004021D1
:101F00004FF4E1333B4A06F053FCBAF5825F7FF4AD
:101F10004EAC0022384B1860384B1A7047E4082347
:101F2000EBE70A221B0193FBF2F300223449A3F5ED
:101F3000B06341F822300132102AFAD142F6F82378
:101F40006380304B402063602F4B2270A36006F00B
:101F5000E5FD00283FF42FACB37A90F90200002B86
:101F60000CBF0023082301930323284A0093402138
:101F7000274B06F01DFC1AE4DA077FF541AC0C2272
:101F80002270244A3BE40133042B7FF472AC00201E
:101F900078E4214A934200F09F8141DC023A934267
:101FA0007FF466AE802391E1CDF80008E1F80008E7
:101FB0001100010845F800085DF80008C9FF000895
:101FC0004D2A0020E42600204C2A00200C28002066
:101FD000302800204E2A0020B7E30008CDE3000897
:101FE000F1FE0008A72A002079FE0008A1030108DD
:101FF000A52A0020CD020108141A0020201A002072
:10200000482900202DFB00085DFB0008750201082F
:10201000A068060031FE00081920C20090D003001D
:10202000B94A9342BED0013293427FF421AE4FF4BD
:10203000807323806380A38822881B02A36053439C
:10204000E360012385F8A039E468C4B14FF0000AC9
:10205000E40A0DF14C0BA2450CDA0AEB04094FEA35
:102060006909102241464FEAC9200BF071FB0F2885
:1020700000F335810BF010FBA44BE4021C60A44B71
:102080009A78A44B02B101221A70039BA2481B78D4
:10209000052B02BF4FF4C872A04B1A800CF07AFDDA
:1020A000C8229F4B00211A809E4AA5F8A2191378D6
:1020B000A5F8A41943F00803137003239A4A85F87E
:1020C000A1391370994B9A4A19805980994B117014
:1020D0001A799946012A0AD13022974817F093FFBE
:1020E0004CF250324FF07E5194480BF02FF9002102
:1020F000934B85F8D81919605960996099F80530A3
:10210000012B09D110228F4817F07DFF4CF250327D
:102110008D498E480BF01AF98D4B8E4A1B684FF093
:1021200001083B608C4B00211B688C489B1A18BF30
:1021300001238B4A85F8188A1370442217F063FF35
:102140000023884C884A20461360C5F81C3A06F0E4
:10215000EDF9029B1B68DA0709D5844B41461B68E1
:102160004046642B38BF6423636406F017FA804B43
:102170001A68984612F0020F09D00121022006F0D9
:102180000DFA7C4B1B6B642B38BF6423A367D8F814
:1021900000100320C1F3400106F000FA01210520E0
:1021A00006F0FCF9744B99F804B01A8C734B0720B5
:1021B00093FBF2F3642B38BF64231BF10001C4F8D6
:1021C000143118BF012106F0E9F999F805A008209B
:1021D0001AF1000118BF012106F0E0F999F8083062
:1021E000002B40F0588199F80930002B40F05381C2
:1021F0003968C1F38041BBF1000F03D1BAF1000F80
:1022000000D15146092006F0C9F90121042006F049
:10221000C5F995F86419062006F0C0F901210A20D5
:1022200006F0BCF9D8F800100B20C1F3800106F0CD
:10223000B5F9D8F800300C2013F0140F14BF0121A9
:10224000002106F0ABF939680D20C1F3802106F0BA
:10225000A5F939684B0507D5337A083B012B9CBF9C
:102260004FF4FA63C4F8B4320E20C1F3004106F013
:1022700095F94FF4804006F051FC68B10022032329
:1022800090F902004FF48041009301924FF4E13342
:1022900006F08EFAC5F8200AD5F8203A63B101217C
:1022A000022385F8241A85F8251A85F8261A0F20A6
:1022B00085F8273A06F072F995F8C53463F07F0384
:1022C00085F8C5341FB0BDE8F08F202323804FF47C
:1022D0008073AFE64023F9E74FF40073F6E700237D
:1022E0005BF8232001320BD10133042BF8D14C468B
:1022F000B1E632F83330002B7EF4F0ADFEF7E6BDE8
:1023000009F1010AA146F2E71740EF00E43A002084
:10231000D43A002060230020743C00209A1C002046
:10232000981C0020ED260020F9350020221A0020FC
:10233000341A0020FE350020C80F0020CC0F0020EA
:1023400018230020FC0F0020CDCCCC3E0C10002028
:10235000681800209BAE000838310020C41500200A
:1023600058120020DC000020C01500202041002071
:1023700018250020A82200203241002040420F00F2
:102380000022464B00B21A7014F02EFB444914F0A0
:102390007FFB0746B4F9A00614F026FB404914F071
:1023A00077FB0646B4F9A40614F01EFB3C4914F072
:1023B0006FFB3C490546384614F062FA0AF08FFB81
:1023C000814638460AF08BFB36490746304614F002
:1023D00057FA0AF084FB804630460AF080FB314908
:1023E0000646284614F04CFA0AF079FB8346284644
:1023F0000AF075FB49468246584614F049FB4946A7
:102400000290504614F044FB59460390384614F0AD
:102410003FFB51460490384614F03AFB4146059084
:10242000584614F035FB204D5146286008F1004015
:1024300014F02EFB04996860AE60304614F028FB5F
:10244000039914F01DFA0599E860304614F020FB5A
:102450000146029814F012FA4146286107F1004043
:1024600014F016FB02996861304614F011FB014626
:10247000059814F003FA0399A861304614F008FB9C
:10248000049914F0FDF94946E861404614F000FB58
:102490002862FEF7C2BE0121ADE600BF1D04002088
:1024A00035FA8E3CDB0FC93FC0270020000000003A
:1024B0002DE9F047B0F908308CB0DDB2382D064672
:1024C0000C460B8100F0CC8100F2B380042D00F0AB
:1024D0004A8171D8022D00F0318100F23581012D41
:1024E00000F01D815C2D00F0E38401F22D83362D78
:1024F00001F0C28401F2AB822C2D00F0888301F23E
:102500005A82222D01F0CA8401F247820A2D00F07E
:10251000AA82742D336800F00C85772D00F01685A3
:10252000472D40F0208572683046D51A0AF022F90E
:10253000052D074640F2138530460AF031F9002692
:10254000054694E80C009B1A103BAF4AAB42A846E4
:10255000B8BF9DB2D3683946DB1B9D42204688BF79
:102560009DB291460AF031F93EB9294620460AF05B
:1025700040F923685A1C22601E70D9F80C307A1971
:102580009A42D4F800A088BFDD1B0BF085F82A46DC
:10259000514638460BF0DCF8236803442360002ED4
:1025A00000F0AC800022804540F3A8802368013011
:1025B000591C21601A70F6E7202D00F0758111D8A2
:1025C000052D8FD120460B2290490AF0F4F82046C1
:1025D00008228F490AF0EFF807228E4920460AF0B8
:1025E000EAF88BE0242D00F0DE80282D7FF47AAF0E
:1025F00001250B68884E5A1C0A601D700B68204626
:102600005A190A6006221A700B685A190A600A22BF
:102610001A700B685A190A601D7031880AF0E9F8BF
:10262000718820460AF0E5F868B265810CB0BDE813
:10263000F087802D64D02FD8522D00F0548107D818
:10264000442D7FF44FAF002A58D0744B136055E0EF
:10265000542D00F04E816E2D7FF444AF704B0A680C
:102660001B88511CFF2BA8BFFF236E4D21601370E8
:10267000A968204681F3100189B20AF0BAF86A4BC2
:10268000204619880AF0B5F82968204601F30F01A1
:1026900089B20AF0AEF831E0822D00F08A800FD3C3
:1026A000A02D70D0FE2D7FF41DAF00255F4E36F8B3
:1026B0001510204601350AF09CF8042DF7D11DE0D5
:1026C0004FF6FF765A4B0A2519689F68B142A8BF9A
:1026D0003146236821EAE1715A1C226089B2204602
:1026E0001D700AF086F805FB07F1B142A8BF31461C
:1026F00021EAE17189B220460AF07BF8012593E7CF
:102700000A684C4B511C1B8821600A21FF2BA8BF73
:10271000FF2311702268511C21601370EEE70B68D3
:102720005A1C0A6000221A700B685A1C0A601D703D
:102730000B685A1C0A6024221A7075E704223E496D
:1027400020460AF038F8D9E70B6801255A1C0A60C0
:1027500002221A700B685A1C0A601D700B685A1905
:102760000A600022E8E72A46344920460AF023F8A6
:10277000334B204619780AF03CF823685A1C226033
:1027800000221A70BAE72F4B204619680AF01DF88C
:102790002D4B204619680AF018F82C4B2046196872
:1027A0000AF013F8AAE72A4B204619680AF00DF838
:1027B000A4E7284B20461A780B681A4D591C216053
:1027C0001A70254BD9880AF014F8154B22681B881B
:1027D000511CFF2BA8BFFF2321601370A96820465E
:1027E00081F3100189B20AF004F82968204601F348
:1027F0000F0189B209F0FDFF184B1A782368591CA4
:1028000021601A707AE700BF38040020FEBE01087C
:102810000ABF010813BF01083C1100209BED00080E
:10282000221A002018230020F4350020EC2200207A
:10283000FC0F0020C80F0020F4BE0108F9BE0108FB
:10284000E40A0020E8F7FF1FECF7FF1FF0F7FF1F77
:1028500068180020341A0020FE350020F9350020C9
:1028600001250B685A1C0A601D700B685A190A6012
:1028700005221A700B685A190A600A221A700B682E
:102880005A190A6000221A70B14B2268197850193F
:1028900020601170226859785019206011709A7860
:1028A00023685919216047E7AA4D0B686A78591CBB
:1028B00021601A7023682A78591C21601A702368D5
:1028C000AA78591C21601A70E988204609F091FF06
:1028D00023682A79591C21601A7023686A79591C67
:1028E00021601A700AE70B685A1C0A6000221A70ED
:1028F00004E70B685A1C0A6000221A700B68591C06
:1029000021601A70FAE600264FF6FF78924FDFF842
:1029100084920196029603960496F157481C0BD0B8
:1029200048FA06F3DA0707D5B9F800303341DB0778
:1029300002D503A80AF043FD01360B2EEDD1002687
:102940000FF20429D9E9008932464046494613F07E
:10295000E3FA002100F0010050EA010307D0F0B2D1
:102960000FF06EFD18B1314603A80AF028FD0136BC
:10297000242EE9D1794BDFF820821B78DF074FF056
:1029800000073E4642BF039B43F0010303933946D1
:1029900040460AF020FD48B1394603A80AF01BFD65
:1029A00018B1314601A80AF00AFD01360137242F7B
:1029B000EDD16B4B2046B3F8501009F01AFF694B6C
:1029C00020461988684F89B209F013FF674B2046EB
:1029D00019684A01C1F3400302F020021343C1F316
:1029E000800243EA4203C1F3C00243EA8203C1F317
:1029F000401243EAC20301F01001194309F0F9FE45
:102A0000042220460DEB020109F0D5FE23683A7836
:102A1000591C21601A70564B204619886429A8BF9A
:102A2000642109F0E6FE962D18D123685A1C226015
:102A300003221A7023687A78591C21601A700822C0
:102A4000193E96FBF2F2236882F30402591C2160BE
:102A500020461A7002A909F0AEFE4FE6002120467A
:102A600009F0C7FEEBE7434813F04EFA00233E4956
:102A700098427FF743AE5A18157922680133561CE5
:102A800026601570F4E710223B49204609F093FEBA
:102A900034E600251826394FDFF8008106FB057360
:102AA000597C31B92046013509F0A3FE082DF5D136
:102AB00024E658F8250014F0DBFF81B2F2E736F87F
:102AC0001510204609F095FE01353B789D42F6DB56
:102AD00014E62B4D2046298809F08BFE6988204694
:102AE00009F087FE0A23B5F90410204691FBF3F1A3
:102AF00089B209F07EFE01E6224B2046196809F0F2
:102B000064FE214B2046198809F073FEF6E51F4D3F
:102B10002046298809F06DFEA988204609F069FE43
:102B20002989204609F065FEE8E5194B2268997865
:102B3000501C206011705A782368591C21601A704B
:102B4000DCE500BFAFF3008090E33FF40800000035
:102B500038110020FE35002022A20108A4350020F3
:102B6000DC000020B83B00200816002018250020BB
:102B70002E1600200C160020442300208025002063
:102B80008C310020A01000201C150020BC0C00205F
:102B900070110020F6350020CC0C0020F822002017
:102BA0000021AC48036801EB41029D5C23680131C0
:102BB0005E1C26601D7003680A2913445D78236833
:102BC00003F1010626601D70036813449A78236898
:102BD00003F1010525601A70E4D18FE52168481CD6
:102BE00020600A7013F8012F002AF7D186E501252D
:102BF00023685A1C22601D7016E5974D2046A9894E
:102C000009F0F7FD6989204609F0F3FD76E5934D5B
:102C100023682A7A591C21601A70A98B204609F072
:102C2000E8FD298B204609F0E4FD698B204609F078
:102C3000E0FD2368EA7C591C21601A70E98C20466B
:102C400009F0D7FD298D204609F0D3FD2368AA7F1E
:102C5000591C21601A70236895F82020591C2160A6
:102C60001A70A98C204609F0C4FD2368EA7A591C21
:102C700021601A70E968204609F0A7FD23682A7CC4
:102C8000591C21601A70236895F82120591C216075
:102C90001A7033E5724D23682A78591C21601A7026
:102CA00023686A78591C21601A706988204609F0E7
:102CB000A0FD23682A79591C21601A70E9882046F2
:102CC00009F097FD23682A7A591C21601A7015E5CE
:102CD000236816F81510581C06EB45022060197081
:102CE0005178204601EB810101EB810101F2EE21D7
:102CF00089B209F07EFD01353B789D42E8DBFDE4B9
:102D0000564B5A7D2368591C21601A70F6E4002541
:102D1000544E56F825102046013509F056FD202D59
:102D2000F7D1EBE44F4D002306272846002107FB8F
:102D300003F6226802F1010EC4F800E01370226865
:102D400002F1010EC4F800E011708A192A4492F8C9
:102D5000C0E02268013102F1010C0629C4F800C06C
:102D600082F800E0E5D10133062BDFD10022216893
:102D70004D1C25600B7021684D1C25600A70811860
:102D800091F8E450216801324E1C0B2A26600D7028
:102D9000EDD123685A1C226007221A7023685A1C3E
:102DA000226000221A70236890F8F020591C2160DC
:102DB0001A70A3E40AF092FB002814BF0322022237
:102DC0002368294D591C21601A702988204609F072
:102DD000FCFCE968204609F0F8FC0AF05FFB0146BC
:102DE000204609F0F2FC89E4012523685A1C226080
:102DF0001D701E4B2268997850192060117022684E
:102E000019785019206011705A7849E50025236817
:102E100029465A1C22601D70236820465A1C2260D5
:102E20001D7023685A1C22601D7009F0CEFC2946D3
:102E3000204609F0CAFC61E40D4D2046298809F0BE
:102E4000D8FC6988204609F0D4FCA988204609F0FE
:102E5000D0FC53E410250020F02600203836002056
:102E6000B83100202434002038040020D43A002057
:102E7000A42D0020AB4B1A782368591C21601A70CE
:102E8000A94B9A782368591C21601A70A74B9A782D
:102E90002368591C21601A7030E4B278591C2160F3
:102EA0001A70A34B1A782368591C216000F010BED9
:102EB0009C4E236872799F4D591C21601A702B68B3
:102EC0002046198C09F095FC2B682046598C09F096
:102ED00090FC7189204609F08CFCB189204609F0EC
:102EE00088FC2B682046998C09F083FC2B682046CF
:102EF000D98C09F07EFCF189204609F07AFC318AF0
:102F0000204609F076FCFFF7F9BB874BDA78236897
:102F1000591C21601A70884B1A782368591C21604B
:102F20001A70824BDA782368591C21601A70FFF7F7
:102F3000E5BB72689A420FBF00215A1C32601978B3
:102F40007E4A20460BF05EFFFFF7D8BB72689A42BC
:102F50001DBF5A1C326019780021794AF1E7012619
:102F60008025FFF7EEBA292D2AD0392D1ED0212D2C
:102F700035D15A1C32601A46724D12F8021B304687
:102F8000697032605A782A70DA1C32609B78AB70B4
:102F900009F006FC3368E8805A1C32601A4612F8C1
:102FA000021B297132605B786B7105E05A1C32603C
:102FB0001A780A2A00F0AE874FF0FF35FFF734BBCE
:102FC0005A1C32601B780A2BF6D1304609F0E8FB18
:102FD0005D4D2880304609F0E3FB6880ECE77768B8
:102FE0005D2DA7EB030700F0B78300F25C81352D60
:102FF00000F0B58200F2B2802B2D00F067842FD84C
:10300000232D00F0948217D80B2DD5D10021112249
:103010004E4816F0F8FF102F4FF0000328BF10277E
:103020004B49BB42BFF46AAB3268501C3060107829
:103030005A1810710133F4E7252D00F03C84272D38
:10304000BAD1304609F0ACFB424D2860304609F059
:10305000A7FB6860304609F0A3FBA860FFF74EBBF2
:103060002F2D00F05D844FD82D2DA5D15A1C326034
:103070001B78394D30462B7209F092FBA8833046FD
:1030800009F08EFB2883304609F08AFB3368688399
:103090005A1C32601B78082FEB747FF62FAB30463A
:1030A00009F07EFBE884304609F07AFB0C2F288576
:1030B0007FF624AB336830465A1C32601A4612F849
:1030C000021BA97732605B7885F8203009F068FB35
:1030D000102FA8847FF612AB336830465A1C32603A
:1030E0001B78EB7209F046FB3368E8605A1C3260CB
:1030F0001A78162F2A747FF601AB9A1C32605B781F
:1031000085F82130FFF7FABA312D00F02284332DF3
:103110007FF452AF5A1C32601A780F4B5A75FFF782
:10312000EDBA00BFBA3B0020F02600206411002059
:10313000582C0020102500208827002079ED000859
:10314000DDEC0008FE3500203C1100200C160020AC
:1031500008160020BC0C002038360020482D00F056
:10316000A68339D83C2D3FF4C9AA23D8372D7FF444
:1031700023AF0723B7FBF3F3C3EBC302BF1A7FF4FC
:103180001BAFDFF874A35FFA83F8FBB298453FF4F6
:10319000B5AA002533685A1C326093F900300AEB57
:1031A000C50999F902209A4200F0DE860135042D06
:1031B000F5D101E73E2D00F0AE81412D7FF4FCAE4C
:1031C0000023C2493268501C306012785A540133CF
:1031D000082BF7D1FFF792BA4E2D00F07E8320D84E
:1031E0004C2D7FF4E9AE5A1C32601A46B84D12F8E5
:1031F000021B3046297032605B786B7009F0D0FAA0
:10320000336868805A1C32601B7830462B7109F095
:10321000C7FA3368E8805A1C32601B782B72FFF7BC
:103220006DBA512D00F02E835B2D7FF4C5AE5A1C74
:1032300032601A46A74D12F8021BA74FA9703260E0
:103240005978A64A30461170DA1C32609A783A7181
:103250001A1D3260DB78042BA8BF0423BB7009F071
:103260009FFA96E80C009B1A012B388003DD30464C
:1032700009F096FAF881336872689A4206D05A1CAF
:1032800032601B78003318BF0123EB710BF0DEFEB8
:10329000336872689A423FF431AA5A1C32601B7834
:1032A000FB70FFF72BBAD42D00F0C98100F28980A2
:1032B000CC2D00F07B8168D8612D00F0928241D83E
:1032C0005F2D7FF479AE304609F06AFA304609F096
:1032D00067FA304609F064FA3368814D9A1CD5F8D4
:1032E000008032605A78304688F82F20DA1C32602D
:1032F0009A7888F83A201A1D3260DA78073388F80D
:103300003B20336009F04CFAA8F83E003046D5F86F
:10331000008009F045FA112FA8F83C002B460CD983
:1033200032682868511C3160114611F8025B80F840
:1033300031503160527880F8322018680FF04EF921
:10334000FFF7DCB9C82D00F09880CA2D7FF434AEA9
:10335000634B1868034600F11E0532680333511CA5
:103360003160114611F8027B03F8037C316051781B
:1033700003F8021CD11C3160927803F8012C9D42A5
:10338000EBD10FF02BF9FFF7B9B9CE2D00F06E821B
:10339000C0F06182D02D00F05182D22D7FF40CAEAE
:1033A0005A1C3260187806065ED44E4B1B78DD0737
:1033B0003FF5A4A9032828BF00200BF07FFDFFF7ED
:1033C0009DB9DC2D00F0B68125D8D92D00F08E8175
:1033D00013D8D62D7FF4F0AD0025434FDFF81C81C4
:1033E0003B789D42BFF68AA9304609F0D9F913F01F
:1033F000F7FA48F825000135F2E7DA2D00F085816B
:10340000DB2D7FF4D9AD364B4A223849186814F0C9
:10341000C9F9FFF773B9EF2D72D014D8DD2D00F084
:10342000AB82DE2D7FF4C8AD304609F0B9F92A4DE4
:103430002882304609F0B4F96882304609F0B0F9C4
:10344000A882FFF75BB9F22D00F02581FA2D7FF4F9
:10345000B3AD244B1B78DB073FF5AEAD0BF044FD5D
:103460000BF06EFEFFF74AB900F07F00032828BF7B
:10347000002012F0B7FCFFF741B9C7F34707122F3E
:103480003FF69AAD00250DF10C08BD420CDB002380
:10349000174A03A99F420ED10021154A122B10D1C1
:1034A0000125144BFFF7A7BB304609F079F928F83E
:1034B00015000135E9E731F8130022F81300013354
:1034C000E8E722F813100133E8E700BF38360020A0
:1034D000B8310020BA3B002068230020582C00207F
:1034E00010250020A4350020F422002054B001084B
:1034F000EA290020E8290020324100205825002038
:10350000304609F04DF9C04DA881304609F048F920
:103510006881FFF7F3B85A1C32601A46BB4912F8AB
:10352000020B887032605B784B70FFF7E7B85A1C6B
:1035300032601D78132D3FF63FAD00210C279A1CF9
:1035400032605A78DFF8ECE207FB01E090F808C03F
:10355000944500F0EE8401312429F5D12CE55A1C64
:10356000326019780E293FF627AD9A1C32605D78DB
:10357000032D3FF621AD06224A43A54881184D711F
:10358000DD1C35609D7885541A1D3260DA784A70EA
:103590005A1D32601A798A709A1D32605A79CA703F
:1035A000DA1D32609B790B71FFF7A8B8092F7FF6FF
:1035B00003AD98495A1C0D6832601A4612F8020B86
:1035C0008846287032605B78681DAB700023022B40
:1035D0000CBF4FF0FF0E4FF0640E316801334A1CF0
:1035E00032600A787245A8BF7246032B00F8012B9F
:1035F000EDD18B1C33604B783046642B28BF64239D
:103600002B72CB1C33608B78EB700B1D3360CB7847
:103610002B7109F0C5F80A2F68810CD03368D8F8EF
:103620000020591C316019780B2F51721FBF991C53
:1036300031605B7853700EF053FFFFF75FB80F2FC8
:103640007FF4BAAC5A1C32601D78072D3FF6B4AC3B
:103650000C27304609F0A4F86F43DFF8DC8108EB53
:103660000705A880304609F09BF8E880304609F04D
:1036700097F8336828815A1C32601A4612F8021BE8
:103680003046A97232605B78EB7209F073F848F843
:103690000700FFF733B85A1C32601A780F2A3FF63A
:1036A0008BAC991C31605D785B48C2EBC2028554DB
:1036B0008118DA1C32609A784A701A1D3260DA7802
:1036C0008A705A1D32601A79CA709A1D32605A790E
:1036D0000A71DA1D32609A794A7103F10802326088
:1036E000DB798B710CF072FFFFF708B8304609F0F8
:1036F00057F84A4D2880304609F052F86880304625
:1037000009F04EF8A880FEF7F9BF19465A1C32603E
:1037100011F8020B424A10703160597830465170EE
:10372000D91C31609B78937009F03AF83B4BD880F4
:10373000FEF7E4BF5A1C32601A463A4912F8020BEF
:10374000087032605978304A9170DA1C32609A7889
:10375000354B9A70FEF7D2BF5A1C32601B78334D3E
:10376000DFF8C0803046D5F8009088F8053009F0C1
:1037700017F8A9F820003046D5F8009009F010F8A5
:10378000052FA9F8220023D9304609F009F8A8F836
:103790000A00304609F004F8A8F80C003046D5F8C5
:1037A000009008F0FDFFA9F824003046D5F80090FD
:1037B00008F0F6FF0D2FA9F8260009D9304608F0C9
:1037C000EFFFA8F80E00304608F0EAFFA8F8100056
:1037D0000BF03CFC11F028FE28680EF0BDFFFEF750
:1037E0008DBF5A1C32601A46074912F8020BC87086
:1037F000326059780E4A1170DA1C32609A780A4B9E
:10380000DA70FEF77BBF00BFF026002070110020A9
:103810001C190020AC2D0020862B0020A42D002098
:1038200080100020BA3B00206411002010250020E9
:10383000882700209CAE0108F82B0020B44B1B7891
:10384000D8073EF55BAF0BF04DFE0BF04DFB0BF0D8
:1038500077FCFEF753BFAE4B1B78D9073EF54EAF52
:103860004FF4C872AB4B1A80FEF748BFA84B1B78C9
:10387000DA073EF543AFA84A137843F00403137008
:10388000FEF73CBFA54A1278012A3EF637AF19462B
:103890005A1C326011F8020BA14A907031605978BD
:1038A0001170D91C31609B785370FEF727BF09F067
:1038B00031FFFEF723BF00239A4D30462B6008F0FE
:1038C00059FF2B6818432860FEF718BF5A1C326056
:1038D0001A78954B1A70FEF711BF5A1C32601F7888
:1038E000112F3FF669AB9A1C32605B788F4D3046E2
:1038F00005F8173008F054FF40F6CA039842A8BFF5
:10390000184640F2EE239842B8BF18461923A0F299
:10391000EE2090FBF3F005EB47056870FEF7EEBE76
:10392000834D05F14007304608F03AFF3368A5F8AB
:1039300080005A1C32601A4612F8021B043585F8C2
:103940007E1032605B7885F87F30AF42EBD1FEF7B6
:10395000D5BE5A1C32601D781F2D3FF62DAB052FAA
:103960007FF42AAB304608F005FF714B43F8250081
:1039700011F0CCF8FEF7C2BE5A1C32601A4612F89B
:10398000020B3260DA1C597832609A7811F03EF8F6
:1039900000287EF4B3AEFFF70FBB262D3FF4B7A887
:1039A0002A2D7EF4B6AD604B1A782368591C21602D
:1039B0001A70FEF7A3BE302D3FF4A9A91BD82E2DF7
:1039C0007EF4A7AD5A4D05F14006B5F880102046AB
:1039D00008F00FFF236895F88220591C21601A70A7
:1039E000236895F883200435591CB54221601A706C
:1039F000EBD1FEF783BE322D3FF482A9342D7EF445
:103A000088AD4C4B03F15A0122685879551C25604A
:103A1000107022681878551C25601070226858783C
:103A2000551C2560107022689878551C2560107010
:103A30002268D878551C25601070226818790633E2
:103A4000551C994225601070DED1FEF757BE462DF9
:103A50003FF4B0A919D83B2D3FF4C9A808D83A2D96
:103A60007EF457AD0021204608F0AFFEFEF746BEBB
:103A70003D2D3FF45AA8402D7EF44BAD08222E492F
:103A8000204608F098FEFEF739BE4F2D3FF4BEA940
:103A90000AD84B2D3FF4FEA84D2D7EF43AAD0025FB
:103AA000264F224EFFF728B9502D3FF49DA95A2DDD
:103AB0007EF42FAD224E2368F278002A3FF4EDA960
:103AC0005A1C226008221A7023685A1C22600122A4
:103AD0001A701C4D23682A79591C21601A702368BA
:103AE000AA78591C21601A702988204608F081FEA6
:103AF000E989204608F07DFE2368F279591C21608F
:103B00001A702368EA78591C21601A70FEF7F6BD16
:103B1000A43500209A1C0020ED2600206023002000
:103B2000D43A0020681800201C250020E92A002033
:103B3000243400201C19002038360020D829002009
:103B4000BA3B002068230020702D3FF429A800F222
:103B5000E180672D3EF497AF00F28A80602D3FF43C
:103B6000D4A94FD85E2D7EF4D4AC0021204608F0B5
:103B700040FE0021204608F03CFE0021204608F0CF
:103B800038FE2368AE4D5A1C226000221A702B6842
:103B900093F82F102368581C206019702B6893F835
:103BA0003A102368581C206019702B6893F83B105A
:103BB0002368581C2060197023682046591C216016
:103BC0001A702368591C21601A702368591C2160DF
:103BD0001A702B68D98F08F00CFE2B682046998F3D
:103BE00008F007FE2B6893F831202368591C2160E8
:103BF0001A702B6893F832202368591C21601A70C0
:103C0000FEF77CBD652D3EF47EAE662D7EF481AC64
:103C10008C4E0025328AB2F5007F8CBF0427012725
:103C20007319596B204691FBF7F1043589B208F0FE
:103C3000E0FD0C2DF4D10125834E844F396A56F8EE
:103C4000250012F0D9FF13F013FF013581B2204691
:103C500008F0CFFD042DF1D100257D4E36F825105A
:103C60002046013508F0C5FD032DF7D1FEF746BD0E
:103C70006C2D3EF42EAF0AD8682D3EF40AAF692DA4
:103C80007EF447AC0025734F734EFEF71EBF6D2DBB
:103C90003EF432AF6F2D7EF43CAC704D2B681A7839
:103CA0002368591C21601A702B689A782368591C64
:103CB00021601A7000232A681A445179226801335E
:103CC000501C032B20601170F5D12B6820461A7A06
:103CD0002368591C21601A702B68DA782368591CF4
:103CE00021601A702B681A792368591C21601A7098
:103CF0002B68598908F07DFD2B685A7A2368591C76
:103D000021601A702B685A782368591C21601A7038
:103D1000FEF7F4BC7E2D3FF4ADA825D8782D6DD0EC
:103D200005D8752D7EF4F5AB4D4BFEF75BBF7C2DB2
:103D30003FF482A87D2D7EF4ECAB4A4B22681978C3
:103D4000501C2060117022685978501C206011703E
:103D50009A7823682046591C21601A70424BD988F2
:103D600008F047FDFEF7CABC962D3EF4CCAD14D842
:103D70007F2D3EF4D7AF832D7EF4CBAB3B4D204659
:103D8000298A08F036FD698A204608F032FDA98AA2
:103D9000204608F02EFDFEF7B1BCF02D3EF42DAF0D
:103DA000F12D7EF4B6AB324B03F170012268187826
:103DB000551C2560107022685878551C25601070BD
:103DC00022689878551C256010702268D878551C98
:103DD0002560107022681879551C256010702268C3
:103DE0005879551C25601070226898790733551C46
:103DF0008B4225601070D9D1FEF780BC1D4D05F1B6
:103E00006006A988204608F0F4FCE988204608F0FE
:103E1000F0FC2989204608F0ECFC2368AA7A591C9A
:103E200021601A702368EA7A591C21601A7055F8CB
:103E30000C1B204608F0C9FCB542E2D1FEF75EBC7F
:103E400010250020A822002020410020CC3B00208B
:103E500088330020D8290020CC350020AC2D00204C
:103E60002CA2010880100020A42D0020682300202F
:103E7000862B0020F82B00204B4D4C4F05F12006DF
:103E8000002395F90220D957914226D00C33302BCC
:103E9000F9D10835B542F3D1FEF730BC444D05F1F8
:103EA000500628780AF09AFF2368027A591C21608C
:103EB0001A7023686A78591C21601A702368AA78DE
:103EC000591C21601A702368EA780435591CAE42E7
:103ED00021601A70E5D1FEF711BC23682046591CF9
:103EE00021601A70298808F084FC2368EA78591C3C
:103EF00021601A7023682A79591C21601A7023687E
:103F0000AA79591C21601A7023686A79591C2160AA
:103F10001A70BEE79A1C32605978264A1170D91C73
:103F2000316099785170191D3160DB789370FFF71B
:103F300043B801781E4A002002F82510D91C3160D0
:103F4000997802EB85025170191D3160D978917012
:103F5000591D31601B79D3700EF038FA164B80F082
:103F600001001870FEF7CABB89F80230304608F02D
:103F700017FC33682AF8350019465A1C326011F8CC
:103F8000022B013789F8032031605A7889F8042020
:103F9000DA1C32609A7889F806201A1D3260DB78C4
:103FA00089F80530FFF7F1B8324100205841002070
:103FB0007C18002038110020000000202DE9F04F6F
:103FC000B34B9DB01B780690012B07D1B149B24A83
:103FD0000968C9691180B14909885180B04D2A78B2
:103FE000002A00F0D384072B40F0F8810DF054FB39
:103FF0000790AC4F3B68059713F4806F05D0AA4833
:10400000836813B100F144019847A84BA8491B6885
:10401000B1F906405A890891944280F2E2814FF04A
:104020007E536B6095F90C304FF00009002B14BFE4
:1040300001234FF0FF339F4A95F809B0168B95F88E
:1040400008A09D4F04930992089B33F91980A8EBAF
:1040500006000028D8BFA6EB0800B0F5FA7F82F270
:104060003D83B9F1020F02F03F83824580F2CC819B
:10407000A0EB0A0012F0B8FCB04547F82900C2F2E4
:10408000418309F10109B9F1030FDDD1059B1F68D7
:1040900017F4805800F0BA81B4F5FA6F2046A8BF33
:1040A0004FF4FA60B0F57A7FB8BF4FF47A70A0F59C
:1040B0007A724FF0640C92FBFCF38049581C31F982
:1040C00013E031F91000DFF8F091A0EB0E016FF072
:1040D000630000FB0320484390FBFCF0704400B2F7
:1040E00012F082FC8246C9F80C00B8F1000F1DD016
:1040F0001D200EF0A5F9C8B1714BDB78B3B9714939
:10410000504612F0BBFB12F09FFE4FF47A7300B2E0
:10411000000390FBF3F3C6F5FA6000B2584340F396
:104120000F30304412F060FCC9F80C00664B1E885A
:1041300072063BD5654BB3F904000A2390FBF3F0FC
:10414000EB89C01A00B212F04FFC614912F0A0FCDA
:104150006049054612F094FB08F0C1FC83462846EE
:1041600008F0BDFC544D81462B685946184605930E
:1041700012F08EFCD5F804A004905146484612F087
:1041800087FC049A0146104612F078FB59462860D5
:10419000504612F07DFC059B82461946484612F0B7
:1041A00077FC0146504612F06BFB68604A4B3C4D71
:1041B0001B6813F0140F1AD016F4027F17D0474B68
:1041C000DFF8F490197811F0100100F034812B7CA5
:1041D0006869002B0CBF01234FF0FF33584312F0E6
:1041E00003FCD9F8041012F04BFBC9F804003C4B57
:1041F000DFF8C0901A780593A2B1B9F81A30A3423B
:1042000010DB384B1B78012B01D0192B02D1364A19
:10421000927B3AB90E2B05D0082B1FBF0023264AEC
:10422000EB63936095F84240002C65D0B30763D0F0
:104230002E4B2F491E6A304612F0D2FD002840F066
:104240004A81304613F08CFC696C12F021FC13F0AB
:104250000FFCB0F5617FA8BF4FF4617012F0C4FB92
:10426000244912F015FC08F03AFC0646204612F0EC
:10427000BBFB314612F00CFC13F0FAFB00B212F05B
:10428000B3FB0D4C0146E06812F0FAFAE06033E04F
:1042900014250020A41B0020EC2200202E16002054
:1042A000781000200C360020CC3B0020AC2D0020E4
:1042B000CC35002038360020381A0020B02D0020E0
:1042C0001036002000007A44F63500208C310020A2
:1042D00035FA8E3CDB0FC93F18250020ED26002063
:1042E000000000201C2500207A2C00204C310020EA
:1042F0008FC2753CD06D393A95F848A099F81F40A7
:10430000BAF1000F5CD0794B0420D3F8EC6044F68E
:1043100020639E42A8BF1E46B6F57A7FB8BF4FF411
:104320007A76B6B2A5F84A600EF08AF808B9FF00AE
:1043300046D54FF47A73B6FBF3F6642393FBF6F697
:10434000DFF8BCB1142EA8BF1426DBF80030B8F19A
:10435000000F00F0C280DF8E7F086549EB6CD1F85A
:104360000C805A1CEA6405EB430340460892049310
:1043700012F06AFD089A049BB242A3F85000A4BF51
:104380000023EB64EB6C05EB4303B3F9500012F030
:104390002BFB0146404612F071FA12F055FD00B2B7
:1043A0000028B8BF4042B84240F39A80DBF80030A2
:1043B000188F12F019FB4F4912F06AFB059B5860E9
:1043C00099F81E30002B00F0BE81022B00F09A807D
:1043D000032B00F08C81484B588898E0002307930A
:1043E00007E6B4F5FA6F187ABFBFA31A5843C2F5AF
:1043F000FA6290FBF2F0C0F1640012F0F5FA3F4966
:1044000012F046FB68600DE6002033E6099B598BED
:104410008C420EDBB4F5FA6F2046A8BF4FF4FA6069
:104420004FF47A72401A5043C1F5FA61B0FBF1F2D1
:104430003FE60846F4E7B5F9183095F80BE0A87A9E
:10444000E21ABEF1000F2BD0002AB8BF52428242BE
:1044500010DD01229C42E96185F82020C8BF40425E
:1044600012F0C2FA0146D9F80C0012F009FAC9F8A4
:104470000C00BCE695F820201AB1AA6A85F8201035
:104480006A6268691844B0F5FA6FA8BF4FF4FA6021
:10449000B0F57A7FB8BF4FF47A7012F0A5FAE6E76C
:1044A00082EAE271A1EBE271814209DD022192FB15
:1044B000F1F2EA62012285F8302085F82020E0E759
:1044C00095F82020002ADCD0AA6A85F830E06A62DC
:1044D00085F820E0D5E70020D0E6B3F936703CE758
:1044E0004FF07E53059A53606AE700BFDC0000205E
:1044F000381A00206F12833AD82900200AD7233CAB
:1045000010250020B5F84A0000F57A7080B2023418
:10451000E4B2BAF1000F00F0FF80002800F0FC8048
:104520008D4B00261B688D4FB0FBF3F000B2A5F851
:10453000780012F059FA01464FF07E5012F05CFB01
:104540008046DFF8209207F1100AA642C0F2D78019
:10455000834B1B78092B11D1824B834E186813F0C3
:1045600087FA824B3080D3F8EC004FF47A7390FBDB
:10457000F3F012F039FA12F067FC7080B5F9783078
:10458000002B40F3E28000273E46DFF81482DFF87C
:10459000D4A1A8F11009A742C0F2C48095F8483010
:1045A0000024002B18BF0226714BDFF8F891D3F8D6
:1045B00000806B4B1B78089308F105030993B44204
:1045C00040F3F280089B6B4C092B07D1664EB4F880
:1045D0007830606BB38012F037FCF080664B93F854
:1045E0002160002E60D01E200DF02AFF00285BD035
:1045F000624B1B88580657D494F8B430B34214D099
:1046000084F8B460304612F0EFF95D4912F040FAD8
:104610005C49064612F034F908F061FA5A4B98608A
:10462000304608F05CFAC4F8B800059B6E6BD3F80E
:1046300008903046494612F02BFAD5F83C80D5F860
:10464000B87082463946404612F022FA014650467A
:1046500012F014F94D49824612F0C2FB08B9DFF896
:104660002CA14B49504612F0C5FB08B9DFF820A138
:1046700049464046C5F834A012F00AFA3946804649
:10468000304612F005FA0146404612F0F9F83F496B
:10469000064612F0A5FB00B93C4E3D49304612F0EB
:1046A000A9FB00B93A4EEE63002384F84830394B39
:1046B0001B78002B40F05D81374DAA78002A00F06E
:1046C0005881364C2378013B0D2B00F23F81DFE807
:1046D00013F0110124012E0123023D013D013D0291
:1046E00051026C0589059A05B905C405CD0599F8EF
:1046F0002000C0EB401300EB8300C00006E75AF82F
:10470000261059F8260012F0B9F8414612F0C0F907
:1047100047F82600013618E7B5F87830013BA5F8D0
:1047200078302BE758F8270059F8271012F0A8F82E
:10473000022F3E46B8BF022648F827004AF8270055
:10474000F6B2013727E7A5F8783095F84830002B06
:10475000ADD0002622E700BFF8240020F41000208E
:1047600014250020381A0020EC220020DC00002054
:10477000AC2D00207810002038360020F6350020BF
:1047800035FA8E3CDB0FC93F0000002000C0F94421
:1047900000C0F9C4C4260020D43A002060230020C1
:1047A000041100200AD7233C022C15BF98F8000002
:1047B00098F8010098F802B098F809B012F014F9CE
:1047C000494612F065F94FF08041074612F01CFB94
:1047D00060B14FF08041384612F050F8AA4912F00B
:1047E00057F90146384612F04BF80746A3000493E8
:1047F000A64BA74953F8240012F04AF920F00043D1
:10480000A44A0493049B42F824000C32824642F8E6
:104810002430BBF1000F20D0584612F0E5F849468D
:1048200012F036F983465146504612F031F9049998
:1048300012F02EF9594612F02BF959460A904FF012
:104840007E5012F01BF80A9A0146104612F018F832
:104850000146504612F01CF982468F49384612F044
:1048600017F9514612F014F9099B074613F8010B8A
:10487000099300B312F0B8F8494612F009F9049907
:1048800012F006F98549824612F0BEFA68BB002193
:10489000504612F09BFA50BB51464FF07E5011F03B
:1048A000EDFF01464FF07E5012F0A6F90146384662
:1048B00012F0EEF80746089B0C2B05D1384612F093
:1048C000C3FA774B23F814007649384612F088FA79
:1048D00000B9744F7449384612F08CFA00B9724F1F
:1048E000724BA200D750013469E64946DAE74FF02F
:1048F0007E51D7E76E4B1B78D90707D5802010F083
:1049000023FF08B103F03CFF12F008FD1F200DF05B
:1049100097FDD8B10C23237018E00022654B1A6074
:10492000654B1A60654A12685A600323F3E710F07A
:1049300097FA614E614B1A6873686433934205D2EB
:10494000402010F065FA002800F0C28010F0B0FAA4
:104950000646002800F0918423780C3B022B08D9EE
:1049600001232370564B93F8FB2012B1002283F8E9
:10497000FB20544B1B78072B05D10CF08DFE079BB9
:10498000C01A474B988000224D4B1A704D4F3B7810
:10499000072B40F0CC840CF07FFE07904A4C6368F4
:1049A00020469847A246002855D00026B4F8A850C3
:1049B00084F84960DFF81491002D40F00185E26A27
:1049C000B4F9243094F84A109B1AA363226BB4F90B
:1049D000263004F138009B1AE363626BB4F9283087
:1049E00004F134089B1A23640AF0E4F84C46DFF81B
:1049F000B0900AF5707658F8040F11F0F5FFDAF868
:104A0000201012F045F83B788346082B03D113F0B1
:104A10002FF829F815005946DAF8BC333046984784
:104A2000DAF84434014606F1880098473B7883461B
:104A3000032B03D113F01CF829F81500DAF8AC3079
:104A40005946D8F8780398470135032D44F8040FE8
:104A500006F12C06CFD11B4C2278072A05D10CF089
:104A60001BFE079BC01A0E4B1880154B93F80121B3
:104A70001D460592002A00F07185013A83F8012154
:104A80001DB0BDE8F08F00BFD7A36841381A0020E1
:104A90006F12033B1411002000004843A4707D3FB7
:104AA000EC22002000C0F94400C0F9C4AC10002082
:104AB000A4350020D03A0020EC240020801B0020E8
:104AC0007810002014250020CC3B0020204100203D
:104AD000DFF864834027C246DFF86093336818F834
:104AE000030068B110F062FAD9F80030013F03F119
:104AF000FF33C9F80030336803F101033360EDD1AF
:104B000033681AF80330002B7FF420AF33604FF086
:104B1000FF3373600423FEE610F0A2F9934A50219C
:104B2000A2F10C0301932623029200934920A2F1E3
:104B30000A03163A07F050F900287FF407AF4FF048
:104B4000FF328B4B18605A600723E4E610F088F9B7
:104B5000052300210093874B02910191A3F10802E4
:104B6000532007F039F900287FF4F0AE804B18602D
:104B70000823D0E610F074F97F4B804E186812F0CD
:104B800077FF8046D6F8BC0012F072FF81464020C5
:104B900010F03EF9314600287FF4D8AE744E784FBD
:104BA00033687878492B01F28D85DFE813F04A00ED
:104BB00050005E00650069006E00730078007D00A3
:104BC0008400890095009F00A400AF00B400B900E4
:104BD000BE00C600CE00D600490151015901610155
:104BE000690176017F01880191019A01A301AC015D
:104BF000B501BE01C401CD01D301D901DF01E50139
:104C0000EB01F201F901000206020C0213021A0282
:104C1000200226022C02320236023A023F024402ED
:104C200049024F02AB02B802BD02C202C702CC0267
:104C3000D102D702DC02E102E602EB02F002F50249
:104C4000F902504A5049514806F0D6FD09E0504B50
:104C50004C4A01934F4B504900935048504B06F03B
:104C6000CBFD33680133336070E64E4B4E4A4F49FB
:104C70004F4806F0C1FDF4E74E4A43494E48E3E78A
:104C80006B782A784D494E48F3E74E4B4E491A8AC5
:104C90004E48D9E74B4B4C495A8A4D48D4E74FF020
:104CA0007E524C494C48CFE71FFA89F31FFA88F22D
:104CB0004A494B48DDE74B4B4B491A8A4B48C3E7FF
:104CC0004B4B1B68DA0404D591F8C020494846498B
:104CD000BAE70C233360C4E7474948488B784A78E1
:104CE00009780091464906F087FDBAE7454B3E49F1
:104CF0001A884548A8E7404B5B79012BB1D1B1F93F
:104D0000C430B1F9C62041483449B2E7404B2E497E
:104D10001A68404898E7404B2B499A783F4893E7F8
:104D20003F4B29491A783F488EE70C2303FB0011BB
:104D30003D4891F8C820244986E70C2303FB001165
:104D40003A4891F8CA2020497EE70C2303FB001162
:104D5000374891F8C9201C4976E70C2303FB001162
:104D6000344891F8D12018496EE700BFD6A2010857
:104D7000EC24002090A4010880230020781000205B
:104D8000081600201DBF010892CC010829BF0108A8
:104D90005DBF010813BF01083DBF01084BBF0108FB
:104DA00037BF01080ABF0108FEBE0108A4CE0108F2
:104DB00062BF01080C16002070BF01087BBF01080C
:104DC00081BF010868230020F5CE01088CBF0108CF
:104DD00098BF0108ABC50108A4BF01087BC001084A
:104DE000AFBF0108A822002093CE0108BBBF010875
:104DF00064230020C2BF0108FE350020D6BF010891
:104E0000CDBF01087E230020E6BF0108EEBF0108E8
:104E100020410020FCBF0108BA3B002005C001086A
:104E2000582C002015C0010827C001082FC0010818
:104E300037C0010843C0010860A20108D03A002031
:104E40000C2303FB0011844891F8CB208349FBE637
:104E50000C2303FB0011824891F8CC207F49F3E634
:104E60000C2303FB00117F4891F8D0207B49EBE62F
:104E70000C2303FB00117C48B1F8D2207749E3E60C
:104E80000C2303FB001191F8CE3091F8CD2091F85E
:104E9000CF1076480091764925E7764B7648196819
:104EA0004B780A788978009171491CE7714B7348F7
:104EB00019680B79CA78497900916D4913E76D4BF0
:104EC0006F481968CB798A79097A009168490AE7AD
:104ED000684B6C4819688B7A4A7AC97A00916449A0
:104EE00001E7644B684819684B7B0A7B897B00911A
:104EF0005F49F8E65F4B654819680B7CCA7B497CC3
:104F000000915B49EFE65B4B61481968CB7C8A7C7A
:104F1000097D00915649E6E6564B5E4819688B7D3F
:104F20004A7DC97D00915249DDE6524B4B491B68D1
:104F300059481A7E88E64F4B584819680B7FCA7E3D
:104F4000497F00914A49CEE64A4B44491B68544880
:104F50009A7F79E6474B41491B6852481A8C73E6A1
:104F6000444B3E491B6850485A8C6DE6414B3B49C7
:104F70001B684E489A8C67E63E4B38491B684C4884
:104F8000DA8C61E63B4B35491B684A4893F8282088
:104F90005AE6384B31491B68474893F82F2053E6AF
:104FA000344B2E491B68454893F830204CE6314B72
:104FB0002A491B684248DA8E46E62E4B27491B6871
:104FC00040481A8F40E62B4B24491B683E4893F813
:104FD0003A2039E6274B21491B683C4893F83B208F
:104FE00032E6244B1D491B6839489A8F2CE6214B29
:104FF0001A491B683748DA8F26E61E4B17491B688B
:1050000035485A8D20E61B4B14491B6833489A8D4E
:105010001AE60A7A3248114916E64A7A31480F49A7
:1050200012E6314B0D49DA7830480DE62E4B0B492C
:105030001A792F4808E62C4B08495A792D4803E67F
:10504000294A2D49D3892D48528912E6264A2A49F0
:10505000138A2B4892890CE64FC00108F5CE01084F
:1050600057C0010860C0010869C0010881C001087B
:1050700078C001081025002087C001088FC00108F2
:1050800098C001089FC00108A6C00108ADC0010872
:10509000B5C00108BDC00108C6C00108BFC00108F5
:1050A000CDC00108DFC00108ECC00108F7C001084D
:1050B00006C1010819C1010826C1010834C101084F
:1050C00045C101085CC101086EC1010888C1010821
:1050D0009EC10108ACC10108B6C10108C3C10108E5
:1050E000CCD90108D4C10108BA3B0020E1C10108B4
:1050F000EAC10108FCC101087BC001080CC201081B
:105100001AC201088C4B188811F06EFC8B4911F003
:10511000BFFC11F099FE8A4902468A4894E5864B05
:105120008749DA7888488FE5884B85491A78884816
:105130008AE591F8EF208748814985E591F8F820C4
:1051400085487F4980E5854B7D499A7F84487BE58A
:10515000824B7B4993F82020824875E57F4B784944
:105160009A8C814870E57D4B75491A7A7F486BE5CA
:105170007F4B73491A797F4866E57D4B70499A7871
:105180007D4861E57A4B6E491A887C485CE5784B2E
:105190006B49DA897A4857E5BA786949794853E51D
:1051A000794B67491A6879484EE51A200DF048F99D
:1051B000A0B1774B1B888BB9764B14A91B680E20C6
:1051C0001493069B159306F063FB4FF48052724BC9
:1051D0001A800A232370069806F0A8FB06F038FB15
:1051E000FFF7B4BB6D4B1B78002BF4D01A200DF0E9
:1051F00027F90028EFD16A4B93F8FB30002BEAD156
:1052000009232370EAE7674B1A68674B5B68C8336A
:10521000934211D2AB78032B0BD1644E306803F06C
:105220009BFA00233360624B1B78022B01D103F001
:1052300097FC0123FFF76FBB12F07AFA0028E9D13F
:10524000FFF784BB012A01D108F064FA0D23132073
:10525000237010F0F7FDFFF779BB012A04D108F0A5
:105260003DF900283FF472AB0E23F0E71F200DF04C
:10527000E7F800287FF46AABDBE7EB78002B3FF41C
:1052800078AB00274FF0010AB9464A4B1B68DB0494
:105290004BBF494B364BB3F804B0B3F814B0584683
:1052A00011F0A2FB454B014653F82700D04611F000
:1052B00083FD00B1C846013746EA0806082FF6B25A
:1052C000EDD1384B364F1B68BEB103F59C53083304
:1052D000C7F8FC302378012B7FF44BAB97F8FB30F9
:1052E000002B7FF446ABAB78032B19D012F016F8E5
:1052F000012387F8FB30FFF73CBBD7F8FC209A422C
:10530000E8D82378012B3FF434AB97F8FB30002B1F
:105310003FF42FAB06F018FE87F8FB60FFF729BBC0
:10532000802010F011FA00287FF423ABDEE7002381
:105330000793FFF733BB00BFF02600200000C842F0
:10534000F5CE01082CC2010837C2010888270020C9
:1053500044C2010852C201085FC201083836002069
:1053600075C2010886C20108A0C20108BAC20108BC
:1053700068230020CCC20108DDC20108F0C2010888
:10538000FFC2010810C30108681800201BC30108F0
:105390005C23002058230020542300201E250020D9
:1053A00078100020801B0020EC240020DC3A002034
:1053B000F52400200C360020A42D002058250020C4
:1053C0005E4BD9F800205B78059608934FF47A730A
:1053D000B3FBF2F3C3EB431203EB8203DB009BB29C
:1053E00004933B7804F12C070993554BB3F90690CD
:1053F000049B5B080A93049B9D4201BF00237B63CF
:10540000E3673B604F4BF318B3F924007B6B034415
:105410007B6311F0E9FAE26F02F10108B8F1010FC4
:10542000C4F87C8007D10023012D2067E066636704
:105430005DD1002030E0D4F86CA00C9251460B9066
:1054400011F01CFA8346404611F0CEFA0146584648
:1054500011F0D2FB514611F013FA0B9B0146824624
:105460002067184611F00AFA594611F011FB616FD6
:1054700011F006FA012D8346A067C4F86CA060679E
:105480000C9A34D1B8F1010FD3DD104611F0ACFA0B
:105490000146584611F0B0FB12F0AAFD099B804668
:1054A000032B05D112F0E4FA01230FFA80F90593DA
:1054B000089BABB1184611F097FA414611F086FCF3
:1054C00070B1059B13B11E4BA3F806901E4809F05E
:1054D00061FB00221D4B5A609A60DA60FFF7BBBA8D
:1054E0000A9A7B6B1344049A93FBF2F33B600236F7
:1054F000062E07F1040704F114047FF47CAF059B2A
:1055000013B10F4BA3F80690012D0FD10022104BC1
:105510001B689A621A63DA620E4B93F8003113B17A
:105520000D4B1B8813B9012010F08CFC054AB2F812
:10553000A830013BA2F8A830CBE700BFBA3B00205F
:10554000EC220020CC3B0020743C002020410020B5
:10555000A41B00207810002034360020AC4B5B796F
:10556000002B00F03184AB4B1B78013BDBB285F89C
:1055700001312378072B40F02A840CF08DF80B9032
:10558000A54B4FF07E501B6807936B680D93D5F8C1
:10559000043119460A9311F071F9A04B196811F002
:1055A00077FA4FF07E510C9011F01AFC10B94FF0C1
:1055B0007E530C939A4B002509939A4B9A4C08936F
:1055C00000230493049BDFF8B0929E0059F82370E7
:1055D000049A964B294653F82280404611F0ECFB82
:1055E000E8B9049B09F1D40959F823903846494693
:1055F00011F044F9824620F00041404611F0E6FBEC
:1056000058B12946504611F0FFFB002800F0E38313
:105610004946404611F034F90746854BF750854B13
:10562000B3F800A01AF0030F3DD0049B022B3AD030
:10563000079B93F8320011F0D7F97F4BF15811F026
:1056400027FA079B814693F831B0CBF1000011F0A7
:10565000CBF980460146484611F0B8FB40B95846A0
:1056600011F0BEF94946804611F0BAFB00B9C846B0
:10567000049A724B33F91200089BB3F90030C01A38
:1056800011F0B2F96E4911F003FA0146404611F0EB
:10569000F5F81AF0010F0E9000F0CE83694B1968EF
:1056A00011F0F6F9074694F81431002B57D0049BFB
:1056B000022B54D0089BDFF88481B3F90000049BCF
:1056C00038F91330C01A11F08FF95E4B07465C4968
:1056D000186811F0DDF90146384611F0D9F9069A3B
:1056E000D4F818310746D31A574A1268934231DC6E
:1056F0004FF07E510A9811F069FB80B3534B544927
:105700001A68B1F90A00B8F900301B1A002BB8BFAB
:105710005B42934223DAB8F90230B1F90C105B1AFC
:10572000002BB8BF5B429A4219DD4A4BDFF8289143
:10573000D3F80080D9F80400414620F0004011F071
:1057400045FB60B1D9F80810404621F0004111F046
:105750005BFB20B1002084F814010CF02BF93E4BC8
:1057600038463344D3F804A0DFF81091514611F0C5
:1057700085F88046394B0D98F15811F089F941466A
:1057800011F086F9049B0146022B46F8090006D168
:10579000334A344B10681B689847C9F80800099BC6
:1057A00053F8049F0993304B5968304B186811F037
:1057B0006FF90C9911F06CF92D4BF15811F068F953
:1057C000414611F065F9494611F05AF8049B8346A9
:1057D000022B40F0008494F81C31012B02D0192BCD
:1057E00040F0F9834FF00103224940460E9311F037
:1057F0000BFB0E9B00B90346DBB2002B40D02BF015
:10580000004029F0004111F0E1FA00283BD037E0D8
:10581000BA3B0020582C002010250020202E00200C
:105820008C220020FA26002078100020142E002060
:1058300080110020F6350020141100208C3100204A
:10584000CDCCCC3DFC2D0020242E0020282E002085
:10585000F02600202C2E002020410020D02D0020FA
:105860002431002020310020000000205C2C00208A
:10587000DC2D002000009642AC1000208422002085
:10588000099BC3F800B0049B022B6DD0A24AA34B26
:1058900051461B68B0589847A14AA24B01461B6865
:1058A000B0589847079B814693F83A30632B00F233
:1058B0009C839D4B1B88002B40F097839B4BF1589A
:1058C0009B4B186811F0E4F84FF07E51824611F0BE
:1058D00087FA08B94FF07E5A964B5046196811F076
:1058E000D7F80146384611F0D3F8494610F0C6FF04
:1058F000914B8146F15810F0C1FF904B196811F09F
:105900007BF98D4B074646F80390079B93F8489028
:10591000B9F1000F1ED04FF07E510A9811F06AFACB
:10592000C0B1874B27F00040196811F06DFA88B1BB
:10593000844B28F00040196811F066FA50B101203C
:10594000069BB9F1020F84F81401C4F8183101D193
:105950000CF030F87C4B0D98F15811F099F839465D
:1059600011F096F8794B985194F828312BB9784B6F
:10597000F550099B1D60754BF550049B0133049352
:10598000089B02330893049B032B7FF41BAE714EDC
:105990003278072A05D10BF07FFE0B9BC01A6E4BA5
:1059A00058803378012B40F022830BF075FE6B4951
:1059B000D4F82C31684A0968C31A93805B1A0690A0
:1059C000D380C4F82C01664B664E1B6893F82F8079
:1059D000654B1B6813F4805F644B00F05583644A89
:1059E000B3F818901278F668D70758BF1A8B614B36
:1059F00058BFA4F83021DF88A9EB070B584610F0F8
:105A0000F3FF82460146304611F0EAF9002800F023
:105A1000F782D4F83831C4F83431574B1B68C4F8D6
:105A20003C31D4F84011D4F8480111F0E5F84FF0BA
:105A30007E51044611F0D4F908B94FF07E5400218C
:105A4000204611F0D7F900B900244C4DD5F8343177
:105A5000C5F848410793D5F83C3107981946089393
:105A600010F00CFF464BC5F854011968384B0B90E9
:105A7000186810F005FF354B196810F001FF414917
:105A80000C9011F005F8404B82461D6805F1004668
:105A9000314611F09BF9002840F00A832946504610
:105AA00011F09EF900B9AA46354B5968284B586841
:105AB00010F0E6FE254B596810F0E2FE31490D90DA
:105AC00010F0E6FF07460146304611F09DF930B967
:105AD000394628462E4611F083F900B93E46284B38
:105AE00099681B4B986810F0CBFE26490E9010F079
:105AF000CFFF264B81461D6805F10047394611F05E
:105B000065F9002844D1294648464F4611F068F906
:105B100000283DD12F463BE03C2E0020382E0020AF
:105B2000A02E00209C2E0020F63500202011002001
:105B3000F82D0020F42D0020981100205C2C00206E
:105B4000342E0020302E0020E82D00209C22002042
:105B50008422002014250020EC220020F8240020BC
:105B600010250020381A00200C360020383600207E
:105B7000A4350020A42D00208023002078100020D0
:105B8000902200206F12833A602C0020642C0020A9
:105B9000B8F1000F25D0924B1A7912B3914A1578BB
:105BA000FDB1187810F01CFF8046284610F01CFF4D
:105BB0000146404610F06CFF8B4B0546188810F0EC
:105BC0000FFF0146284611F017F88849054611F0E5
:105BD00007F900B9854D4FF07E51284611F00AF9BA
:105BE00008B94FF07E55824B4FF000095B78002BCF
:105BF000804B14BF01204FF0FF3093F800B010F03D
:105C0000F3FE394610F044FF00237B4F0F900A93B8
:105C10000993D945C0F266820A99099810F02EFEC0
:105C2000764D4FF07E51C5F80401064611F0ECF8B0
:105C3000002800F0988231464FF07E5010F0DCFFD3
:105C40000024074614AEA34500F384820CF0FEFB4B
:105C500018B14FF07C53C5F84831DFF8A0A10025FA
:105C6000DAF8483109939AF8D8310A93644BDB7813
:105C70001093644BD3F80080404611F0E5F881465C
:105C8000614B1E6806F010031193604B06F48056BA
:105C90001C785F4B04F00104B3F906705D4B5A8B1E
:105CA00012930AF5AC730F9213935D45C0F0808296
:105CB00024B9594B594AA34500F3C2824F4BD3F83C
:105CC000DC21002A00F08E8493F81C31192B09D8AE
:105CD00001229A40524B1340002B40F0B782100330
:105CE00000F1F883484E4F4D336813F0200F30D049
:105CF00000200AF093FC4C4C8046208001200AF0E2
:105D00008DFC0746608008200CF09AFB08B33B4BE3
:105D100095F90A1093F80232012B444B40F0E583C9
:105D2000484295F91620B3F90210B3F90030414307
:105D3000534332206FF0310291FBF0F193FBF2F20A
:105D400093FBF0F00A44A8EB020222800844384496
:105D500060800023364AEC18B4F90410B2F902004E
:105D6000B4F90640884203DB84422146A8BF0146BD
:105D70000C33602B22F8021FEDD12E4DAB89002B86
:105D800040F0C3831D4F97F81C31013B182B00F2E4
:105D9000F283DFE813F0E203F003F0035404F003AE
:105DA000F003F0034104F003F003F003F003F00309
:105DB0006004F003F003F003F0038404540471045E
:105DC000F003F0036004E2030123FFF7D0BB0023DC
:105DD0000B93FFF7D5BB4146484610F04FFD1BE43F
:105DE000FE350020341A0020221A0020713DAA3FFF
:105DF0001C250020F4220020D01100207810002063
:105E000010360020C82600200C360020A4350020C3
:105E1000CC35002038360020F822002058250020FC
:105E200032413003F82B0020442300208C31002025
:105E3000422300207A2C0020D4F8A890D4F8AC801B
:105E40004946404610F0C2FF00287DD049464FF039
:105E50007E5010F013FD974B8146B3F90000B3F963
:105E6000023080EAE07183EAE372A1EBE071A2EB19
:105E7000E37291426ADD0028D8BF404210F0B4FDC1
:105E80008D4910F005FE8D4B80461B78002B62D0AB
:105E90008B4B2946D3F800B0584610F0B5FF0028C8
:105EA00000F09780874B2946D3F800A0504610F0A9
:105EB000ABFF002800F08D804FF07E51484610F077
:105EC000DDFC814910F0E4FD594610F095FE4FF0DD
:105ED0007E5110F0D5FC41468146504610F0CEFC74
:105EE000514610F089FE4FF07E51804610F078FF49
:105EF00008B94FF07E582946404610F07BFF00B9A4
:105F0000A8464946404610F0C3FD81466F4B0E98A7
:105F1000196810F0BDFD4FF07E518046484610F0E4
:105F20005FFF08B94FF07E592946484610F062FFDE
:105F300000B9A9464946404610F0AAFD0146384638
:105F400010F09EFCFFF7AEBB414680E7002BCCBFB4
:105F50001846584292E75E4B5E49D3F800A050467F
:105F600010F034FF002830D051464FF07E5010F032
:105F700085FC594910F08CFD41468346574810F086
:105F80007DFC0146584610F083FD514610F078FC28
:105F90004B4B196810F07CFD80462946404610F0B6
:105FA0001FFFB0B94FF07E51484610F067FC4146E4
:105FB0008146454810F020FE0146484610F068FD35
:105FC0004FF07E5110F05CFC9FE73D4BD3F8008012
:105FD000E3E7A9469AE74FF001034FF07E51D4F86A
:105FE00004010E9310F006FF03E429467AE4072B20
:105FF00003D10BF051FB0690E5E400230693E2E4A5
:1060000009EB070010F0F0FC0146304610F0F2FEFC
:1060100000B3D4F8BC303046C4F83431D4F844313D
:10602000C4F83C3110F036FFA4F83001484610F0B7
:10603000DBFC0146304610F021FC0546384610F0E6
:10604000D3FC0146284610F019FCC4F84801D4F8E6
:106050004C11E8E4B4F830319B450ADBD4F8383110
:10606000C4F848A1C4F834311D4B1B68C4F83C3156
:10607000D7E4D4F8BC30C4F84851C4F83431D4F86B
:106080004431C4F83C31E2E7588B10F0ADFC0146D6
:10609000F06810F0F3FB124BC4F848011B68D4F809
:1060A0005011C4F83C31D4F8BC30C4F83431BAE4EF
:1060B000B246F9E48C310020CDCCCC3D082E002036
:1060C000042E00200C2E00200000C842002E0020CC
:1060D000102E0020AE47813F610BB63B00003443D9
:1060E000802300207968504610F0D2FCB9688046C1
:1060F000304610F0CDFC0146404610F0C1FBF96877
:1061000080460F9810F0C4FC0146404610F0B8FBE2
:106110004FF07E518046284610F076FE20B1404672
:10612000294610F0B5FC80464146099810F04EFE15
:1061300068B941460A9810F053FE08B9CDF8288096
:1061400014AB43F82980103709F1010961E5CDF856
:106150002480F5E756F82400394610F099FC46F8FB
:10616000240001346FE50CF071F938B94FF07C511F
:10617000204610F049FE00283FF46FAD4FF07C51EF
:10618000304610F085FC05460146204610F01EFE04
:1061900050B929464FF07E5010F070FB214605465D
:1061A00010F01EFE00B92546BB4BC3F8485154E51C
:1061B000139A2B019958099810F06AFC14AB53F804
:1061C000251010F05DFB0B9910F062FC089910F09F
:1061D00057FB0A9B82463BB10899079810F050FB89
:1061E000514610F04BFB8246109B5046FBB110F01D
:1061F0002BFE4845824606DB079810F025FE5045E9
:10620000A8BF504600E0484610F0EEFB119B8246C6
:1062100043B13CB136B90CF019F918B90F9B9F4244
:10622000B8BFC2469D4B43F825A001353DE510F0AF
:106230000BFE8246089810F007FE8245E4DBDBE7A0
:1062400052F8241043F82410013434E5944B1B8891
:10625000D90540F18C80934C206810F0F5FDADF825
:106260005000606810F0F0FDADF85200A06810F02A
:10627000EBFDADF854004FF47A724FF461618A4837
:10628000B0F9023003F5E163534393FBF1F3A3F557
:10629000FA73ADF86830B0F9003003F5E1635A43A2
:1062A00092FBF1F27D4BA2F5FA7280491868ADF8C5
:1062B0006A2010F0E3FA10F0C7FD7D4A129B1188A6
:1062C0001B8BADF85600C91AADF858105188C91A81
:1062D000ADF85A109188C91AADF85C10D188C91A66
:1062E000ADF85E101189C91AADF860105189C91A4C
:1062F000ADF862109189D289C91AD31AADF8663007
:106300000023ADF8641019466A4A22F813100133CD
:10631000082BFAD14FF00C096427674B674C1B78A8
:10632000674DC3EBC3032344DFF8A481DFF884A1E6
:106330000993099BA3423DD100254FF00C09642726
:10634000604EDFF88C8109FB0583B6F9024093F9B2
:106350000A00444394FBF7F4E8B274800AF05EF953
:1063600001352044082D26F8020FECD1BAE4564935
:106370000C9810F08DFB10F067FD5349ADF85000FC
:106380000D9810F085FB10F05FFD4F49ADF85200FD
:106390000E9810F07DFB10F057FD00B2ADF85400E0
:1063A000002E3FF468AF494B1B8B9F42BFF663AF93
:1063B00040425EE7A07928B11630C0B20CF040F838
:1063C000002867D094F800E094F9051009FB0E83CB
:1063D000DA889B8894F801C0D21A94F9043092B2FA
:1063E000534393FBF7F34FEA520BA3EB0B030891D4
:1063F000E1781BB207934FEA4C0681BB1CA90E44FF
:1064000036F8201C2980012309FB0EF158F80110F1
:1064100003FA0CFC1CEA010FB5F9006094F90210B4
:1064200008BF184601FB06F191FBF7F1079B18BF67
:106430004FF0FF30994209DB089B5A4392FBF7F279
:10644000A2EB0B031BB28B42A8BF0B463AF81E20EF
:1064500000FB03232AF81E300235073469E71CAB22
:106460001E44B5F9000036F9206CB04208DA014448
:10647000884203DC8E423046A8BF08462880C2E727
:10648000C1DD411AB14203DB8842A8BF0846064677
:106490002E80B8E72880DFE778100020F82200205F
:1064A000F6350020381A00208C3100200080BB44D3
:1064B000CC35002044230020152B0020162B002073
:1064C0005A120020422300203333333F3836002055
:1064D000F82B00208F4A904830F8131022F8131040
:1064E0000133082BF8D1FFF7FDBBB3F90220B3F954
:1064F00000004A43322192FBF1F24244228095F996
:106500001620504390FBF1F021E4DFF808820024CC
:10651000C346824FDFF81C9238F9140010F064FA79
:1065200001462C2000FB049005F0C4FD11F0A0FAF8
:10653000B7F9043000B298424FEA440AB7F906208E
:1065400003DB82421346A8BF03460134082C2BF814
:106550000A3007F10C07DFD114E4AB7B002B54D0D9
:106560006C4BB3F90A0010F03FFA0146002005F029
:1065700087F80123059333689A0603D497F81C31F2
:10658000052B16D1634CB4F9000010F02DFA01462A
:10659000059805F085F8B4F9020010F025FA059B7E
:1065A00001460133D8B205F07BF8059B0233DBB21C
:1065B00005933368DB0215D50024EE7B564FE5B218
:1065C0007319DBB2112B0DD8331937F9130010F002
:1065D0000BFA059B01461D44E8B2013405F060F852
:1065E0000E2CECD14E4C94F8E021002A67D14D4B93
:1065F0001B78072B05D10BF04FF8069BC01A4A4BAE
:10660000D88001232370FEF73BBA484B187810F06E
:106610000100A5D10021AAE73E4CB4F9060010F014
:10662000E3F90146002005F02BF8B4F9080010F05A
:10663000DBF90146012005F023F802239AE7354CE7
:10664000B4F9080010F0D0F90146002005F018F860
:10665000B4F90A00EBE70224DFF8B88038F9140037
:1066600010F0C2F9A31E01460134D8B205F018F8A3
:10667000082CF3D106237DE7264C049B34F9130044
:1066800010F0B2F9049B0146033BD8B205F008F8BC
:10669000049B0133072B0493EFD104236AE7002402
:1066A000DFF8708038F9140010F09EF90146E0B26E
:1066B000013404F0F5FF082CF4D105945BE70CF0ED
:1066C00035F994E711F034F800283EF43FA94FF46F
:1066D0008052174B1A800A23FEF71DB9B9F1020F39
:1066E0004FF4FA707DF4C4AC8345A8BF0020049B2E
:1066F000B8BFA0EB0B00584310F076F9B045B86076
:10670000BDF6C4AC57F8292002F1004247F8292011
:10671000FDF7B7BC44230020CC350020F82B002027
:106720007810002014250020EC220020A435002041
:10673000542300207C1200202DE9F04FA94B00F5D6
:106740009C4808F12008C3F80080A74B87B01C784C
:106750000746002C6AD0A54A1268904201D9013C34
:106760001C70A34C2368D90405D500200BF068FEEB
:1067700008B904F01DFD9F4A537D9346002B00F09D
:1067800080819D4A013B32F913009BF817301BB101
:10679000C0F53B60083000B2A0F57A70B0F57A7FA2
:1067A000A8BF4FF47A7020EAE07010F01DF9934909
:1067B00010F06EF910F06EFB914B18802368DFF833
:1067C0007CA213F4807F00F0D7818E4BDFF85092CB
:1067D0009F4205D999F8022012B9012289F80220B6
:1067E00099F80220002A00F0C7819AF8005099F821
:1067F000217005F001031B2000930BF021FE012FF7
:1068000008BF0025804EDFF83882019018BF05F0E0
:10681000020599F82020052A00F2AA81DFE812F08B
:106820006F01CF01DA01FA010702220209F058FED6
:106830000646764DDFF8BC91DFF8F0A1A64246DCB3
:1068400042F201024FF47A71694BB7FBF1F91B6810
:10685000134001936E4B06D06E4A12781A706E4A3E
:1068600011786E4A11701B78009323B16B4B1E7820
:1068700086F0010300930F230024DFF8C8B1DFF88E
:1068800078A185F8243009F02BFE844249DB95F885
:106890002430634C0F2B0CBF01220022614B5A4D58
:1068A0001A7040F0D1801B200BF0CAFD002840F088
:1068B000CB802B68E268A3609B1AC82B02D9012306
:1068C00084F82130584A13780133137049E7072CB4
:1068D000E1B25648D8BF14F80910DAF804309847E6
:1068E000032C1ADCC8B1524B33F8242003EB84018B
:1068F000831A4FF47A7058434B889B1A90FBF3F03D
:1069000040F2EE2300F57A709842B8BF184640F680
:10691000CA039842A8BF184680B225F81400013473
:106920008CE7009A6300D2B135F91400314A80B285
:10693000D18C81424FEA840103D8B2F828E0864521
:1069400020D23C4A515889450BD23AF80300019AAB
:10695000EAB92AF8030001340BF1060B93E700981B
:10696000E4E7E0B2029309F0D3FD032C029BEEDCD6
:10697000012101FA04FE95F8241021EA0E0185F8A0
:106980002410E4E72B4E09F596727250DFE7264992
:1069900003EB040E91F800C00321BCFBF1F101EB05
:1069A0004101ACEB0101C9B2714405EB4101C8845E
:1069B00095F86E1029B9BCF1020FCAD9012185F8EA
:1069C0006E10BBF80010BBF802000844BBF80410BE
:1069D0000844194900B2C852032190FBF1F080B27B
:1069E000B7E700BFE4290020142B0020102B002063
:1069F0000C36002038360020CC350020AAF1823F2A
:106A0000F4350020404B4C00801B00202414002053
:106A1000A5350020B42900202004002021040020F6
:106A200010360020EE260020380F0020D829002044
:106A30006C2D00203C0F002094140020A435002071
:106A4000B83100204A1400200123914A1370914A62
:106A500013702B68A268E3609B1A62688E4D9342A4
:106A600084BF002384F82130002409F039FD8442DA
:106A7000BFF628AFE0B209F04BFD25F81400013451
:106A8000F3E7226812047FF599AE844AD2F88810A1
:106A9000791A0029FFF692AE8149C2F88880487CB5
:106AA000804931F810009BF8161080B290FBF1F08D
:106AB00092F88C10013101F00F0182F88C10114412
:106AC00081F88D0018468D32815C01300B4410280E
:106AD0001BB2F9D193FBF0F31BB2002B0ADB642B42
:106AE000A8BF64239BF8172032B918B20FF07CFFBF
:106AF0006D495DE60023F5E7C3F16403F5E7009B0C
:106B00006BB30BF0B1FC012807D164203168B8F8F1
:106B1000062000FB0212C9F81020019B63B198F80F
:106B200004204AB10CF01EFB032289F820204FF408
:106B30007A72C9F81C206CE6012F19D03268D9F896
:106B40001010914207D20CF00DFB032289F820208F
:106B500040F6B832EDE7012289F8202059E6019B82
:106B60004FF4806043B30FF0B9F90022C9F8102048
:106B700015B128460FF066F90BF076FC06460BF0CF
:106B800065FC4A4D002800F099809AF80030DF0734
:106B900040F19480BBF824000FF026FF444B0146DF
:106BA000D86810F027F9002800F01E8101223B4B25
:106BB00083F89D20012394E00FF080F9D5E7012FA1
:106BC00001D10522C8E798F80820012ABBD00CF0B3
:106BD000C9FA1EE6012F08BF0522009B08BF89F8ED
:106BE00020204BB10325BBF918102B4A118051808E
:106BF0009180B8F80210D1803268D9F8141091420F
:106C000002D3009B002B3FD147F23052C9F81C2021
:106C10000322A1E702200FF06FF904F0C9FA3168EE
:106C2000D9F81C200A44C9F81820042294E7012F3F
:106C300011D13268D9F81810914299D21D4B1878A9
:106C400018B90BF0FDFB002892D11B490A8822F0ED
:106C500002020A80B5E73168D9F81C200A44C9F855
:106C6000182085E764203168B8F8062000FB02127E
:106C7000C9F8102000224FF4806089F8202089F89C
:106C800003200FF01BF9C4E5012F3FF4C2AD6FE7FD
:106C90002004002021040020CC35002024140020F2
:106CA000A00C0020B40C002014AE2341A011002041
:106CB000381A002000000020343600200022704BDB
:106CC00083F89D20002E7FF475AF00226D4B1A6073
:106CD0005A609A606C4B1B6893F83030002B7FF43D
:106CE00069AF2B709AF80030DD0723D52368D806EA
:106CF00020D5664A1278D1061CD4DA041AD40BF0D7
:106D0000A5FBB8B9624B5E4D1B78002B00F0878065
:106D1000604B9B78002E71D1002B00F082805E4B7F
:106D20001A685E4B1B689B1A002B7ADA04F040FA53
:106D300085F89E6000221346BBF81A50BBF81C7001
:106D4000574931F912009B08A842C4BF63F07F0382
:106D5000DBB20132B842B8BF43F04003042AF0D19D
:106D6000474D95F89F209A4262D195F8A020F92AC4
:106D700002D8013285F8A020454F85F89F3097F85A
:106D80000080B8F1000F08D140460BF059FB0028F5
:106D900050D085F8A18004F09BFA95F8A030142B10
:106DA00040F09D803B7853B195F89F305F2B06D122
:106DB0009AF8003013F001065BD004F0F9F99AF864
:106DC000003013F0010240F08A8095F89F30572B75
:106DD00074D1344807F0DEFE334B1B6858077ED56C
:106DE0000A22324B1A807AE0002E7FF4E3AE244B65
:106DF00093F89D30002B7FF4DDAE66E73BB14FF496
:106E00007A71254A126801FB0323244A136095F81E
:106E10009E30002B8ED00EF0F9FF002305E0002EEF
:106E2000F5D110200FF00EF8012385F89E3081E790
:106E300000229FE71E4B18609AF80030DB07ACD5A4
:106E40001C4B1B78002BA8D01B4BDB78002BA4D14C
:106E500095F8A1300133DBB2032B85F8A1309CD922
:106E60000C4B5B7813B104F0A3F996E7002E94D194
:106E7000F9E70B200EF0E6FF85F8A0609FE700BF62
:106E8000241400209022002010250020ED26002050
:106E90000000002070110020801B0020A41C002096
:106EA000CC350020743C002018250020981C0020C0
:106EB000A81C0020A53500201036002021684907B5
:106EC00040F1F2805A2B40F0EF8095F8A230002B71
:106ED00000F0DD80012385F8A22085F8A330236827
:106EE0005E0728D595F8A4309BB19AF80030D807F2
:106EF0000FD5994BB3F90620BBF81A309A4208DD3A
:106F000000200BF09DFA20B9322385F8A400A5F8E3
:106F1000A63011200BF094FA002800F00C8195F8AF
:106F2000A8302BB995F8A23013B93223A5F8A630B2
:106F3000012385F8A8300023884E04AF049306F19E
:106F400050087B60314616F8010C0BF053FA30B153
:106F500016F8021C232902D8384606F030FA043607
:106F6000B045EFD17E4B97E8030083E803007D4BEB
:106F70001F78002F00F0108101200BF061FA7A4F8A
:106F80007A4E40B92368DA0540F10983784BDB7803
:106F9000002B00F004833B689B0740F10083358899
:106FA00015F0010540F0008301200EF097FF02204C
:106FB0000BF046FA002800F0F982002D00F0F6826E
:106FC00001200EF07BFF33889D0702D402200EF0D3
:106FD00085FF3188012011F0030118BF01210AF05B
:106FE00015FD3B6813F00A0F17D006200BF028FAA6
:106FF000002800F0DF823388580602D440200EF0CB
:107000006DFF07200BF01CFA38B10A22594BB3F977
:10701000043093FBF2F3584A13800C200BF010FA63
:10702000002800F0CB824FF480700EF057FF534BD6
:107030001B78082B01D00E2B02D140200EF03EFF12
:10704000236859050FD54E4B1B79002B40F0BB82AE
:107050009AF80030DA0740F1BC823C200EF074FB55
:10706000002840F0BB820122464B1A7004F0BAF8A7
:107070003B685B0708D503200BF0E2F9002840F0DD
:10708000B38208200EF01AFF07B0BDE8F08F95F824
:10709000A43083F0010385F8A4301BB10C200EF05E
:1070A000D1FE1CE70D20FAE75D2B00F0B2825B2BCE
:1070B00000F0B5825E2B40F0B4820320AAE20022E9
:1070C000314B1A6095F89F30972B03D14FF4C8725B
:1070D0002E4B87E6A72B05D12D4A137843F00403E6
:1070E0001370FCE60022BB2B049213D10223ADF8EF
:1070F0001230284BBDF810105A890A445A81BDF845
:1071000012109A890A449A8108F0E2F9002385F85E
:10711000A030E4E6B72B02D14FF6FE73E7E7BE2BB3
:1071200003D10223ADF81030E3E7BD2B7FF4D7AED7
:107130004FF6FE73F6E795F8A230002B3FF4FBAE56
:107140009AF8003013F0010302BF85F8A230012342
:1071500085F8A330EFE600BFCC3500207E18002074
:10716000E4240020C426002018250020F635002045
:10717000103600208C310020861000201C250020B5
:10718000261A0020C0100020A81C00209A1C0020F5
:10719000ED260020F02600204FF00C09BB4E06F132
:1071A0005A08314616F8010C0BF024F9E8B1317990
:1071B000B37809FB0150B64A013B03EB4303134488
:1071C000D0F8B02096F803E093420ED0C0F8B0306B
:1071D000012303FA01F195F8DC3080F8ACE023EAF2
:1071E0000101C0F8B47085F8DC1006364645D8D1E8
:1071F000A84BDFF8B0821E68A74BA8F1AC051B684E
:107200000193A64B1B78029300230093D8F8043017
:10721000002B6BD01F78002F68D0D8F80820019978
:107220008A1A002A0DDB01F5FA720121C8F808203C
:10723000009A01FA02F295F8DC1021EA020285F8C0
:10724000DC20029A002A51D098F8002059780432A4
:10725000D2B2002940F05081914931F91210BBF8A7
:10726000182002F1C80081422ADD93F8029095F8B7
:10727000DC20009B1A41D10738D4B9F1000FCCBFF4
:107280000220012001F0BEFC7A1E162A41D8DFE858
:1072900012F035004E00580068007F008600A10003
:1072A000BC00D800E400F0004000680075008600D3
:1072B000A100BC009500B000CC000B011701250116
:1072C000C83A914203DA9978C1F10009CFE7012267
:1072D000009B02FA03F395F8DC2022EA030385F809
:1072E000DC30019B03F5FA73C8F80830009B08F105
:1072F0000C080133042B009388D13DE6317801203E
:107300004944FA29A8BFFA2121EAE17131700BF052
:10731000D3F8D5F8E0000BF061F90122009B02FAE6
:1073200003F395F8DC20134385F8DC30DEE7B17811
:10733000022049446429A8BF642121EAE171B170A7
:10734000E5E731798944B9F1640FA8BF4FF06409CA
:1073500029EAE97986F804900BF0C2F8494603203F
:10736000D5E7B1790D2049446429A8BF642121EAF9
:10737000E171B1710BF0A0F80D2FCAD071790E2018
:1073800049446429A8BF642121EAE1717171BEE713
:10739000F1790520494481F30801F171B7E7D5F887
:1073A000E0200F20D1784944C829A8BFC82121EA8C
:1073B000E171D1700BF080F80F2FAAD0D5F8E02042
:1073C000122011784944C829A8BFC82121EAE171D7
:1073D00011709CE7D5F8E020102011794944C829A4
:1073E000A8BFC82121EAE17111710BF065F8102FD7
:1073F0008FD0D5F8E020132051784944C829A8BF80
:10740000C82121EAE171517081E7D5F8E02011200F
:1074100051794944C829A8BFC82121EAE1715171B5
:107420000BF04AF8112F3FF474AFD5F8E020142088
:1074300091784944C829A8BFC82121EAE171917017
:1074400065E7D5F8E020092091794944C829A8BF0B
:10745000C82121EAE171917159E7D5F8E0200A20AD
:10746000D1794944C829A8BFC82121EAE171D17165
:107470004DE7D5F8E0200B20117A4944C829A8BF70
:10748000C82121EAE171117241E700BF1D190020F6
:10749000B1A40108AC2D0020801B0020A5350020E0
:1074A000CC350020D0140020717815204944B1F566
:1074B000967FA8BF4FF4967121EAE171717026E7BB
:1074C000D5F8E020162092F83B104944FE29A8BFC9
:1074D000FE2121EAE17182F83B1018E7D5F8E0209F
:1074E000172092F83A1049446429A8BF642121EA80
:1074F000E17182F83A100AE701297FF40EAF514991
:1075000031F9121040F633029142A8BF11469A7821
:107510004FF49663B1F5617FB8BF4FF4617193FB8F
:10752000F2F3A1F561710C2F91FBF3F11ED0182F2E
:107530007FF4F3AEC9B2C8290B46A8BFC823D5F85B
:10754000E020D8B292F817E070453FF4E6AEA3EB26
:107550000E034FF0080E93FBFEF30133DBB2D07540
:10756000384603930AF0A8FF039B11E0364ACBB2DA
:1075700052789A423FF4D1AE184603930EF032FC93
:10758000039B384619460AF097FF039B0133DBB291
:10759000002B3FF4C2AE184601F034FBBDE60120DB
:1075A0000EF08CFC012502E5002500E502200EF01E
:1075B00085FC0EE540200EF081FC22E54FF4807042
:1075C0000EF07CFC33E514200AF03AFF00287FF42B
:1075D00044AD03F047FA01F0C3FA44E501F0D0F8F6
:1075E0003C200EF07DF83BE5348814F008047FF46D
:1075F0004BAD08200EF072FC144B1A68144B1A6045
:10760000104BDA88134B1A80134B1C60134B1C6011
:107610003AE501200138C0B207F050FC5FE40220D7
:10762000F8E7562B01D107F053FF3B78002B3FF4CE
:1076300049AD95F89F306F2B7FF441AD03F048FEC4
:107640004DE400BFCC35002008160020A01000201B
:107650009C10002090100020941000208C1000201E
:107660002DE9F04F85B0804603F0FCF9C74B1B783D
:10767000002B40F06C83C64E3368009613F4806F85
:1076800000F06583C34BC44D1B78002B00F049818B
:10769000C24C2A68E368D31A7C2B40F2428124272B
:1076A000237CDFF830B30133DFF82C93E2602374DE
:1076B000ABF1300A384603F0C5F95BF8040F0FF060
:1076C00093F90190BAF810000FF08EF9019B014672
:1076D00018460FF091FA49460FF0DAF90FF0B4FBB3
:1076E000013700B2FFB203F09BF9272FE2D130201F
:1076F00003F0A8F9B4F9140003F092F903F09AF931
:10770000237C980733D141F28833E2689A421BD92F
:107710006427DFF8C892102003F094F9D9F800002C
:1077200090FBF7F000B203F07BF9212003F08AF917
:10773000D9F8003093FBF7F007FB10300028D8BFD2
:10774000404200B203F06CF9142003F07BF9944B33
:10775000B3F904000A2390FBF3F003F061F91C2055
:1077600003F070F9002003F05BF903F063F9237C68
:10777000590740F0B080022003F064F9894BDFF82C
:107780006092D8696423323090FBF3F000B203F0CA
:1077900047F9032003F056F9834B1B7813F0010FD0
:1077A00000F073810AF060FE804B81490746D8687B
:1077B0000FF06EF90FF06EFB80B22FB9009B1B68C3
:1077C00013F0100F18BF002000B203F029F999F848
:1077D0000430002B4DD0DFF80CA29AF800B0BBF1BA
:1077E000000F46D06427734B06201A88019307FBCD
:1077F00002B24FEA4B07B2FBF7F2278B3F01BFB251
:1078000047EA0227BFB2C2F30322174303F01AF973
:1078100038B203F005F9228B019B013292B292FB40
:10782000FBF10BFB112B644A1F88537AA4F818B0A4
:10783000012B40F03081392003F004F938B203F015
:10784000EFF8282003F0FEF80A235C4F386890FB1D
:10785000F3F000B203F0E4F8042003F0F3F8B9F811
:107860000630002B00F03B8100F022FE00B203F056
:10787000D7F802A9524803F0A9F8132003F0E2F860
:10788000BDF9080003F0CCF81B2003F0DBF8BDF9CC
:107890000A0003F0C5F8232003F0D4F84E2003F0CB
:1078A000BFF802A9464803F091F8122003F0CAF885
:1078B000BDF9080003F0B4F81A2003F0C3F8BDF9CD
:1078C0000A0003F0ADF8222003F0BCF8452003F0D5
:1078D000A7F803F0AFF8237C282B22D10023172030
:1078E00023742C6803F0AEF84EF660203C27B4FBFE
:1078F000F0F3B3FBF7F007FB1030000200B203F027
:107900008FF8182003F09EF84FF47A70B4FBF0F46F
:10791000B4FBF7F007FB104000B203F081F803F06E
:1079200089F8284B1B78002B00F099801B4C264AC5
:10793000E369A8EB030393427DD90022234B9A709D
:107940001A711C4A1288D1B2120A9977DA7719751E
:107950005A752968226A891A174AD07A4FF47A72BE
:10796000424391420AD32A682262194A1278013AA4
:10797000012A9FBF10229A7002221A710A200F4A10
:10798000C4F81C80116892682EE000BFC426002055
:107990000C360020681B0020801B002008150020EA
:1079A0008C31002024230020A4350020381A002028
:1079B000CDCC4C3E221A0020261A0020182300208D
:1079C00080969800721B00203F0D03008C0F002052
:1079D000F9350020D822002000007A44A0100020B1
:1079E000FE350020341A002091FBF0F192FBF0F2FA
:1079F000642083F82020121283F82120BA4A1977D4
:107A00001268091292FBF0F202F5FA7292B29A76BB
:107A1000120ADA766269597702F1300183F822108E
:107A200002F5EA4192FBF0F230310912783283F824
:107A3000231083F8242094F824A0BAF1000F00F05A
:107A4000A283E36A5BB194F82430002B71D040F636
:107A5000B732636BA8EB0303934200F29880A34B09
:107A6000D5F800801B78002B00F06C81A04F3B689C
:107A7000002B00F067819F4B1B78013B012B00F22C
:107A80006181DFF884929C4CB7E00523B9F80600C9
:107A9000B0FBF3F098E66E2315217B43527B93FBFA
:107AA000F1F322B19AF800209BB293FBF2F34FF06E
:107AB000640B9FB23A2002F0C5FFB7FBFBFA0FFA46
:107AC0008AF002F0ADFF3B2002F0BCFF0BFB1A7006
:107AD0000A2780B2053090FBF7F000B2AFE6B86835
:107AE00080F31000C2E63B7823B1C4F8288087F801
:107AF00000A0A6E7A36AA8EB0303B3F57A6FA0D3AF
:107B00000123D9F800003B7009F07FFE0746D9F841
:107B1000000009F07AFE7A0693D18E2891D194F86C
:107B20002430002B8DD1754BE3622D2384F8303047
:107B300087E7012284F83830714B84F824201B68D1
:107B40009B781E3B93426F4B1CD91868022104306E
:107B500002F0F2FE94F830206A4F013AD2B284F873
:107B6000302094F8381094F83930D2B94A1C0133D7
:107B700084F8382084F83930386809F04CFEC4F8AD
:107B800034806CE70221186809F039FEE2E794F8C6
:107B90003030002BDED1E36284F8243002F0FCFEAA
:107BA000D8E7E06A013310F801EB84F839300EEBC6
:107BB000010284F83820E0627146DDE7386809F098
:107BC00024FE83B27E2B2A6807D1002384F83A3042
:107BD00084F83B3089F801300FE099F8012062B950
:107BE00094F83A1061BB1B2B22D1386809F010FEC3
:107BF000002844D1012384F83B30386809F008FE9E
:107C000001460028DAD13C4C94F83F30002B00F0BC
:107C10008B80637884F83F00302B40F08580A37818
:107C20005F09012F37D084F8400002F03FFE7BE06F
:107C30000D2B24D10122237084F83A20A187DCE7A0
:107C40007D2B03D1012384F83E30D6E794F83EE043
:107C5000BEF1000F04D080F02000C3B284F83E20B3
:107C60004A1CD2B2092A84F83A20635409D1A28F5F
:107C7000C2F1FF02934202D1012384F83F30012375
:107C8000A8E7082AB9D8A08F034403EB132303F015
:107C9000FF03A387B1E703F00F0013F0100337D001
:107CA00094F803E0237904F15402A4F84C306264A0
:107CB00083EA0E03724484F89430A4F84E10A26450
:107CC00084F84070631D002194F89420DFF83CE0B4
:107CD000676CA66CBE423DD1002948D173454BD19B
:107CE00084F8950020E000BFA0100020741B002045
:107CF000181A00207C1B0020081500208C0F002083
:107D0000601B00205C1B00200C00002010150020D0
:107D100094F8402042B194F89520013202F00F020D
:107D2000824227D084F84030B94FDFF8209394F88E
:107D30003B303BB12B68A3EB0803012B4AD900234E
:107D400084F83B30B34B1B78002B40F0178205B012
:107D5000BDE8F08F13F8011B07F1010C734582EAAF
:107D60000102C4F844C039704FF00101B0D384F867
:107D70009420B3E7E31CA6E71A7894F894309A426B
:107D80004FF0000284F8402003D0B4F94C100120D9
:107D90004BE7A14F636CDFF88892A048A36460644E
:107DA00009F58073394610387B60C7F800903A8136
:107DB0007A81FAF77DFB01304B4604D13A68511CB9
:107DC0003960022111703A683B607A600122904B61
:107DD0001A70A9E797F800A0BAF1000F60D08E4A98
:107DE0008F4913688B4294F8963038D1581C84F828
:107DF0009600B2F90A0003F00F0343F010030028C5
:107E0000B8BF43F020038DF8083053685B1A117A2D
:107E10008DF809304B4084F897300DF10A030025A6
:107E2000D2F804C094F897100DF10E00834228D2C6
:107E30001668ACEB060EBEF1000F1ADC0DB184F82B
:107E4000971094F897105A1C19700023824224D37B
:107E500002A9322002F03EFD4FF0000A1AE0591C40
:107E600003F00F038DF8083084F896100DF1090324
:107E7000D5E7751C1560357803F8015B694001256D
:107E8000D4E70DB184F897108342DAD102A93220E9
:107E900002F020FD87F800A051E702F8013BD5E78A
:107EA00094F8983039F8130018B984F898004FF412
:107EB000036094F89830B0F5826F03F1010384F801
:107EC000983000F0E0805AD8B0F5007F00F095803F
:107ED0000ED8B0F5807F00F0BB80B0F5887F7FF4CE
:107EE00026AF504B1B685E077FF521AF61697CE0D0
:107EF000B0F5047F64D0B0F5806F7FF418AF94F8CC
:107F0000993042F210710133DBB2032B88BF012399
:107F100084F8993094F899305943434B1B88002BCF
:107F200040F0AF800131414B1B78D807404B48BF30
:107F300004311B88DA0748BF0A319E0748BF143155
:107F4000180648BF2831DA0548BF28315E0748BF08
:107F50006431180748BFC8319A0548BF01F5C87198
:107F60009E0648BF01F57A71D80648BF01F5FA614F
:107F70005A0648BF01F57A614FF4806035E0B0F5EC
:107F8000E26F7BD00ED8B0F5C06F69D0B0F5E06F6E
:107F90007FF4CDAE274A516B64234B43118A93FB88
:107FA000F1F122E0B0F5046F62D0B0F5116F00F08E
:107FB000B380B0F5E46F7FF4BAAE1E4AD16BEBE745
:107FC0001D4B1B79002B3FF4B2AE1C4B19780029D6
:107FD0003FF4ADAE1A4B1B4A5B7B63B1138893FB36
:107FE000F1F30A214FF40470594302F08DFC002391
:107FF00084F83B309BE61388F3E70F4B5B79002B4B
:108000003FF495AE104B19680A2391FBF3F1ECE7AE
:10801000581B0020851B0020481A00205C150020FA
:10802000581A00201825002034360020A4350020DE
:10803000F6350020A8220020FE350020341A00204A
:10804000261A0020221A002018230020FAA4010872
:10805000564B1B685B077FF56AAE554B1968C4E742
:10806000544B5B79002B3FF462AE534B9968BCE7ED
:108070000A21524BB3F904305943B6E7504A916B89
:108080008AE702314FE7494B1B6813F0200A7FF45F
:108090004EAE009B1B681B0605D5514602F034FC12
:1080A00084F83BA043E6474B1B7B002B3FF43FAEDD
:1080B00094F89A30032B2DD8DFE803F002181F261E
:1080C000414A1268107892F803E09179090401EBB3
:1080D0000E21014401EB03610133DBB2042B08BF25
:1080E00000234FF4826084F89A307EE7364A1268A3
:1080F000507892F804E0D179E8E7334A1268907832
:1081000092F805E0117AE1E7304A1268507992F866
:1081100006E0F0E70021DDE7264B1B79002B3FF45A
:1081200006AE2B4B197800293FF401AE294B1A8873
:108130000A23534333E7306809F067FB264D804636
:108140002B783BB1013B2B70306809F061FB0028B4
:10815000F1D1FCE521460322601E11F03AFF042113
:10816000601E87F89E8002F01EFB0028ECD0601E87
:1081700002F034FB2B7818442870E5E7174F184EAF
:1081800007F19C04E0E7DFF86090D9F8000009F0FF
:108190003FFBC0B201287FF654AC0228114F3FF4D8
:1081A000A2AC02F0E9FB01233B704AE41825002051
:1081B000A0100020FE350020182300208C31002064
:1081C000A8220020261A002010250020AC2D002017
:1081D000341A0020221A0020901B002008150020CD
:1081E0008C1B00200C0000205C1B0020024B1A8816
:1081F0009B780280837070471CA50108064A1168AD
:1082000049B1642350684343B3FBF1F303490B8046
:108210000023136053607047A81500202E1600201D
:1082200070472DE9F843304B06461B782BB92F4A8F
:10823000136053609360BDE8F8832D4B9F6898608E
:108240002C4B5B79012B09D001D3042B04D90022DC
:10825000264B1A605A609A60BDE8F88340F6E449FC
:108260004FF47A74244BDFF8A480DA79234B244D41
:1082700033F81200B8F9023080B209FB00F2C3EB08
:1082800012336343B8F9002093FBF2F3EB600EF076
:10829000A7FB01461B4803F00DFF0EF0FBFD80B26B
:1082A00009FB00F9B8F90200B8F90030C0EB193940
:1082B00004FB09F494FBF3F4D5F80C80F01BAC60DC
:1082C00008FB00F00EF090FB0F490EF0E1FB69682F
:1082D0000EF0D6FA68600EF0B7FD044B286083E814
:1082E00010019860BDE8F883341A0020182300209C
:1082F000A8150020FE350020A00C0020B40C0020A2
:10830000FC0F00200C1000202FE33E313C11002018
:108310002DE9F843224B234D1B79012B3BD1224BF6
:10832000224E9A78224B33F81240A4B220460EF027
:1083300057FB0146304603F0BDFE1E4B9F7893F875
:10834000009093F801800EF0A5FD44F6FB7209EB56
:10835000491983B209FB032309FB0424C8EB08383D
:10836000B3FBF8F3B4FBF8F4B3FBF7F3B4FBF7F4A7
:108370009BB2A4B226F8043C26F8024C2B806C80F9
:108380000D4B1B78022B04D10C4B6A881A802A886B
:108390005A80BDE8F88300232B806B80F0E700BF94
:1083A000FE350020221A0020A00C0020CC0F002057
:1083B000B40C00203811002014250020EC220020ED
:1083C000F8B524220021044611F01DFE00222346A8
:1083D0000521042510460A4FD65D0132042A9E70FD
:1083E000D9701D719871597103F10803F4D10123FB
:1083F0002380522384F8223064232384F8BD00BFF5
:10840000D0A10108F7B5264E3368002B44D0254B88
:108410001B78022B40D10024234D244F04F120006F
:10842000C0B20AF00DF8C8B32B7883BBE25D72B31B
:10843000306850B355218DF8001001218DF80220CD
:10844000AA228DF8011019468DF804308DF803200A
:108450001DF801205340082213F0800F02F1FF3273
:108460004FEA430318BF83F0310312F0FF02DBB27F
:10847000F2D101310429EBD18DF80330AA23052272
:1084800069468DF8043009F0C9F901232B700134D5
:10849000032C05F10105C1D103B0F0BD2870F6E74A
:1084A0004010002047100020441000201FA50108A4
:1084B00038B5194B187808B31849CC88FCB1204658
:1084C0000EF08EFA164B054698680EF08DFA0146AE
:1084D00028460EF0D3F913490EF0DAFA0546204685
:1084E0000EF082FA014628460EF086FB0EF0ACFC38
:1084F0006428A8BF642020EAE070C0B238BD0A4BEF
:108500004D781B880A7800FB15346423521B6343A3
:108510005043B3FBF0F0EBE7341A0020FE350020A7
:10852000182300200000C842221A0020194B2DE910
:10853000F0411C6807460F2C984607DC0023164ABA
:108540009C4206DC0025144EA54208DD0020BDE853
:10855000F08152F823108F42F8D00133F0E756F83B
:108560002530681C7BB98000621B011F92003144DA
:108570003044013411F02DFD46F82570C8F8004054
:108580000120BDE8F0811A7D3B7D9A42EBD3054680
:10859000DAE700BFC0150020C41500201128F8B587
:1085A0000FD00F280CD83422124B02FB003009B137
:1085B000C3684BB90022104D10492C68A24206DB5B
:1085C000F8BD0F4B1868F2E7BDE8F840AEE751F888
:1085D00022709300B84203EB010609D1A21A0433BA
:1085E000920019443046013C11F0F3FC2C60F8BDB8
:1085F0000132E3E7DC000020C0150020C415002094
:10860000A41B002008B50C4B197801290CD00AD303
:1086100002290DD009F040F8084B00F5F42000F5D0
:108620009070186008BD0021002009F0EFF9F1E713
:10863000002009F012F9EDE79C1C0020A01C00208E
:10864000F8B506460D2009F0FBFE10B10A200DF02A
:10865000F9FB294CE268002A4DD02369B3424AD87D
:10866000264BA18A1878576838BB012018707B5CAC
:10867000002B34D01378224A013B126800FA03F32E
:10868000134201D109F096F901221E4B1A70FFF72F
:10869000B9FFA38A43B9E3681B78053B012B03D8D4
:1086A00008F0FAFF184B1860E368A28A5B689B5CCD
:1086B000FE2B0ED10023A382F8BD00251D707B5C2C
:1086C0006BB1284609F076F90E4B1D70FFF79AFF43
:1086D000EAE7FF2B07D1BDE8F8400DF097BBE36850
:1086E000A28A5B689B5C42F2107101FB036301325A
:1086F0002361A282F8BDF8BDA8150020AD35002089
:10870000741800209C1C0020D824002010B50446BA
:10871000204609F077F800B110BD0A2009F00FF8E3
:10872000F6E70023F0B51C46FF260949094D0A78F3
:108730005F57874204BF5E5502F1FF3203F10C031D
:1087400004BFD2B20124302BF2D104B10A70F0BDC3
:108750004C0B00205841002000230C2130B5074C61
:1087600001FB03425568A84203D00133042BF7D123
:1087700030BD0023C3621381536030BD58410020D7
:10878000F8B505460024094EA359A719AB4207D1F5
:108790002846FFF7E1FFCC220021384611F033FCD8
:1087A000CC34B4F5197FEFD1F8BD00BFD40C002054
:1087B0002DE9F04F07464FF000090C2093B00293CB
:1087C0009DF870809DF874A02A4B0591039200FBE0
:1087D00009F2D118D256BA424ED009F10109B9F1C5
:1087E000040FF4D100207FE11F2FFBD1CDF800A0B2
:1087F0004346029A0399012039E00135072D67D1DC
:1088000000256CE00132072A40F08280002287E0D8
:10881000049B53B1711CC9B220B14FF00B0EC17152
:1088200080F806E01A2109F04DF818F0010F00F069
:10883000BD800136F6B215B10C21EE71A9714A2145
:108840002846B1E04FF6DF72236D1A80DA6842F0F5
:108850002002DA6006E1226DD36843F08003D36022
:108860002FE143462846029A0399CDF800A002F072
:10887000A9FD2DE1584100200D89002DB2D11E2FF8
:10888000EFD0B1DC012FADD8994BFEB253F82740A1
:10889000002C00F01C81974BD4F854B02360029B4D
:1088A000DBF80420A36004F15A03636104F5AD739F
:1088B000A3614FF480732265E36023619BF8160087
:1088C0000CF03EFCDBF80C20CAB18B491C208C4616
:1088D00000FB051EDEF804309A428ED1EDB21C2159
:1088E00001FB05C5854B29695869014359610C2174
:1088F0002976711C69762263226D0432E264DBF80A
:108900000810002935D07C4800224FF01C0E054687
:108910000EFB020CDCF8043099427FF473AFD2B244
:108920001C2101FB0255754A2969506908435061B1
:108930000B202876701C687653699BF81900194340
:1089400051616F4A8009AA606A7B8DF81D008DF81D
:108950001C2000228DF81E2001226C6107A88DF8D2
:108960001F200CF00BFCDBF808206263226D043240
:10897000A26494F8580008F07FFF054694F8590067
:1089800008F07AFF08F002031AF0080F04933FF48E
:108990003FAF0136F6B210B10B22C67182711AF0E8
:1089A000100F14BF1A211E2108F08CFFDBF80C20D9
:1089B00012B1DBF808208AB99BF8182007A88DF8B7
:1089C0001C209BF81A309B098DF81D3000238DF870
:1089D0001E3001238DF81F300CF0D0FB0123002640
:1089E00084F84430039B2662E362029BE661A66240
:1089F000666284F80580A36084F806A0204600F033
:108A0000EBFB18F0010F2DD0236B002B3FF41AAFB6
:108A100007A801F085FCE36C206B07934FF48053AB
:108A2000109380230C93E36811960A9320230F93ED
:108A300063690B9608930D960E96099601F09BFCC0
:108A400007A9206B01F079FC226B216D136843F0BC
:108A5000010313608B8A9BB243F040038B825368FF
:108A60009BB22364049B002B2BD0636B002B3FF441
:108A7000F2AE07A801F054FCA36C002507934FF455
:108A80008053109380230C932369606B0A93102307
:108A9000119509930B950D950E950F9501F06BFCB3
:108AA00007A9606B01F049FC636B1A6842F002028F
:108AB0001A60226D5D605D60938A9BB243F0800313
:108AC0009382226D93899BB243F400539381204695
:108AD00050B10C230B4A077103FB0929BDF8143070
:108AE000C9F80400A9F8083013B0BDE8F08F00BF42
:108AF000400B002024A501081400002000100240B3
:108B0000079000085841002038B1038813EA01009B
:108B100003D08B420CBF0120022070470023F0B528
:108B20001D460D490D4E8B75DAB2032A03D905B1E6
:108B30008A750020F0BD5F1C06EBC30436F83330A5
:108B400001321842D2B24FF0010502D08A75204698
:108B5000F0BD3B46E8E700BFA815002032410020E9
:108B60002DE9F74F0120FFF7D9FF0024214D224EB8
:108B700068B3022C2BD84FF0CC0909FB04F855F848
:108B8000087005EB080A17B10134E4B2F0E70323DB
:108B9000C27890F902000093184B019753F82230E5
:108BA00001213A46FFF704FE834640B14A46394662
:108BB0005046013411F027FAE4B245F808B000211C
:108BC000B27D0F4FD3B2032B04D901B1B37503B0FB
:108BD000BDE8F08F02F1010E07EBC20037F832203A
:108BE0000133D207DBB24FF0010101D5B375BFE706
:108BF0007246E7E7D40C0020A81500206CA90108F4
:108C0000324100204000402830B4A8BF402000235B
:108C100002251424064A9D5402339918984201F8FB
:108C2000014CF8D8FF21D1540F2030BC0DF00AB907
:108C3000D019002090F8493013B1002280F8492063
:108C40001846704737B50446056D90F85C106B46C2
:108C500006221830A847A8B101209DF800209DF8F1
:108C6000013043EA0223A3849DF802209DF80330DB
:108C700043EA0223E3849DF804209DF8053043EA8B
:108C80000223238503B030BD37B50446056A6B4621
:108C900006223B210830A847A8B101209DF80020FA
:108CA0009DF8013043EA022363829DF802209DF87B
:108CB000033043EA0223A3829DF804209DF8053087
:108CC00043EA0223E38203B030BD0346012283F866
:108CD000352053F8043C143803B118477047022379
:108CE00010B50168047B0A68A3401A420AD0002428
:108CF000054A40681470026822F001021204120C46
:108D000002604B6010BD00BFAC35002070B504465A
:108D1000192004F1180508F012FD636D00221521D9
:108D20002846984710B9022008F0C7FE94F846205C
:108D3000636D42F01802162128469847636D0022A1
:108D4000172128469847636D01223D212846984700
:108D5000636D2846BDE8704001223E21184713B5D7
:108D60000446C06908F012FE0723104A6946A0694C
:108D700003F04FFAE06908F00EFE01209DF8012093
:108D80009DF8023043EA0223A3849DF803209DF856
:108D9000043043EA0223E3849DF805209DF8063061
:108DA00043EA0223238502B010BD00BF4CA5010891
:108DB00068200CF001BA10B5082204460F211820D3
:108DC0000CF0FAF90E22102118200CF0F5F94FF4EE
:108DD0008053238210BD134B10B51B780446082224
:108DE0002D215320A3B10CF0E7F90A2231215320A1
:108DF0000CF0E2F90C222C2153200CF0DDF990222A
:108E0000382153200CF0D8F94FF48073238210BD21
:108E10000CF0D2F90A22312153200CF0CDF90A22AC
:108E20002C21EEE7FE26002068200CF015BA13B5C1
:108E3000062204466B4601211C200CF00DFA08B3F3
:108E400004219DF800309DF8012042EA032242F3FC
:108E50008D0292FBF1F29DF8023062829DF80320B0
:108E600042EA032242F38D0292FBF1F29DF80530B3
:108E7000A2829DF8042043EA022343F38D0393FB6F
:108E8000F1F3E38202B010BD13B5062204466B462F
:108E9000022118200CF0E0F9B8B19DF801309DF8DE
:108EA00000201B0203EB920363829DF803309DF8C0
:108EB00002201B0203EB9203A3829DF805309DF86C
:108EC00004201B0203EB9203E38202B010BD304B7F
:108ED0002DE9F3411B780546002B3BD000242646A4
:108EE0002746A04601346B46082232215320E4B2C3
:108EF0000CF0B2F918B9002002B0BDE8F0819DF87D
:108F000001209DF80030202C03EB02231BB29DF8BA
:108F1000032098449DF8023003EB02231BB21F4448
:108F20009DF805209DF8043003EB02231BB21E447C
:108F30009DF8073003F07F0301D0002BD2D198FBBE
:108F4000F4F897FBF4F796FBF4F4A5F81280AF82DF
:108F5000EC82D1E76B460622322153200CF07CF9DB
:108F60000028C8D09DF801209DF8003003EB0223B3
:108F70006B829DF803209DF8023003EB0223AB8245
:108F80009DF805209DF8043003EB0223EB82B3E744
:108F9000FE26002010B500222A2104461C200CF0D9
:108FA0000BF902220E211C200CF006F903220F21DE
:108FB0001C200CF001F912222B211C200CF0FCF8D3
:108FC000152008F059FC18B1202383710023C371C8
:108FD000062108F077FC02222C211C200CF0ECF872
:108FE00001222D211C200CF0E7F800222E211C204C
:108FF0000CF0E2F805222A211C200CF0DDF84FF4D9
:109000008073238210BD022210B4047B0168A24049
:1090100043694A6041680A6822F001021204120C96
:109020000A60596A9A6A914203D0184610BC08F047
:10903000B5BB012210BC83F84420704710B5084B23
:1090400007281B68C8BF14381844007E0C4608F077
:1090500013FC20B12146BDE8104008F0A1BC10BDB2
:10906000680C0020F7B5054690F84D00002874D034
:1090700008F002FC044618B1202383710023C37159
:109080000621204608F01EFC354B6B61002C64D095
:10909000A388B3FA83F3C3F11F035A1C50D04FF0D7
:1090A0000F0E30481435C218D6792F4A216842F87D
:1090B0002350DAB202F0030502F0FC0202F1804212
:1090C00002F580329768AD000EFA05FE27EA0E071A
:1090D00001F140419760A1F584319768C1F3872180
:1090E000A9403943012707FA03F39160D9431F4A86
:1090F000536115680D40156055680D405560156841
:109100001D43156095680D409560D5682940D16074
:1091100091680B439360164B9A5DF02A10DDF022A4
:1091200030449A55C37D01A88DF8043003238DF88F
:10913000053000238DF807708DF806300CF01EF80E
:10914000A3880122B3FA83F3C3F11F0312FA03F3D6
:109150001FBF06490A6813430B6003B0F0BD00BF90
:10916000CB8C00084CA50108F80A0020000401403F
:10917000380B0020026D70B515880446ADB2A90603
:1091800006D5036B23B9C36AA3B1908880B2984710
:109190002B0620D5636AA26A9A42236D17D0511C10
:1091A000A069A162825C9A802369994213D300234B
:1091B000A36270BDE169928840694E1CD2B2E6613B
:1091C0004254E169E268914228BFE361E0E7DA686E
:1091D00022F08002DA6070BD70B50446056D8668C5
:1091E000AB8986B023F400531B041B0CAB8183793D
:1091F000617913F0020F14BF4FF40052002213F0F4
:10920000040F14BF4FF48060002011F0010F14BF51
:10921000042300238907298A48BF43F0080389B241
:1092200021F4405111432982AA8922F4B05222F03C
:109230000C021204120C02431343AB81AA8A01A848
:1092400022F440721204120CAA8201F00DF9294A8C
:10925000039B0499954218BF19461922AB894A43CA
:1092600013F4004F14BF7100B100B2FBF1F164269A
:10927000B1FBF6F3AA891801120406FB13132ED5CD
:10928000DA003232B2FBF6F202F0070242EA0003E1
:109290009BB22B81A379DB070BD5236D154A934233
:1092A00025D0A2F57442934203D101200121FFF79A
:1092B000C5FEA379226D13F0080F938A0BBF23F02C
:1092C00008039BB21B0443F0080308BF1B0C9382E6
:1092D00093899BB243F40053938106B070BD1B0188
:1092E0003233B3FBF6F303F00F030343D0E7002060
:1092F000DCE700BF00380140072838B5D8BF044676
:109300000B4BC8BFA0F114041B6805462344187E0C
:1093100008F0B2FA58B127220134C47182711221C7
:1093200008F0D0FA2846BDE83840002186E638BD6E
:10933000680C00202DE9F04300234FF00F0E0126AA
:109340000F8847FA03F2D20723D58C784FEAD30867
:1093500014F0100F18BF91F8039003F0070504F004
:109360000F024FEA850550F828C018BF42EA0902EB
:109370000EFA05F92CEA090CAA4042EA0C02282C44
:1093800040F828200AD1C26806FA03F422EA04024F
:10939000C2600133102BD4D1BDE8F083482CF8D142
:1093A000C46806FA03F22243F2E70348D0F8B0306B
:1093B0000BB1A83018477047140000200348D0F8BC
:1093C00094300BB18C301847704700BF1400002058
:1093D0000248836F0BB170301847704714000020AB
:1093E0000248C36D0BB15430184770471400002079
:1093F0000248036C0BB13830184770471400002046
:109400000248436A0BB11C30184770471400002013
:109410000248836803B11847704700BF140000205A
:109420001FB5074B074A0293074B08490193084BA6
:1094300008480093084B08F09FFC05B05DF804FB5A
:1094400013BF01085DBF01080ABF01081DBF010865
:10945000FEBE0108E3C3010837BF010838B50A4B57
:109460000D4603EBC00494F8B820084853F82210C6
:1094700008F0CBFB94F8BE302BB1691C0448BDE862
:10948000384008F0C2BB38BD6CA5010892CC010879
:10949000F4CE01082DE9F04F00252F46AA465E4E76
:1094A0008BB05E4B5E491A680023934223DB013583
:1094B000102D06F13406F4D1584991F84B30BBB168
:1094C0004FF47A73086E4A6EB0FBF3F35209896E5B
:1094D000544808F051FC0A2297FBF2F39AFBF2F190
:1094E00002FB13775048009702FB11A208F044FCDE
:1094F0000BB0BDE8F08F51F82300864222D0013333
:10950000D3E74346079A0121484808F07EFB4C46C2
:109510003AE038B10DF068FA014645480DF06CFBB1
:109520000DF092FC044642462946424808F06DFB85
:109530004FF0000928E0584631E021463E4808F047
:109540001BFC5BE07368012D0793336BD6F800803A
:109550000893B36AD6F82CB00993F069D9D138B121
:109560000DF042FA014632480DF046FB0DF06CFC5E
:10957000324B81461B78012B90FBF3F4C1D9424654
:1095800001212C4808F041FBBBF1000FD3D041F280
:1095900088314FF47A700BFB0411B1FBF0F0099B9A
:1095A0005B091DBF41F288324FF47A7103FB04223C
:1095B0001A4618BFB2FBF1F21849052D91F84B106D
:1095C0001CBF8244BF180029B7D04FF47A7E089997
:1095D000B1FBFEF104910A2192FBF1FE01FB1E2278
:1095E000039290FBF1F201FB120100920191CDF880
:1095F00008E05A462146124808F0BEFB012D7FF4D0
:1096000056AF0E4B1B78012B7FF651AF4A46079998
:109610000C4808F0B1FB4AE7DC000020C015002030
:10962000C415002053C4010873C401080CC4010808
:1096300000247449FDC301084FC40108582C0020C0
:109640001FC4010843C40108374B2DE9F3411968D1
:109650004FF47A733548B1FBF3F108F08DFB344BCE
:1096600034491A78344B098803EB8203334AD3F820
:1096700030311278324808F07FFB324B324819689B
:10968000324B334FB1FBF3F108F0BFFA08F05DFB4A
:10969000304B314A1C883149314808F06DFB314A62
:1096A000314BA4B2314DD31A2146B7F86C20304863
:1096B00008F062FB2E6D002E33D030460DF094F989
:1096C00001462C480DF098FA0DF0BEFB8046D5F807
:1096D000EC0038B10DF088F9014626480DF08CFAFF
:1096E0000DF0B2FB0446E86938B10DF07DF9014692
:1096F00020480DF081FA0DF0A7FBB7F86E10434635
:1097000064290190A8BF6421009432461A4808F0E9
:1097100033FB1A4B1A48198802B0BDE8F04108F033
:109720002BBBB046D3E700BF801B0020A1C40108BB
:10973000F9350020221A00206CA50108341A0020F7
:10974000BBC4010810000020E1C4010840420F0022
:10975000C0150020B83B0020005000200008000089
:10976000F1C401080000020800F80108DC00002034
:1097700015C50108002474494FC50108343600207E
:1097800095C501082DE9F04F0746304C87B0237886
:109790002F4A608852F8238002F0BEFE2D4BD0F88D
:1097A00004A093F8703082689BB1D346924601269C
:1097B00007F040030593A379721E002B08BF012315
:1097C000934208DC244B08349C42E0D107B0BDE84A
:1097D000F08F9B46EBE7A38813441AF803501BF85D
:1097E0000330EA1AD2F1000949EB020993B9009655
:1097F00043461A4A4946384608F080FBC5B9059BDE
:1098000033B900964346154A4946384608F08CFB62
:109810000136D0E703F00F021B0940330292019397
:10982000009643460E4A4946384608F067FBE5E78E
:1098300005F00F032D09403502930195009643462C
:10984000074A4946384608F06FFBE1E724A60108BD
:109850006CA50108C01500209CA60108B0C5010830
:10986000C4C501082DE9F04F89B007460CF04CFB48
:10987000044628B94120FFF785FF09B0BDE8F08F05
:1098800002469149384610F001FC904D06460028EA
:1098900049D18F4808F08EFC8E4CDFF86C82DFF8DF
:1098A0006C9204F58C77A2882168B2FA82F201F1F9
:1098B0004041A379A1F58431890A413155F823301B
:1098C000C2F11F02404608F0A0F9E17911B1484603
:1098D00008F09BF9083408F038FAA742E3D108F001
:1098E00034FA7D4808F066FC7C4CDFF82482DFF80F
:1098F0002492DFF824A2237E01363246012140461D
:1099000055F8237008F081F9627E39463AB1504625
:1099100008F032FA072E04F11C04ECD1ADE74846FA
:1099200008F02AFAF6E7384607AA6D490DF06EFFEF
:1099300005F1B80782460026B84617F836302246A9
:1099400055F8231050464FEAC60910F09FFB30B17E
:1099500001360F2EF1D1634808F02CFC8DE707AAE1
:109960005F490DF053FF04460DF0F4FE4D4495F8A9
:10997000BE200746EAB9002828DCC844B8F802002F
:1099800002F0CAFDFBB20193019AB8F804302778BF
:109990001344029343680393002F00F092805249CE
:1099A000204610F038FBD8B9039B029A98544F48D0
:1099B000D2E7002805DD1346BB4209DA002A08BFBA
:1099C000012201214A4808F0E4F956E70123F3E7B0
:1099D00007AA434900200DF019FF013F0446CCE7D8
:1099E000A7F14105EDB2072D04D9A7F16105EDB24C
:1099F000072D66D8601C0DF0ADFEC3B20F2B82465A
:109A00005FD86C1C40EA0414E4B2204607F034FF2F
:109A1000002856D0002C49D04FF0000823094033CD
:109A20000493DFF8F89004F00F03059300272FE06C
:109A3000B9F8020002F070FDB9F8043042683B4406
:109A4000D15CA14223D1464504D101998F421ED059
:109A50000021D154059A0499264808F0D6F85FFAF7
:109A600087FB5FFA88F3594618460093FFF7F6FC28
:109A7000464509D1204808F0C8F800985946FFF734
:109A8000EDFC1E4808F0C1F81D4808F093FB0137B3
:109A900099F80630002B08BF01239F42C8DB08F16C
:109AA0000108B8F10F0F09F10809BFD15FFA8AF276
:109AB00005F14101134808F05FF9039B029A9C5499
:109AC000DBE608F07DFBD8E6DAC501086CA50108E5
:109AD000DFC5010834160020EDC501081400002080
:109AE00079CD01080BC60108BFC5010819C60108D8
:109AF00013C601081FC6010843C6010846C601086F
:109B0000D9CC010850C60108E2C50108F4CE01080D
:109B1000F2C5010891CC010804C6010824A6010879
:109B20002DE9F84304460CF0EFF9054620B1012871
:109B30001ED123782A2B1BD1104808F03BFB0024B0
:109B40004FF00D09DFF83C800D4F09FB04863846C5
:109B5000316808F05AF8291C18BF01213046013439
:109B600008F0E8F808F0F1F8B22CEED1BDE8F8837F
:109B70002046BDE8F84309F013BB00BF5CC60108EE
:109B80002DCF0108B8B101082DE9F84F0024804617
:109B900025464FF00D0ADFF85090DFF850B00AFB71
:109BA000049637684146384610F0BEFA78B1394617
:109BB000584608F02AF80021304608F0BBF808F0B3
:109BC000C4F8304608F0ECF808F0BFF8013501346D
:109BD000B22CE4D125B9BDE8F84F024808F0EABA42
:109BE000BDE8F88F6FC60108B8B101082DCF010894
:109BF0002DE9F04F0D468DB0C249044604F0E4F95A
:109C00000646002840F02882BF49204604F0DCF9CF
:109C10000646002840F02282BC49204604F0D4F9D0
:109C20000646002840F01C822046B94904F0CCF9D1
:109C30000028064612BF0824264601240DB144F030
:109C40001004B44DB44FBD42C0F00C820123B34D9B
:109C500085F8703005F046FC03F0CAFBB049304689
:109C600004F0B2F908B144F0200414F0090F00F038
:109C7000DB810020FFF7D4FB04F01803182B04D17C
:109C8000A74807F0EBFF08F060F895F89031A54A77
:109C9000002B0CBF01210021A34B204618BF134607
:109CA000A24A08F041F92046FFF76CFDDFF8E48294
:109CB0009F4B98F800601B789E4FA6EB0309D9F1E3
:109CC000000646EB090607EB83033146D3F83C3127
:109CD000994A204608F012F998F80030314607EB0F
:109CE0008307D7F83C31944A204608F01DF900213B
:109CF000D5F8A4014FF001060DF05EF800B9064654
:109D000006F001018D4A204608F00EF98C4A2046E3
:109D100002F180018B4E07F029F98B4A8B492046CE
:109D200006F0B2FD96F902104FF00009B1FA81F188
:109D3000874A4909204608F0F7F832468549204607
:109D400004F060F9DFF850B2D5F8A472D5F8A88213
:109D5000814B53F82960002E40F08B81B14668EAB0
:109D60000703DFF838B203937B4B53F82960002ECA
:109D700040F0A081D5F8AC32DFF824920393039A27
:109D8000D5F8B432DFF81CA25340DB43059301271A
:109D9000059A07FA06F31A42039A14BFB8464FF021
:109DA0000008134004934FF00C036C4A414603FB38
:109DB0000623D3F808B014BF4A4652465B462046F5
:109DC00008F09CF8049A5B46002A14BF52464A46A3
:109DD000414620463E4408F0A7F8132ED7D1002371
:109DE0005F4EDFF8C4E1DFF8C4C19A5D13F80E10CE
:109DF0000CA8104400F8181C13F80C000DF13008E2
:109E0000804408F80C1C2FB1A2EB0008D8F1000721
:109E100047EB08070133082BE7D1002609AB514A6D
:109E2000394620468DF8206008F068F806AB4D4AA8
:109E30003946204608F078F84B4A4C49204608F04D
:109E400085F84B4A4B49204606F000FF4A4A4B49E9
:109E5000204606F067FE464A4649204606F0AAFD1F
:109E6000474A204602F1500108F0E4F8454A2046EE
:109E700002F15A0107F0B8F9434A4449204606F076
:109E8000DFFF4FF00108DFF828A1DFF828B17300E9
:109E900003931AF816201BF816309A4240F03181CD
:109EA00018F80A7018F80B10781A47424741022A2E
:109EB000DFF8809040F0278119211BF808204B44DF
:109EC0004A4393F8243302F2EE2201920093304A7F
:109ED00033463946204608F011F8192218F80A309E
:109EE0003946534303F2EE230193730013F80A300B
:109EF000274A994499F8243320460093334608F0C2
:109F000013F859E093C60108CAD3010881C00108BB
:109F10009AC60108C0E101086CE50108C0150020DF
:109F20009EC60108501700207CC60108A7C601087C
:109F30001C2500206CA50108AFC60108B8C60108A1
:109F400064170020862B0020F82B00208C2C00208A
:109F5000C7C60108EC2C002018A7010894A7010827
:109F600064370020EBC60108324100208841002000
:109F70002434002070360020A4340020F036002065
:109F80007C1800201C1900206C2D00205C2D002066
:109F9000F2C601081F250020D4C60108E0C601084A
:109FA0007EC6010888C6010864AB01083836002067
:109FB0007C2D0020E92A00200136122E08F102082B
:109FC0007FF465AF2146002007F028FF210740F10C
:109FD000B2802146002095F88C6103F0E1FF214614
:109FE000012003F0DDFF2146022003F0D9FF3046B7
:109FF00004F064FF594803F0FDFB2146002095F86A
:10A000008D6103F0B9FF2146012003F0B5FF214621
:10A01000022003F0B1FF30460BF0E4FE4F4803F09E
:10A02000C9FB4F4807F01AFEA20704D5214695F850
:10A030008C0103F0B5FF630704D5214695F88D0127
:10A0400003F09AFF474C484B9C427FD3002385F88E
:10A0500070300DB0BDE8F08F0124EFE50224EDE58E
:10A060000424EBE56A886968A8680DF09BFB143549
:10A07000E9E53378DBB14FF0010A68EA07030AFA31
:10A0800009FA13EA0A0F14BF0121002133465A4688
:10A09000204607F033FF67EA080313EA0A0F5A461F
:10A0A000334614BF01210021204607F03DFF09F18E
:10A0B00001094DE633780BB34FF0010A0AFA09FAA9
:10A0C00018EA0A0F0BD067EA080313EA0A0F5A4688
:10A0D000334614BF01210021204607F00FFF17EA85
:10A0E0000A0F0BD0039B5A4613EA0A0F18BF01212F
:10A0F000334608BF0021204607F016FF09F1010989
:10A1000032E60027D3E64B4493F8243339460093D4
:10A11000164A3346204607F0F1FE154B72009B5C51
:10A120003946994499F82433104A0093204633461F
:10A1300007F0FAFE40E7214695F88C0103F030FF66
:10A14000214695F88D0103F017FF6DE76288A1683D
:10A1500060680DF027FB143475E700BF7FDC010851
:10A160000FC70108C0E101086CE5010802C701083A
:10A170007C2D0020084BDA68D10709D4DA68520731
:10A1800008D4DB6813F0100F14BF032004207047BD
:10A190000120704702207047002002402DE9F04165
:10A1A0000E46054607464FF6FF7443189F4211D1ED
:10A1B000DFF83880BD4212D1E1B2D8F8000007F0D4
:10A1C0002AFBD8F80000210A07F025FBB01CC0B21A
:10A1D000BDE8F08117F8012BA41AA4B2E6E715F840
:10A1E000011BD8F8000007F016FBE3E7141A002063
:10A1F00007B58DF80610090A8DF80710042106230B
:10A2000060F05F008DF805000DEB01008DF8043063
:10A21000FFF7C4FF03B05DF804FBA0F17D03012B41
:10A2200070B504460D460B4E11D87D21706807F0BD
:10A23000F2FA84F02001706807F0EDFA35B1288851
:10A24000204400EB102000F0FF00288070BD014684
:10A25000F1E700BF141A00205E2810B50146094C32
:10A2600009D15D21A06807F0D6FA3E21A068BDE8BB
:10A27000104007F0D0BA5D29A068F8D107F0CBFAFA
:10A280003D21F3E7141A0020F0B50C46054689B0CD
:10A290001422002120460FF0B6FE04A92A680023EC
:10A2A0000D461D4EC2F3855040FA03F7FF0748BF25
:10A2B0009F5D03F1010344BF0F700131062BF3D101
:10A2C000002315480B70C2F3032101448979C2F3BE
:10A2D00005368DF818100D300DF1190146FA03F707
:10A2E000FF0748BF1F5C03F1010344BF0F7001313A
:10A2F000062BF3D100230B70C2F38343029306AB0A
:10A300000193009502F00F030449C2F303122046A3
:10A310000BF0BEF909B0F0BD00A9010816CB010889
:10A320000023036043608360C36003614361836112
:10A33000C36103624362836270478B6810B50C6A25
:10A34000026823430C6922F4FF4223434C6922F044
:10A35000700223438C692343CC6923434C6A234313
:10A360008C6A234313430360CB6843600B688360AC
:10A370004B68C36010BD036823F001031B041B0C72
:10A3800003600023036043608360C360284B9842EE
:10A3900004D1284A536843F00F0326E0264B984225
:10A3A00004D1244A536843F0F0031EE0234B984243
:10A3B00004D1204A536843F4706316E0204B98425E
:10A3C00004D11C4A536843F470430EE01D4B98427D
:10A3D00004D1184A536843F4702306E01A4B98429C
:10A3E00005D1144A536843F4700353607047174B08
:10A3F000984204D10F4A536843F07063F5E7144B59
:10A40000984201D1134AC5E7134B984201D1114A32
:10A41000C8E7124B984201D10E4ACBE7104B984245
:10A4200001D10C4ACEE70F4B9842DFD1094AD1E760
:10A4300008000240000002401C00024030000240C0
:10A4400044000240580002406C000240800002407C
:10A4500008040240000402401C0402403004024090
:10A460004404024058040240214A10B5536803F0E6
:10A470000C03042B25D0082B26D01E4B03605368F9
:10A480001D49C3F303130B44DC7C0368E3404360C2
:10A490005468C4F302240C44E47C23FA04F484607A
:10A4A0005468C4F3C2240C44E47CE340C3605268A3
:10A4B000C2F38132114491F82320B3FBF2F303611C
:10A4C00010BD0E4B1B68D9E753685168C3F3834333
:10A4D000C90303F1020302D409494B43CEE7516893
:10A4E00011F4003F0549096818BF4908F5E700BFA6
:10A4F0000010024000127A0000A90108D8000020D4
:10A5000000093D0010B50446FFF734FE012806D1CE
:10A510000CB9052010BDFFF72DFE013CF6E7002C1D
:10A5200008BF052010BD0B88F0B54E88B1F804E0D7
:10A530000F89CC88002B3CD1038C23F001031B0432
:10A540001B0C0384018B824B89B221F0F301058C33
:10A550004EEA010141EA07119842ADB289B212D028
:10A5600003F5006398420ED0B0F1804F0BD0A3F5F5
:10A570009833984207D003F58063984203D003F5DF
:10A580008063984212D125F0020546EA050343F0A4
:10A59000010301830384038B23F00C031B041B0CB6
:10A5A0000383038B9BB21C430483F0BD25F00A0593
:10A5B000EBE7042B44D1038C4FEA0E2E23F010035B
:10A5C0001B041B0C0384038B4EEA073723F44073F0
:10A5D0001B051B0D1F435E4B018C984289B2BFB215
:10A5E00012D003F5006398420ED0B0F1804F0BD02B
:10A5F000A3F59833984207D003F58063984203D0BF
:10A6000003F58063984214D121F0200141F010033A
:10A6100043EA06139BB207830384038B23F440634E
:10A620001B041B0C0383038B9BB243EA0424A4B2D8
:10A63000BAE721F0A00146EA010343F01003EAE77C
:10A64000082B038C3FD123F480731B041B0C038461
:10A65000818B3F4B89B221F0F301028C4EEA01015C
:10A6600041EA0711984292B289B212D003F5006311
:10A6700098420ED0B0F1804F0BD0A3F5983398429A
:10A6800007D003F58063984203D003F580639842B6
:10A6900013D122F4007343F4807343EA06239BB280
:10A6A00081830384838B23F00C031B041B0C8383A3
:10A6B000838B9BB21C438483F0BD22F4206333431D
:10A6C00043F48073ECE740F6FF4223F480531B040D
:10A6D0001B0C0384818B038C0A40390341EA0E2151
:10A6E00011431B4A9BB290421FFA81FE12D002F521
:10A6F000006290420ED0B0F1804F0BD0A2F598329C
:10A70000904207D002F58062904203D002F5806249
:10A71000904215D123F4005343F4805343EA0633A7
:10A720009BB2A0F81CE00384838B23F440631B04DA
:10A730001B0C8383838B9BB243EA0424A4B2BAE745
:10A7400023F400735B045B0C334343F48053E8E76A
:10A75000002C01400F4B1A6842F001021A60596840
:10A760000D4A0A405A601A6822F0847222F480323C
:10A770001A601A6822F480221A605A6822F4FE02D3
:10A780005A604FF41F029A604FF00062034B9A60C8
:10A79000704700BF001002400000FFF800ED00E02D
:10A7A00080F30888704702464FF6FF7330B58C1E61
:10A7B000151AAC420BD8014411F8012CB2EB132F3F
:10A7C0000AD1005DDBB2C31A5842584130BD12F8BD
:10A7D000015B5B1B9BB2EBE7002030BD13B5304B38
:10A7E0004278197B02F00F0409B904B11C73197B7C
:10A7F0008C4203D3611AC8B202283ED900204CE033
:10A80000902A13D106238DF80430264B64F06F0490
:10A81000194491F8273004218DF8063002238DF871
:10A8200005408DF807300DEB010034E0A02AE5D19A
:10A830001C4A114491F82720022A19D0032A09D072
:10A84000012ADBD10A21184BB3F94430594301F5F1
:10A85000C87108E00A21DA895143DA7F1AB193F806
:10A86000203091FBF3F189B22046FFF7C1FC14E0E0
:10A87000186B0CF00FFB81B2F6E702F0F002802AB1
:10A88000BED10423022164F07F048DF804308DF8DA
:10A8900005400DEB0300FFF781FC02B010BD00BFC7
:10A8A000141A002000A90108CC3B00204FF6F672D4
:10A8B000074BDA8703F144025A630122998703F1B7
:10A8C000450183F84400996383F84421704700BF31
:10A8D000141A0020002373B502AD25F8023D0C4682
:10A8E0002946FFF79AFCA61D14F8010B2946FFF72D
:10A8F00094FCB442F8D19DF806000021C043C0B2D8
:10A90000FFF78BFC02B070BD07B50B0A8DF8000095
:10A910008DF802108DF80330000A0B0C090E8DF82B
:10A9200001008DF80510102069468DF80430FFF7FE
:10A93000D1FF03B05DF804FB73B50E4C0646D4F8A6
:10A9400048010D46FDF708FFE37D227E003318BF66
:10A9500001230AB143F00803019396F90000009522
:10A960004FF4964300220821FDF722FFC4F8480166
:10A9700002B070BD141A002010B5064CD4F848017E
:10A9800006F046FF00B910BDD4F8480106F03DFFBF
:10A99000F4E700BF141A002008B50B4BD3F84C2184
:10A9A00092781E3A012A08D9D3F8480101210430CF
:10A9B000FFF7C2FFBDE80840DEE70121D3F84801F8
:10A9C00006F01DFFF6E700BF141A00200028114A08
:10A9D000B8BF404290FBF2F330B50F4C04FB0305C7
:10A9E0003C2068430D4D90FBF2F26D7E75B903EB90
:10A9F000830303EB830302EB83030B804FF47A732F
:10AA000004FB020292FBF3F24A8030BDC3EB031356
:10AA1000F1E700BF80969800806967FF141A002054
:10AA200010B50446C0B2FFF717FCC4F30720BDE819
:10AA3000104011E4024B5E21986806F0ECBE00BFA6
:10AA4000141A002038B50546054C5E21A06806F0B2
:10AA5000E2FE2946A068BDE8384006F0DCBE00BF33
:10AA6000141A002073B56F4CD4F8506176B130469B
:10AA700009F09EFF50B194F8543133BBD4F85831EB
:10AA80001BB3A360012384F854311EE094F85C01E9
:10AA900009F0A6FF94F854310546834215D00028EA
:10AAA00000F09D808EB1E37D96F90200B3FA83F346
:10AAB0005B09019302230022009304214FF41653F3
:10AAC000FDF776FEA0600028DCD194F85D0109F066
:10AAD00087FF94F85E31054683421DD0002800F0C0
:10AAE0008580D4F84C31BBB1227E93F90200002A54
:10AAF0000CBF0022082203230192009300224FF48E
:10AB000096430821FDF754FEC4F8480120B1FFF731
:10AB100043FF012384F85E3194F85F0109F060FF80
:10AB200094F860310546834222D0002867D0D4F8DB
:10AB30006421EAB1237E92F90200002B14BF08239E
:10AB40000023E27D2021002A08BF43F00103019386
:10AB50000323002200934FF46143FDF729FE606058
:10AB600030B1012384F8683184F86031D4F86C3155
:10AB700094F8700109F034FF94F87131054683426E
:10AB80002BD0002844D04FF47A72274BC3F8B82258
:10AB9000D4F874310BB31A8802F48252B2F5825F92
:10ABA0001BD093F90200E37D0022002B14BF092380
:10ABB0000823019303234FF4805100934FF4E133B2
:10ABC000FDF7F6FDC4F8780138B1002301222060BA
:10ABD000237384F8712184F87C3102B070BDA068C1
:10ABE000FDF7BAFDA56084F854516EE7D4F848012A
:10ABF000FDF7B2FDC4F8485184F85E518CE76068F7
:10AC0000FDF7AAFD656084F8685184F86051AFE7EC
:10AC1000D4F87801FDF7A0FDC4F8785184F871519B
:10AC2000DBE700BF141A0020D8000020426A806AC7
:10AC3000131A5842584170474171704743799B0736
:10AC40000AD5436A8269D154436A01690133B3FB6F
:10AC5000F1F201FB123343627047437913F00203B0
:10AC600008D00369426A806A013B101A1840C0B2DA
:10AC7000181A704718467047437913F001031FBF35
:10AC8000C369026AC0689B1A1ABF00F1FF301840FE
:10AC90001846704710B54379014613F001030ED0F2
:10ACA000FFF7EAFF60B10B6A4A69CC68D05C0133F8
:10ACB000B3FBF4F204FB1233C0B20B6210BD1846B2
:10ACC00010BD90F8433230B53BB9012490F84112E1
:10ACD00090F84232DAB2914200D830BDB0F84A5210
:10ACE00004FA03F22A43A0F84A220133F2E7836B05
:10ACF00019685A79012393400A8C9BB292B222EAD6
:10AD000003020A840A8C92B213430B84704710F832
:10AD10000A3C0133DBB20A2B00F80A3C07D90023B6
:10AD200010F8131C024A22F8113000F80A3C704750
:10AD3000BC29002070B51424454B1A780132B2FBAF
:10AD4000F4F004FB102298681A705A6C8142DC6897
:10AD50000A4404D293F84C0008B102F580323D4811
:10AD60000678B2FBF6F2944223D293F84C501DB110
:10AD70004FF4803595FBF6F5101B451B1D61DA601D
:10AD800040F68C2200209960196983F84C009142AA
:10AD900041D9187993F94920904230D1021F082AED
:10ADA0002DD893F84A20182A0BD8013283F84A206C
:10ADB00009E04FF4803090FBF6F0001B104418615E
:10ADC000DDE783F8480093F9482090420FD193F8CB
:10ADD0004B1061B10021204C204D914211DB002429
:10ADE0001E490B2A13DD1E490A7801320A7001221E
:10ADF00083F84B20002283F849001A7170BD0022AD
:10AE0000D4E754F8046F25F811600131E5E721F823
:10AE100012400132E5E793F84B20C2B140F2DA521A
:10AE2000A1F2EF20904207D81A790B2A04D803EB3D
:10AE3000820041610132E0E7002283F84B20114695
:10AE400013460848C2180433302B1161FAD170BD83
:10AE5000A81B00201C040020B81B0020BC290020D7
:10AE6000B5290020AC1B002010B51424094B1A781A
:10AE70000132B2FBF4F004FB10221A705A6C01325A
:10AE80000A445A644FF6FF72914204BF012283F8CC
:10AE90004C2010BDA81B00207047704738B5A0F5A6
:10AEA00017746379A579DB0744D594F840321BB356
:10AEB000A06B0268938DC3F34E03938494F85132D0
:10AEC000012B07D094F8453223B1B4F84C3201334A
:10AED000A4F84C32E94301F001010AF08CFA012395
:10AEE00084F84332002384F8413284F8423284F8F3
:10AEF0004032A4F84A3238BD94F843322046012B40
:10AF000004BF94F8413284F84232FFF7DAFE94F835
:10AF100043324BB90123E94384F843321940A06B13
:10AF2000BDE838400AF067BA002305F0010184F853
:10AF30004332F4E738BD10B583790446DB07006B74
:10AF40004CBF2A214A2106F0BDFC012384F844327B
:10AF500084F840320023204684F84132BDE8104096
:10AF6000C5E6084B10B41A681346B3FBF1F4B4F508
:10AF7000803F03D3012BFAD95B08F6E7A1B210BCDE
:10AF800006F0E2BA100000208160806BE9E7837967
:10AF9000406BDB0744BFB1FA81F1490909B106F002
:10AFA000FABC06F0F3BC10B5A0F5157463799A07E6
:10AFB00014D594F84522002A59D1A36A616A9942AE
:10AFC00021D194F844324BB9A3791B0706D5606BA5
:10AFD000062106F077FC2046FFF7ADFF6379D9071D
:10AFE00040F1998094F84032002B40F0948094F81E
:10AFF00041320133DBB2092B84F841324DD1204676
:10B00000BDE810405DE6591CA069A162C35C2069DF
:10B01000DBB25B0043F40073A4F848320A23814298
:10B020004FF0010184F8463294F8443228BFA262FE
:10B0300084F84512002BD1D0A3791807CED5A06B88
:10B0400002684079138C81409BB223EA0103138488
:10B05000138C206B9BB21384062106F033FC002373
:10B06000122184F84432606B06F02CFCB6E794F9A8
:10B0700046327BB1B4F8481220464B08A4F8483257
:10B0800001F00101FFF783FF94F84632013B84F899
:10B090004632A3E784F84532A0E70A2B3BD194F867
:10B0A00043322BB9B4F84A3243F00103A4F84A32D0
:10B0B000B4F84A02820501D4C3071AD4B4F84E3258
:10B0C0000133A4F84E320122002384F8402294F880
:10B0D000432284F84132012A1DD1A179A06B84F862
:10B0E000433201F001010AF086F92046BDE8104024
:10B0F000FDE5E36AC0F347000BB19847E3E7E36976
:10B100006269D054E369E1680133B3FBF1F201FBFA
:10B110001233E361D7E710BD182370B50E465843CC
:10B12000074A14181558A16830460BF0B1FCE168C5
:10B130000BF0A6FB0CF09CFC80B2288070BD00BF19
:10B14000802500202DE9F047182550264FF02808CB
:10B150004FF00009144C154F05FB0045A54201D1E5
:10B16000BDE8F087237CCBB1D4F804A0504606F0AC
:10B1700023FAEFF3128386F31288BAF8242008FB2F
:10B18000007092B201324267BAF81420DBB292B278
:10B1900042F00102AAF8142083F3118854F8183BF6
:10B1A000A3F80090DAE700BF80250020A81B00204C
:10B1B00008B50A4A1378D9070FD523F00103137095
:10B1C000074B9B780BB100F0BFFE002006F0F2FBAE
:10B1D000BDE8084004200AF035BE08BDA4350020B3
:10B1E000D43A002038B5334B1B78D90705D5BDE8D4
:10B1F00038400121002006F009BC1B2007F020F98F
:10B200002D4C00283CD004200AF076FE07F02CF9E3
:10B2100000283AD008200AF06FFE284B1B781A0746
:10B2200038D410200AF068FE254B1B88642B36D9D1
:10B2300020200AF061FE234B234D1B6813F0040FFE
:10B2400002D0B5F8F02042B9B5F8F2200AB19B0758
:10B2500003D41E4BB3F8A83033B340200AF04CFEA1
:10B26000238803B1022385F8F43006F015FAD5F8E7
:10B27000F830C01A00281CDBBDE83840FDF7C2B921
:10B28000238823F004032380C0E7238823F00803E6
:10B290002380C2E7238823F010032380C4E7238898
:10B2A00023F020032380C6E7238823F04003238074
:10B2B000D6E738BDA435002034360020ED26002026
:10B2C0002E16002018250020A81B0020CC3B0020B3
:10B2D00070B5314C23783BB1304D2B7823B93048D1
:10B2E00003F058FC01232B70FFF77CFF2D4B1A88CD
:10B2F00002BB2D4A137813F001014BD143F0030335
:10B3000013700A22294BB3F9043093FBF2F3284A55
:10B310001380284B284A1868A3784FF47A7404FBEA
:10B3200003030520C2F8FC30C2F80011BDE87040EC
:10B330000AF088BD194B1B781BB1204BB3F8A8301D
:10B3400043BB92FAA2F3002AB3FA83F308BF4FF08B
:10B35000FF33194A0133D2F800118B421AD0C2F8D8
:10B360000031DBB29B00402BA8BF402300221426F3
:10B370000A20052512495418565404326070A570ED
:10B380009A4202EB010404F8010CF4D3FF230F20CE
:10B390008B54CBE770BD00BF7011002078110020E6
:10B3A000743C002034360020A43500208C3100206D
:10B3B00086100020801B0020A81B0020CC3B002012
:10B3C000D01900202DE9F04F4FF4187489B0984639
:10B3D0009DF84830814E039300F10A03334493F8FB
:10B3E000D0B593F8C435059144430021054658462D
:10B3F0000292019304F096F900210790019804F05D
:10B4000091F98146584606F037FA0690019806F001
:10B4100033FA039B06F5827713F00803049307EBD6
:10B42000040A069A079B00F09B80B9F1000F03D134
:10B43000002009B0BDE8F08F3319C3F83C91C3F880
:10B440003801C3F8340105F10B03DBB210B10B2254
:10B45000C37182714FF418794FF0000B4FF4807272
:10B4600009FB05695E4BC9F81021C9F80431029B3C
:10B47000C9F81421C9F80C319DF80C30029989F8EB
:10B480000A31059BD9F83C01C9F8303104F1400379
:10B490003B44C9F8183104F5A0733B44C9F81C318A
:10B4A00089F80981C9F824B1C9F820B1C9F82CB1CB
:10B4B000C9F828B189F85453A9F850B3A9F852B380
:10B4C00089F848B389F849B3FFF74BFD039BD9F8D6
:10B4D0003C0103F0010109F08EFF424A04F51773A5
:10B4E000C9F86023404A04F5157418F0020F3B4474
:10B4F000C9F858232744C9F85CB362D0D9F8400191
:10B5000000285ED0D9F83C11026809688A4258D0F8
:10B510000122029989F855230193FFF722FD3A464B
:10B520005946D9F8400106F063F8019B5A4619467E
:10B53000D9F83C0106F05CF8049B63B94FF418732A
:10B5400003FB05651221D5F8380106F0BBF901218E
:10B550005046FFF71CFD5046FFF7EDFC504668E7EC
:10B5600018F0010E12D0BBF1000F3FF461AF002BB9
:10B570003FF45EAF3119C1F83C3105F10B03C1F85E
:10B580003421DBB212B10C21D371917118F0020F8A
:10B590003FF460AF019B002B3FF44AAF4FF41873A8
:10B5A00003FB0563C3F83801BEF1000F06D1B9F102
:10B5B000000F3FF43DAFC3F83C9144E7C3F840911E
:10B5C00041E74FF41870002200FB0560194680F82F
:10B5D00055233A46D0F83C01ACE700BFA81B002039
:10B5E0002CA901089DAE0008A7AF00081FB50123D4
:10B5F000ADF808300023ADF80C30ADF80A30094B37
:10B60000ADF8041093F8E83501A9012B08BF032316
:10B61000ADF8062008BFADF80C30FEF784FF05B08A
:10B620005DF804FBA81B002038B510F80E2C04466A
:10B6300050F8043C52B9012220F80C1C00F80E2CE2
:10B64000597918680222BDE83840CFE7002530F864
:10B650000C2C20F80A1C891A89B220F8081C074A09
:10B6600010F80F0C22F8101004F80E5C2A465979D5
:10B670001868FFF7BBFF04F8065C38BDBC29002042
:10B680001823064A10B503FB0020D0F8EC4524B17E
:10B6900008460CF0EDF980B2208010BDA81B0020F8
:10B6A000072800D8ECE77047084609F07FBC0FB4C4
:10B6B00007B504AB53F8042B04490020019301F0B3
:10B6C000A2F803B05DF804EB04B07047A9B6000817
:10B6D0002DE9F74F3A4C0025D4F8008004F10C0115
:10B6E000464608F1300746F8040B04F1180B04F144
:10B6F000240A04F13009685801910BF0A5FB46F8C3
:10B70000040B55F80B000BF09FFBB06055F80A00D6
:10B710000BF09AFB2B4B7061EB1858680CF0A8F9F2
:10B7200009EB05035B6B043527F8020B0C2DBB807E
:10B730000199E0D10025244F08F1280657F825008B
:10B740000BF082FB0135042D26F8020BF6D1002503
:10B75000B4F8743094F87C70A8F83C30B4F87630C3
:10B76000DFF87090A8F83E30B4F8783008F144065D
:10B77000A8F84030B4F87A30A8F84230BD4216DB61
:10B78000124B5B88A8F86430D4F8A430A8F866306F
:10B79000D4F8C430C8F868300D4B1B88A8F86C305A
:10B7A000B4F8D630A8F85E3003B0BDE8F08F59F891
:10B7B00025000BF049FB013526F8020BDEE700BF40
:10B7C0007822002020410020381A0020221A002070
:10B7D000F4350020F822002010B504467F2C04D850
:10B7E000E0B2BDE8104009F0E1BB64F07F00C0B2F8
:10B7F00009F0DCFBE409F1E70EB477B5064607ACC7
:10B80000482054F8045B09F0D1FB202009F0CEFB5E
:10B81000304609F061FB3A2009F0C8FB23462A466E
:10B8200009490020019400F0EEFF04460A2009F0C7
:10B83000BDFB064A033413681B1B136003B0BDE84D
:10B84000704003B0704700BFA9B60008D03A00208E
:10B850000E4BB3F8DC200132A3F8DC20D3F8E02053
:10B860000132C3F8E020B3F8E420013292B2202A7A
:10B8700003BF0022A3F8E420B3F8E620A3F8E420F5
:10B8800004BF0132A3F8E620704700BF78220020F1
:10B8900038B5244B054693F8E8300C46093B012B9C
:10B8A0003ED8452009F082FB284609F07FFB0E2D8B
:10B8B0000DD003D83DB10D2D0ED038BD1E2D06D0B4
:10B8C000FF2D28D038BD2068BDE8384084E72068C7
:10B8D000FFF782FF6068F7E763782078A3B180F014
:10B8E000800009F063FBA468E0B209F05FFBC4F3D9
:10B8F000072009F05BFBC4F3074009F057FB200E5B
:10B90000BDE8384009F052BB09F050FB6068BDE863
:10B91000384009F002BC044809F0DEFA0020EFE7E5
:10B9200038BD00BF7822002090CB01082DE9F04FF0
:10B93000634C8BB0B4F8E4300546624F002B40F006
:10B94000C7803B78012B04D17B78202B01D102F0FA
:10B9500047FD2846FFF7BCFE256849202E4609F022
:10B9600025FBD4F8E000FFF737FF56F8040BFFF78C
:10B9700033FF304609F0F0FE05F1100009F0ECFE4F
:10B9800010264FF0010905F11C08D4F8EC2009FA43
:10B9900006F3134203D0D8F8000009F0BEFB0136CD
:10B9A000132E08F10408F0D1032105F1280009F055
:10B9B000B9FBB4F80031B5F92E00C01AFFF70CFF3F
:10B9C000D4F8EC30D80408D5B4F80601B5F86430E2
:10B9D000C01AC0F30D00FFF7FFFED4F8EC30990455
:10B9E00003D5B5F86600FFF7F7FED4F8EC301A057A
:10B9F00002D5A86E09F091FBD4F8EC301B0403D5F6
:10BA0000B5F86C00FFF7E8FE032105F1300009F0FE
:10BA100089FBD4F8EC30DE0204D5032105F13600B1
:10BA200009F080FBD4F8EC30980204D5042105F12C
:10BA30003C0009F077FB0126B5F944000AF0D4FF79
:10BA4000D4F808110AF01AFF0BF024FAFFF7C4FE2D
:10BA500094F87C9005F14608B14527DCD4F8EC3029
:10BA6000990505D5B5F95E00A0F2DC5009F055FB4B
:10BA700022686260A2601449144B521A1211534397
:10BA80000322013393FBF2F202EB42029B1A702273
:10BA900002FB03132360012384F85C32BB78012B83
:10BAA00001D101F015FE0BB0BDE8F08F38F9020BA3
:10BAB000B5F944300136C01A09F02FFBCCE700BFBE
:10BAC00078220020D43A002084230020B76DDBB612
:10BAD000D4F86032D4F864229A4207D00AA941F817
:10BAE000203D0020C4F86432FFF7D2FE0422B94999
:10BAF00088180EF05FFA60B1D4F868320AA903938F
:10BB0000D4F86C321E2041F8203DC4F86832FFF7AB
:10BB1000BFFE3978B4F8E43078780B44013BB3FBCE
:10BB2000F0F200FB12339942B8D902F059FC2846D2
:10BB3000FFF7CEFD5020D4F80090D4F8048009F02F
:10BB400035FAA268236810681B68626803441068AD
:10BB500009F10405A3EB400009F0DFFA002308F126
:10BB6000040050F8231055F82320521A02A941F876
:10BB700023200133032BF4D10025084609F0ECFD06
:10BB800009F1100008F1100151F8252050F8253076
:10BB90009B1A02AA42F825300135032DF4D1104634
:10BBA00009F02CFA1026012209F11C0B08F11C0ADD
:10BBB000D4F8EC3002FA06F1194208D0DBF80000A4
:10BBC000DAF800300192C01A09F0A7FA019A01369A
:10BBD000132E0BF1040B0AF1040AE9D1002309F139
:10BBE000280008F1280131F9026B30F9022B921B71
:10BBF00002AE46F823200133042BF4D1002602AB19
:10BC000053F82530B600F6B22BB103F108020F2A23
:10BC100061D846F0010615F1FF35F0D20025304617
:10BC200009F0C4F9AA460DF1080B06F00303022B34
:10BC300063D0032B75D0012B07D1BAF1000F52D17D
:10BC40009A46DBF800502D01EDB20BF1040B06AB68
:10BC50005B454FEA9606E8D1BAF1000F02D02846BC
:10BC600009F0A4F9D4F8EC3013F4805506D001257E
:10BC7000B9F86420B8F86410521A02929A040AD5EE
:10BC80000AAA02EB8501B8F86600B9F8662001350A
:10BC9000121A41F8202C1E050AD50AAA02EB8500CB
:10BCA000D8F86810D9F868200135521A40F8202CCD
:10BCB00018044AD50AAB03EB8502B8F86C10B9F842
:10BCC0006C3001355B1A42F8203C012D68D1029896
:10BCD00009F023FA3BE08033FF2B94BF46F00206C5
:10BCE00046F0030697E7DBF800004FF0000A00F08B
:10BCF0000F00284309F05AF9A7E7BAF1000F04D161
:10BD00009BF8000009F052F99FE7DBF80000C0F350
:10BD10000310284309F04AF9DBF800502D01EDB279
:10BD200093E7BAF1000F04D19BF8010009F03EF946
:10BD3000E6E7DBF80000C0F30330284309F036F9EA
:10BD4000DBF80000C0F30710E4E7002DBDD10321AC
:10BD5000302002F0A1FBD4F8EC30D90203D5032146
:10BD6000362002F099FBD4F8EC309A0203D5042176
:10BD70003C2002F091FB94F87C10442002F08CFBF4
:10BD8000D4F8EC309B0506D5B9F95E00B8F95E3001
:10BD9000C01A09F0C2F963682268A36062606AE6AB
:10BDA00000206B1E02AA52F823204000C0B20AB144
:10BDB00040F0010013F1FF33F4D209F0F7F8002648
:10BDC00002AB53F8260008B109F0A7F90136AE42DC
:10BDD000F6DBBCE7E02400202DE9F74FA3EB020BD4
:10BDE00016460E9B0D9A002914BF062504259B1AA2
:10BDF00001934F4B0446D3F8782289460132984686
:10BE000029D1D3F87422954240F28F80DFF834A113
:10BE10005AF822000AF078F80B3008F0F9FF0746CC
:10BE200018B1012003B0BDE8F08FD8F87412414872
:10BE30005AF82120032994BF21464946FFF737FCD1
:10BE40003D4988F87C720A68101AD8F87822086090
:10BE50000132C8F87822DFF8E090D8F878420C9BDD
:10BE60009C421BDB13D1012008F0D2FF78B9324984
:10BE70000A200A68013A0A6009F098F8D8F8742292
:10BE80000132C8F874224FF0FF32C8F87822D8F88F
:10BE90007402854294BF00200120C3E70D9B53B17B
:10BEA000019B04FB03F20D9B995C01228A40D8F8A8
:10BEB000EC100A4228D004FB0BF4D8F8742237198E
:10BEC00042BB30590AF020F800F1050A504608F04C
:10BED0009FFF0028A5D1D9F8000098F87C22A0EB9C
:10BEE0000A00C9F80000C2B12C2009F05FF8D8F8A8
:10BEF0007422B2B9305908F0EFFF97F904104B1CC7
:10BF000002D00E48FFF7D3FBD8F878220132C8F8E8
:10BF10007822A2E74FF0030AD8E7012288F87C22B2
:10BF2000E5E7174439790648ECE700207AE700BFD7
:10BF3000782200209BCB0108D03A0020AACB010830
:10BF4000F5CE010854A9010810B50C4C94F8E8206E
:10BF50000B2A0BD8012340F60301934019400CD162
:10BF600013F4C06F02D0FF20FFF792FC044B1B6854
:10BF7000C4F878320B2384F8E83010BD7822002012
:10BF8000801B00202D2343702E23C3702F23437169
:10BF90007047074B984209BF064A4FF0FF30538B5A
:10BFA000013301BF9BB25383508B80B2704700BFF7
:10BFB00000380040740C002070B50124B0FBF4F58B
:10BFC0008D4202D21CB91C7070BD4C43F6E7B0FB29
:10BFD000F4F6092E0BDD002A14BF3725572535440A
:10BFE00004FB160003F8015BB4FBF1F4EAE730252B
:10BFF000F5E703685A1C026019707047002B2DE9A1
:10C00000F04106460F46144614BF4FF030084FF07B
:10C010002008069B13F8012B3AB92546002D0FDCAA
:10C0200024EAE47404E0013CF4E7002CFBDC002487
:10C03000069D641B281915F8011B31B9BDE8F08174
:10C0400041463046B847013DE8E73046B847F1E79A
:10C0500070B50446A56808462B1D013544F8231029
:10C06000E168A5600AF00CFC6668E060B54204BFB8
:10C070000023A360A368043354F823100AF0FEFBE6
:10C080000546E0602068864207DB30460AF0ACFCDB
:10C09000014628460AF0B0FD70BD013020600AF06C
:10C0A000A3FC014628460AF0A7FD4FF07E510AF096
:10C0B000E7FB70BDF8B50E460446016830460AF04D
:10C0C000E7FC616A0AF0DCFB6168054630460AF06D
:10C0D000DFFCA16A0AF0D4FBE168074628460AF0B3
:10C0E000D7FC014638460AF0C9FBA16860623046B9
:10C0F0000AF0CEFC2169064628460AF0C9FC014632
:10C1000030460AF0BBFBA0622846F8BD2DE9F0419D
:10C110000E46044601684769C56930460AF0B8FC16
:10C120006168804638460AF0B3FC014640460AF092
:10C13000A7FBA1698046A0680AF0AAFC0146404618
:10C140000AF09EFBE168804628460AF0A1FC014601
:10C1500040460AF093FB216A804620690AF098FC69
:10C16000014640460AF08AFBA76166612562E061EC
:10C17000BDE8F08100232A22036042702B22C270A6
:10C18000012243604271C3717047024B186805F089
:10C1900042BB00BFA83300202DE9F04101270B4D21
:10C1A000DFF82C802C686A6914400CB9BDE8F08176
:10C1B000B4FA84F3C3F11F0358F8230007FA03F617
:10C1C0000368984724EA06046E61EEE70004014024
:10C1D000F80A002041F4807191FAA1F20029B2FA24
:10C1E00082F208BF4FF0FF320388013A23F0400388
:10C1F0001B041B0C038003889BB223F0380343EA23
:10C20000C2039BB2038003889BB243F040030380C8
:10C210007047F8B584894FF6FF764FF47A740BB9FE
:10C220000120F8BD92B1157801320789BF070FD5FB
:10C230004FF47A74ADB285810589ED0712D58589F1
:10C24000ADB209B10D700131013BE8E7FF25ECE724
:10C25000013CA4B2B442E8D1FFF79BFE003018BF06
:10C260000120F8BD013CA4B2B442E5D1F4E708B521
:10C2700040F2E9330289920708D540F2E93389B2E6
:10C2800081810289D20709D5808905E0013B9BB2F3
:10C29000002BEFD1FFF77DFEC0B208BD013B9BB282
:10C2A000002BEED1F6E7F8B504460F4616461D46BC
:10C2B000406805F06BFB47F080012068FFF7D7FF6F
:10C2C0003346002229462068FFF7A3FF606805F087
:10C2D00062FB0120F8BD70B504460E461546406865
:10C2E00005F054FB31462068FFF7C1FF294620685E
:10C2F000FFF7BDFF606805F04EFB012070BD2DE922
:10C30000F74F254C254E264F54F8033C0093002B45
:10C310003AD02422A1464FF0000814F907BC0021AE
:10C3200002FB0B6528460DF06EFE17F80B3007EB8D
:10C330000B0292F802A0019319F8010F019B984299
:10C3400003D1184605F098FAA86099F80300504503
:10C3500003D1504605F090FAE86008F10108B8F101
:10C36000030FE9D1242101FB0BF17218906858B139
:10C37000D06848B1009BE01F536007EB0B0370507F
:10C3800019799B7911745374064B14349C42BBD1B8
:10C3900003B0BDE8F08F00BFB3A90108703B0020D7
:10C3A00038250020DBA9010810B5427A044632B1D5
:10C3B000036800F10A01406898470023637210BDCA
:10C3C0002DE9F341056906460F46002D3BD1D0F813
:10C3D0000080C8F3090373B300234FF40050D6F86C
:10C3E00000800193FEF78EF8042821D12A4C4FF4E7
:10C3F0000050236943F001032361BBB2A8F8003069
:10C40000FEF780F804283CD108F102030193019B58
:10C410003F0C1F804FF40050FEF774F82369042886
:10C4200023F001034FEAC3434FEAD34323612FD0E4
:10C430006FF0010507E04FF43020FEF763F80428A1
:10C4400005D04FF0FF35284602B0BDE8F081124C10
:10C450004FF43020236943F002032361C4F81480B1
:10C46000236943F040032361FEF74CF82369042855
:10C4700023F002034FEAC3434FEAD3432361ABD017
:10C48000DFE7236923F00103DB04DB0C2361CFE743
:10C49000336804333360D6E700200240F8B5044621
:10C4A0000D4600278E18B54201D12069F8BDE3681A
:10C4B000591CE16015F8012B234404291A72F2D1AA
:10C4C000A1682046FFF77CFFE7602061EBE770B5CD
:10C4D0000D46064644880021C4F30B042246284634
:10C4E0000DF091FD33690A4A934209D3094A9342F8
:10C4F00006D222462846BDE8704019460BF052B9D4
:10C5000023B121462846BDE87040184770BD00BFE2
:10C510006CE5010806E60108064B07498B4202D389
:10C520000023184670471A88C2F30B029042F8D0D5
:10C530001433F3E7C0E101086CE50108024A13680F
:10C5400023EA000010607047681800202DE9F843C6
:10C5500002780346202A00F10100F9D0092AF7D019
:10C560002D2A4BD10346444D1C460026DFF80C8192
:10C57000234614F8012BA2F13007F9B2092943D957
:10C580002E2A09D127463D4CA0463B4617F8010B01
:10C590003038C2B2092A44D91A7802F0DF02452A9B
:10C5A00063D15A782D2A4CD10127023300240A2066
:10C5B000013B13F8012F303AD1B2092947D9B4F51C
:10C5C0009A7F28BF4FF49A744FF07E50A046DFF850
:10C5D000B090B8F1070F3DD8DFF8A08004F0070451
:10C5E000002C3DD1002F42D0014630460AF004FB1A
:10C5F000014628460AF04CFABDE8F8832B2A08BF0A
:10C6000003464FF07E55AFE7414630460AF040FA08
:10C61000064638460AF0E8F931460AF031F906468E
:10C62000A6E70AF0E1F921460AF0E6FA01463046AB
:10C630000AF026F94146064620460AF029FA044641
:10C64000A3E72B2A14BF013302330027AEE700FB18
:10C650000424AEE749460AF01BFAA8F10808B8E737
:10C6600041460AF015FA013CBAE74FF07E50014608
:10C6700030460AF00DFABBE7000080BF0000204101
:10C6800020BCBE4C002330B50C4687B000210546C7
:10C690000093019302930AF0B7FB294900283DD08B
:10C6A00028460AF0EDF827490AF0F2F90AF0CCFB27
:10C6B000054680EAE07003A9A0EBE57008F0FEFFF4
:10C6C000002DACBF20232D2303A88DF8003009F0E6
:10C6D0001BFC012826D130238DF801308DF8023063
:10C6E0008DF8033003A968460DF0B3FC684609F0E5
:10C6F0000BFC0338C5B22A46694620460DF0FFFC04
:10C7000000231149635520460DF0A3FC0DEB0501F4
:10C7100020460DF09EFC204607B030BD28460AF0AA
:10C72000ADF8C0E7022805D130238DF801308DF82F
:10C730000230D7E7032804BF30238DF80130D1E75A
:10C740006F12033A00007A44D9CC010870B506464E
:10C75000B6FBF2F40846154614B12046FFF7F6FF83
:10C7600005FB1464024B1B5D00F8013B70BD00BF6C
:10C77000C9CB0108026810B51146531C036011F8BB
:10C78000024BD31C01605178036093781B0443EA89
:10C790000123111D0160D078234343EA006010BDDE
:10C7A00003685A1C02601A4612F8021B026058788D
:10C7B00041EA0020704738B50446154600680AF083
:10C7C000F1FF22682A44226038BD03685A1C0260C7
:10C7D000197003685A1C02600A0A1A7003685A1C0E
:10C7E00002600A0C1A700368090E5A1C0260197064
:10C7F000704703685A1C026019700368090A5A1CC2
:10C800000260197070472DE9F04F82468B4615463D
:10C810001C46002789B00DF114082978002930D072
:10C82000252904D050460135D8470137F5E76A7805
:10C830004FF00009302A12BF00230123AA78029387
:10C84000A2F1300314BFAE1CEE1C092B0CD8A2F1D0
:10C850003003D9B2092918D9A2F16103052B1AD8DE
:10C86000A2F157030A2B10DD6C2A74D13278751CA3
:10C87000642A00F0AB8022D8252A66D012D8002A7C
:10C88000CBD1384609B0BDE8F08F0A2202FB093946
:10C8900016F8012BDBE7A2F14103052BE4D8A2F146
:10C8A0003703DFE7582A18D0632AB6D12E462178FD
:10C8B0005046D847251D01372C463546ADE7732A2B
:10C8C00037D006D86E2AA8D12E46236804341F60BC
:10C8D000F3E7752A65D0782A9FD143461021A2F14B
:10C8E0005800424204F104064241206807E02D232B
:10C8F00040428DF814300DF1150300220A21FFF794
:10C900005BFB3446CDF80080029B4A4659465046B0
:10C91000FFF774FB074480E72D2340428DF8143065
:10C920000DF1150300220A21FFF746FB3546039C53
:10C93000E8E72E4623684A460093594600235046AE
:10C94000FFF75CFB251D0744B6E72E462521504620
:10C95000D8470137B1E7642A31D00AD8252AF5D063
:10C9600002D8002A8DD0A8E7582A0CD0632A9ED07E
:10C97000A3E7732ADED002D86E2AA6D09DE7752AD7
:10C9800014D0782A99D1A2F158014A4204F1040541
:10C990004A412068434610212C46FFF70DFB3546DF
:10C9A000B0E7261D434600220A219EE7231D03937C
:10C9B000002243460A212068FFF7FEFAB6E7206806
:10C9C000231D00280393A7DB4346ABE72068261D01
:10C9D00000288CDB434690E70FB437B50B4906AB14
:10C9E0000B4853F8042B096800680193FFF70BFF0D
:10C9F0000446084D286804F005FF0028FAD02046B8
:10CA000003B0BDE8304004B0704700BFD80A002032
:10CA1000DC0A0020A833002010B541F221040A44AA
:10CA2000914200D110BD11F8013B80EA0320082398
:10CA300010F4004F4FEA400018BF6040013B80B245
:10CA4000F6D1EDE7F8B51A4D2B789F2B2ED16B78E8
:10CA5000BE2B2BD105221749A81C0DF017FB28BBB4
:10CA6000072229464FF6FF70FFF7D6FF124FEC1D45
:10CA700022884AB1A618BE4218D2052A16D92146E4
:10CA8000FFF7CAFF3446F3E721460222FFF7C4FF4F
:10CA90000222A118FFF7C0FF0634084B641B1C805C
:10CAA00041F60F53C31A58425841F8BD0020F8BD53
:10CAB00000F80108F9BE0108000002082C16002049
:10CAC00080EAE073A3EBE0738B4206DB002801DD14
:10CAD000401A704702D0084470470020704770B574
:10CAE00004460AF0B1F9203040284DD8274D284E91
:10CAF000294620460AF088F9002830D1254D244ED9
:10CB0000294620460AF062F900282ED12249204603
:10CB10000AF07AF900282ED021461C4809F0AEFE12
:10CB200004462146204609F0B3FF05461B4909F09B
:10CB3000AFFF1B4909F0A4FE294609F0A9FF1949D6
:10CB400009F09CFE29460646204609F0A1FF014651
:10CB5000304609F09DFF214609F092FE70BD204647
:10CB6000314609F08BFE0446C2E72046314609F003
:10CB700087FE0446C4E70C4920460AF027F900283E
:10CB8000CFD021460348C9E7002070BDDB0F4940E4
:10CB9000DB0FC940DB0F49C0DB0FC93F92E741B94A
:10CBA0009730083C15A82A3EDB0FC9BF70B5044674
:10CBB00010460E4609F014FF0546304609F014FFF2
:10CBC0000146284609F064FF014606480AF014F8B9
:10CBD0000AF04EFF3C28A8BF3C200128B8BF012026
:10CBE000606070BD0024744938B504462568084665
:10CBF000294609F043FE616809F04AFF294609F019
:10CC00003FFE206038BD0846704770472DE9F04F61
:10CC100000220025624B634EB3F80AC087B0346827
:10CC20004FEA0C2A05901889B4EB0A0A65EB020B4F
:10CC3000A0FB0A4500FB0B55B3F80480E00940EA6D
:10CC400045604FEA08440719D8888E464FEAE51137
:10CC5000A0FB0A4500FB0B5541EB0208CDE9027829
:10CC6000B3F80280200A40EA05604FEAC83410EBAE
:10CC700004084FEA252141EB02099A89B446A2FB38
:10CC80000A0102FB0B11C20D42EA412212F5FA60C1
:10CC90004FEAE15343F10001B0F5FA6FCDE900012D
:10CCA00071F100015DDADDE902670524A2FB0401F0
:10CCB00004FB031100FB03F402FB0144A0FB02018F
:10CCC00021444D104FEA3004361B4FEA900467EBC5
:10CCD000050744EA81748D104FF0FF313248B8EBFC
:10CCE000040869EB0509DDE90045844275EB0101A3
:10CCF000CDE9026722DA40F6AC50002112184B4110
:10CD000002FB03F1A2FB022303EB4103D900D00095
:10CD1000101A41EA527163EB0101341847EB010527
:10CD2000CDE902450B24A2FB040104FB03114910C9
:10CD30004FEA3000B8EB000869EB01090AFB0BF37E
:10CD4000DDE90001AAFB0AAB0BEB430B4FEADA72F9
:10CD500042EA4B02801A4FEAEB7361EB0301CDE923
:10CD60000001DCF80410A1FB082301FB0933540D7A
:10CD700044EAC3245D15DDE90223A21A65EB03032F
:10CD80001D46D30B059A43EA454302B11360BEF139
:10CD9000000F02D0009BCEF8003007B0BDE8F08F46
:10CDA000902700204825002024FAFFFF2DE9F74FA7
:10CDB0006A4CDFF8ACE123880091DEF80810B4F982
:10CDC0000480C3EB211252435B00C3EBE103B4F9CF
:10CDD000021005465943131308FB03F84FEAA8381D
:10CDE00008EBE12101EB8102B1F5FA3802F1800292
:10CDF0004FEAE1794FEA222349F1FF39B4F90820DB
:10CE0000A8FB08AB019308FB09F3A16102FB09F140
:10CE10000BEB430BD31708FB0311A2FB08230B44B6
:10CE20001F03160347EA1257B4F90A2002FB0BF15D
:10CE3000D3170AFB0313A2FB0A011944020A42EAB0
:10CE4000016292194FEA2123E6887B410032A2FB5E
:10CE5000060143F5004306FB03114A10CB1752EAC3
:10CE600003016FD0B4F91060B4F90E0006FB0BF1AA
:10CE7000F7170AFB0711A6FB0AAB00FB09F68B4468
:10CE8000C11708FB0161A0FB08898944DEF80C107A
:10CE90004FEA4846C1F5801E1AEB060A76464FEA6D
:10CEA000494747EAD8374BEB070BF7170026F90736
:10CEB00041EA5E014FEACE7040F6354EB4F90C807F
:10CEC00016EB0A064FEAC80747EB0B07861B61EB18
:10CED0000707A6FB0E010EFB071109F0FBFFB4F9D3
:10CEE00016204E1302FB06FE470B47EAC147D31735
:10CEF00007FB03EEA2FB07235643734407FB0366BD
:10CF0000A2FB07233344560E46EAC3163218B4F97F
:10CF100014604FEA636747EB01037143F71700FBA7
:10CF20000717A6FB00013944C60C46EA41369219A0
:10CF30004FEAE147B4F912607B41100A40EA03600E
:10CF4000320112180DB1120A2A60009B13B11A4661
:10CF5000019B136003B0BDE8F08F00BFA427002041
:10CF60004825002070474FF40063038270474FF458
:10CF7000006303827047037F13B1012B04D0704715
:10CF80004FF48063038270474FF40063FAE737B5CC
:10CF90000C46056D01AB02221B211830A84760B179
:10CFA0004FF48C72BDF804305BBA9BB203F54E535C
:10CFB000103393FBF2F32333238003B030BD38B535
:10CFC000054600BF064C206804F0E0FC29460548F1
:10CFD000FFF74DF9206804F0DEFC00BF38BD00BF4C
:10CFE000BC0F00200038004001224821772008F0C3
:10CFF000E3B801225821772008F0DEB83122F4216D
:10D00000762008F0D9B807B5032201AB00217720BC
:10D0100008F022F99DF805309DF804001B0243EA50
:10D0200000439DF80600184303B05DF804FB08B503
:10D03000FFF7E9FF014B586008BD00BF48250020FD
:10D0400008B5FFF7E0FF014B186008BD4825002038
:10D0500007B506226B46F721762008F0FDF89DF80B
:10D0600001309DF800101B0143EA01339DF80210C6
:10D07000094A43EA1113D3609DF804309DF8031068
:10D080001B0143EA01339DF8051043EA1113936035
:10D0900003B05DF804FB00BF4825002070B50446CE
:10D0A00004F11805FBF7DEFF636D80226B21284633
:10D0B0009847642004F043FB636D03226B212846EC
:10D0C0009847636D94F848201921284698470F2007
:10D0D00004F035FB636D94F846201A2128469847E2
:10D0E000636D18221B2128469847636D18221C2166
:10D0F00028469847636D0222372128469847636D7A
:10D100002846BDE8704001223821184738B504464A
:10D1100004F11805FBF7A6FF636D80226B212846FA
:10D120009847642004F00BFB636D072268212846B2
:10D130009847642004F003FB636D00226B212846AE
:10D140009847642004F0FBFA0122636D6B212846A6
:10D1500098470F2004F0F3FA94F847301B21022B74
:10D160008CBF1A221822636D284698470F2004F0BE
:10D17000E6FA636D18221C21284698470F2004F018
:10D18000DEFA636D94F846201A21284698470F204E
:10D1900004F0D5FA636D94F8482019212846984781
:10D1A000642004F0CCFA636D10223721284698479A
:10D1B0000F2004F0C4FA636D2846012238219847F5
:10D1C000BDE838400F2004F0BABA10B504468021FB
:10D1D0008069FEF7FFFF012004F0A6FA2046FFF762
:10D1E00095FF10226A2104F11800FFF774F86420FB
:10D1F00004F0A5FAA0690221FEF7ECFFBDE810409B
:10D20000012004F091BA2DE9F74F054610461F465C
:10D21000884609F0E5FB4C490446404609F038FCD5
:10D220000146204609F034FC80460AF05BFC0446C7
:10D2300040460AF0D7FB39468346384609F020FBC2
:10D240000146204609F0D8FC9DF830600746012EC3
:10D250004FF000044BD008D3022E5FD02346A346E4
:10D260002646A046A146A2461DE059464FF07E50F4
:10D2700009F004FB4FF07C51814609F009FC4FF0A6
:10D280007E518246384609F0FBFA4FF0404106468F
:10D29000584609F0FDFB394683464FF07E5009F0B1
:10D2A000EDFAD046034631465046019309F0A4FCFE
:10D2B00031462860484609F09FFC31466860404688
:10D2C00009F09AFC3146A860584609F095FC019B8C
:10D2D000E8603146184609F08FFCAC6128616C614A
:10D2E0002C62EC61AC626C6203B0BDE8F08F4FF071
:10D2F0004041584609F0CCFB4FF07E5181463846FC
:10D3000009F0BEFA394606464FF07E5009F0B6FAEB
:10D310004FF07E580346CB46C246C4E74FF07E51DD
:10D3200000F1004809F0ACFA4FF04041064658467B
:10D3300009F0AEFB394683464FF07E5009F09EFA65
:10D34000BA460346A146AEE727D4D236002307B536
:10D350000093034BFFF757FF03B05DF804FB00BFDA
:10D36000F304353F70B50D4609F03AFB04462846F4
:10D3700009F036FB0146204609F03EFC0AF06EFB40
:10D38000014609F07DFA4FF08044054601462046EB
:10D390000AF0AEFC4FF07C510646284609F078FBB7
:10D3A000014620460AF0A4FC4FF07E510446304668
:10D3B00009F064FA0146204609F01EFC70BD012305
:10D3C0004A0901F01F0103FA01F150F822300B4322
:10D3D00040F82230704701234A0901F01F0103FA87
:10D3E00001F150F82230194214BF0120002070478B
:10D3F000002201200A4B19780A4B01299DBF5A705F
:10D400009870094B9A7094BF1A705870012995BF93
:10D410002C220122054B064B94BF1A719A7070475B
:10D42000E40A00203A0C0020B80F0020641100200C
:10D43000D43A0020094A0A4913781844C0B210F0BF
:10D44000800F18BF80381070107813460A78904209
:10D4500002BF00220A701A70704700BFE93A00202C
:10D46000E83A002010B50A4B0A4A1B7842609C1823
:10D47000094A0460127893429DBFD31A0B600023BF
:10D48000C3F1800392BF4B600B604A6010BD00BFC8
:10D49000E93A0020EA3A0020E83A00201FB502A845
:10D4A0006946FFF7DFFF044B00981B681844019B97
:10D4B000184405B05DF804FBE43A0020054B1878E9
:10D4C000054B1B78984236BFC3F18003C01AC018C1
:10D4D000704700BFE83A0020E93A002037B5104C09
:10D4E0002078C0B105238DF8003000238DF801307D
:10D4F00000BF0C4D286804F049FA02236A4601A9CE
:10D500000948FEF786FE286804F045FA00BF9DF83A
:10D51000050000F00100207080F0010003B030BD74
:10D52000C00F0020BC0F00200038004070B5064638
:10D53000044C2568FFF7D2FF18B923685B1BB34280
:10D54000F8D970BD801B00202DE9F04F87B0019302
:10D5500000238246029103920093039A93420CDBCC
:10D56000019B002B40F08880FFF7B8FF002840F0B7
:10D570008380019807B0BDE8F08F029A009952F8B5
:10D580002320013311440091E7E702228DF8142093
:10D590001A0C8DF8152006201A0A8DF816208DF821
:10D5A0001730FFF7C3FF0620FFF709FD0123334AB9
:10D5B000137000BF4FF00008D1462746304B186863
:10D5C00004F0E4F9042305AA00212E48FEF721FE09
:10D5D000029D039B984515DA2B684FEA880B002BB8
:10D5E00044D09F4233D83B465AF80B2000212548AF
:10D5F000FEF70FFE5AF80B303B444AF80B302B680D
:10D60000DF1B2F601E4B186804F0C5F900BF1E4BCE
:10D61000361B1B681C441C4B1C60019BA3B19EB1B4
:10D62000194B1B68DCB23219B2F5807F174A88BFEC
:10D63000C4F58074D26898BF34469342A5D30023C2
:10D64000134A1370134A1370009B981B92E7D9F882
:10D65000002000210B48FEF7DCFD2A68D9F80030D5
:10D66000BF1A1344C9F8003000232B6008F10108E9
:10D67000043509F10409ACE7009ED0E7C00F002093
:10D68000BC0F002000380040E43A0020380400209D
:10D69000E83A0020E93A002030B50B4C0B4D2278D7
:10D6A0002B7885B09A420CD002A96846FFF7DAFEC3
:10D6B0000123022202A96846FFF746FF00232B70D0
:10D6C000237005B030BD00BFE93A0020E83A0020E1
:10D6D00030B50E4D0E4C2A78237885B09A4212D080
:10D6E00002A96846FFF7BEFE0023022202A968468F
:10D6F000FFF72AFFFFF79EFE28782378C31A5842C7
:10D70000584105B030BD0120FBE700BFE93A0020D9
:10D71000E83A002008B545F20820FFF707FF062089
:10D72000FFF74DFC0122064BC7201A70FFF747FC9C
:10D730000023044A1370044A1370044A136008BD9E
:10D74000C00F0020E83A0020E93A0020E43A002027
:10D75000032373B58DF80430030C8DF805308DF874
:10D760000700030A06200E4614468DF80630FFF720
:10D77000DDFEC0B100BF0D4D286804F007F9042399
:10D7800000210DEB03020A48FEF743FD2346002269
:10D7900031460748FEF73DFD286804F0FCF800BF5D
:10D7A000204602B070BD0446FAE700BFBC0F00205F
:10D7B0000038004038B504460B4D204604F0CBF944
:10D7C00030B10A4B0A485978BDE8384004F0D4BA61
:10D7D000204609F0BFFF022804D8C0B208F002FBBF
:10D7E0002C46EAE738BD00BF7FDC010808160020A0
:10D7F000EECB010870B504460A4E0B4D204604F0EE
:10D80000AAF930B1074B09481978BDE8704004F017
:10D81000B3BA204609F09EFF022802D830702C4689
:10D82000ECE770BD081600207FDC0108F2CB010890
:10D830002DE9F743074604F08EF9044620B104F0C1
:10D84000BFFC03B0BDE8F083384601AA2E4909F0B9
:10D85000DDFF2E4FDFF8CC80DFF8CC9070B9022CC2
:10D86000EDD1A6F57A73B3F57A7F2DD94FF4FA622C
:10D870004FF47A71264804F08CFAE2E744B1012CA7
:10D880001ED001AA20490020013409F0BFFFE5E7BE
:10D8900009F060FF051E0DDB3B789D4204DA294646
:10D8A0004846FFF799F8ECE7FF2D03D14046FFF714
:10D8B00093F8E6E7397817480139FFF78DF8C0E7A4
:10D8C00009F048FF0646DCE7FF2D0AD104460F4B5E
:10D8D000114F1D78AC4210DB3146104804F04CFA71
:10D8E000AFE7304609F07CF80B4B324643F8250091
:10D8F00029460B4804F040FAA3E7304609F070F8D7
:10D9000047F824000134E5E779CD0108F42200202E
:10D91000B9D0010825CC0108582500205BCC0108AE
:10D920004ECC010810CC0108FDCB01082DE9F047D1
:10D930000546204FDFF88480DFF87C90DFF894A064
:10D94000284608F0E1FA064650B91B4B1B4A1B78E3
:10D950001B48013B52F82310BDE8F04704F00CBA15
:10D960000246394628460CF091FB40B1002458F895
:10D970002410A1B91348BDE8F04704F01BBC1248BD
:10D9800004F06CF9114C124D54F8041F19B12846DB
:10D9900004F03BF9F8E7BDE8F04704F0D6B93246A9
:10D9A00028460CF073FB01340028E0D189F80040D0
:10D9B0005546C5E7DAC501081C250020ACA60108BC
:10D9C0006ACC01086FC6010874CC0108A8A601083A
:10D9D00091CC01087FDC01082DE9F74F824608F061
:10D9E00093FA474D04462F68E8B9464804F00DF90C
:10D9F0000125454EDFF8348105FA04F33B4206D099
:10DA00000C2303FB04634046996804F0FEF80134DC
:10DA1000132CF1D117B93D4804F020F903B0BDE84B
:10DA2000F04F04F092B90246394950460CF02EFBF3
:10DA3000DFF8D490064668B9364804F00FF9364D41
:10DA400009EB0603996828460C3604F0DEF8FC2E34
:10DA5000F6D1E3E79AF800304FF000082D2B0CBF09
:10DA60004FF0010B4FF0000B4FF00C0304BF0AF115
:10DA7000010A04F1FF3403FB0892966850462246DF
:10DA8000314601930CF002FB019B70BBBBF1000F10
:10DA900019D0B8F1130F0BD1204B2B60204804F0A4
:10DAA000DDF831461C4803B0BDE8F04F04F064B91E
:10DAB000B8F1140F01D16B68EFE7012303FA08F303
:10DAC0001F432F60EAE7B8F1130F03D1C5F800B088
:10DAD0001448E4E7B8F1140F1DBF012303FA08F35B
:10DAE0009F436F6018BF2F60F2E708F10108B8F19B
:10DAF000150FC0D10C4803B0BDE8F04F04F05ABB7D
:10DB0000741800207FCC010894A7010889CC010873
:10DB1000DAC5010874CC010891CC0108FFFF0700A9
:10DB200095CC01089ECC01086FC6010890CC010875
:10DB300070B5134C0546134804F090F8206AFEF7C0
:10DB400033FC606AFAF7E2FD0F4B182019780023C6
:10DB50001E4628348B420BDB40F2DC5003F0E4FD20
:10DB60000A4B0B4A15B10B480B490860DA6070BDCF
:10DB700000FB03F2125902B116800133EAE700BF3D
:10DB800058250020A6CC0108F422002000ED00E07A
:10DB90000400FA05EFBEADDEF04F002010B50C4CCE
:10DBA000206AFEF701FC0023D4F8702184F8E830E5
:10DBB000C4F8683184F86C3144F823200133082B11
:10DBC000FAD10020FFF7B4FF0023236210BD00BF8D
:10DBD0005825002008B501F085FC01F085F9BDE865
:10DBE00008400020A4E708B501F07EF9BDE8084030
:10DBF00000209DE701209BE72DE9FF41074608F043
:10DC000083F908284AD1002501AE7C5D09F0AAFD00
:10DC10002044437803F00303022B08BF203CAC559B
:10DC20000135082DF1D10025DFF87C808DF80C50EE
:10DC30007C5D09F097FD20444378404603F00303E0
:10DC4000022B08BF203C7455E4B221460CF010FAB8
:10DC500028B10135214670190CF00AFA20B104F000
:10DC6000AFFA04B0BDE8F081082DE1D10D4930468E
:10DC700002F0F0FB00230B4C0B481A5D04A90A4488
:10DC8000195C0133082B02F80C1CF6D1002301A902
:10DC900006488DF80C3004F06FF8E2E70028E9D070
:10DCA000DDE700BF3836002064AB0108EBC6010891
:10DCB0002DE9F84F054608F027F9364F0446D7F806
:10DCC0000090B0B9344803F0C9FF0126334D344FFA
:10DCD00055F8241049B106FA04F313EA090F02D0EB
:10DCE000384603F092FF0134F2E7BDE8F84F04F044
:10DCF0002CB802462B4928460CF0C8F978B92A48B6
:10DD000003F0ACFF294C2A4D54F8041F0029ECD035
:10DD10000B78002BF8D0284603F077FFF4E72B7838
:10DD200000262D2B0CBF4FF0010A4FF0000ADFF840
:10DD30006CB004BF013504F1FF345BF82680B8F104
:10DD4000000F04D11B48BDE8F84F04F033BA224657
:10DD5000414628460CF09AF9D0B90120B04002069D
:10DD600001D51548EFE78305FBD4BAF1000F0AD0BF
:10DD7000FEF7E4FB114803F071FF4146BDE8F84FA0
:10DD80000B4803F0F9BF40EA090038600C48F2E79D
:10DD90000136D2E768180020B2CC010818A70108A4
:10DDA000BCCC0108DAC5010874CC010814A701082D
:10DDB00091CC01086FC60108C0CC010895CC0108C0
:10DDC0009ECC010870B5054608F09EF8044690B157
:10DDD000112200210F480CF016F922460E49284660
:10DDE0000CF07BF938B1102C2246294628BF1022AE
:10DDF00008480CF084F9BDE87040084B012013F886
:10DE0000042F002A044A06BF012113460021044AB8
:10DE100004F08AB80C1600207CC601080816002001
:10DE2000A7C6010808B50D4804F0C4F90C4B186AE0
:10DE3000FEF7BAFAFFF76EFCFFF750FB48B113206C
:10DE400008F000F803F081FFBDE80840054804F041
:10DE5000B1B9642003F073FCEEE700BFCCCC01083D
:10DE600058250020D5CC01082DE9FF410A48048837
:10DE7000856846888788D0F80C80FFF70FFB8DE80F
:10DE80008001029033462A462146044803F074FF7D
:10DE900004B0BDE8F08100BF38040020DBCC0108ED
:10DEA000F0B585B0054603F056FE002838D104468B
:10DEB0002B78002B3CD1062C42D1BDF904309AB20C
:10DEC000072A3DD840F2DC54BDF90610A1F2EE223B
:10DED00092B2A24234D8BDF90820A2F2EE2080B25C
:10DEE000A0422DD8BDF90A00814229DC824227DBFD
:10DEF000914225DCBDF90C5005F16404A4B2C82C94
:10DF00001ED8BDF90E40112C1ADC0C27194E07FB48
:10DF100003639980DA8018819D72DC7205B0F0BDD0
:10DF200000220120134905B0BDE8F04002F0ACBC6E
:10DF30002D2B03D0A3F13002092A16D8052C04DDBD
:10DF400005B0BDE8F04004F03BB9284609F002FCFA
:10DF500004AB661C03EB440424F80C0C15F8013FD9
:10DF6000303B092BFAD93446A2E7202BE8D1013502
:10DF70002646F8E7F82B0020022810B50C460CD8EE
:10DF800007F030FF0548FFF715FC03F0DEFE2146E1
:10DF9000BDE81040082003F041BF10BD7FDC010840
:10DFA000022810B50C460CD800F088FF0548FFF792
:10DFB00021FC03F0CAFE2146BDE81040042003F016
:10DFC0002DBF10BD7FDC010870B5044608460E4623
:10DFD00007F09AFF3146024620460CF057F808B188
:10DFE000002070BD09F0BEFB0546304607F08CFFEF
:10DFF000235C1D446A78120701D4002BF0D1013054
:10E00000204470BD2DE9F04F824691460E461546DC
:10E0100000278FB0337896F90280089373780993BC
:10E02000F3780A9396F904300B9396F905300C9324
:10E03000B3790D93B8F1000F04D10FB0BDE8F04FE4
:10E0400003F083BEB9F1000F4CD02B78089C6A789E
:10E050009C4295F90210E87895F904E095F905C01D
:10E0600095F806B03CD1099C944239D1884537D106
:10E070000A9C844234D10B9C744531D10C9C64457C
:10E080002ED10D9C5C4514BF002401240390029105
:10E0900001920093CDF818B0CDF814C0CDF810E07F
:10E0A0003B46114A2146504603F028FF0D9BCDF810
:10E0B000088006930C9B0C4A05930B9B2146049306
:10E0C0000A9B50460393099B07360193089B07352B
:10E0D00000933B46013703F027FF102F9AD1ACE79E
:10E0E0000024D3E74C46E1E736CD01082DE9F0479F
:10E0F0008AB0054607F008FF024630B9954901206D
:10E10000FFF780FF0AB0BDE8F08705229249284654
:10E110000BF0BCFF044660B9702201468D480BF03D
:10E1200072FF204622468D4BC2500C306028FBD136
:10E13000E8E704228A4928460BF0A8FF0446002895
:10E1400041D1284603F00FFD06460028DAD007F03B
:10E15000DBFE0746DFF8308258F824501DB98148AD
:10E1600004F028F8CEE73A46294630460BF08EFFF9
:10E1700001340028F0D1774B0246194603F17006AE
:10E180009A719A705A7003F8072BB342F8D1764B04
:10E1900013F8347003EBC404B84205DB2946734816
:10E1A00003F0EAFD724886E06368C0EBC0021344E6
:10E1B000D3F800E08E1841F802E09A880130B2806E
:10E1C0009B79B371E8E707226A4928460BF05EFFA6
:10E1D0000446002875D1202128460BF049FF064649
:10E1E00007F092FE054680BB634803F00EFD2C4607
:10E1F000624D21462846013403F007FD0E2CF8D16C
:10E2000003F0A3FD0024DFF88491544FDFF88081F0
:10E210000C262146484603F0F8FC002506FB047650
:10E22000DFF870A101233268AB40134214BF4146AE
:10E2300051465348013503F0E8FC0E2DF2D101346C
:10E2400003F083FD082CE3D15CE7304601AA4D4979
:10E2500009F0DCFA4B4E02AD00283DD0022C15D15E
:10E26000029A072A2AD803990D2927D80378722BF6
:10E2700017D06E2B22D10C2353430122374802FAC8
:10E2800001F1C25822EA0102C25013E009F062FA19
:10E2900001AA45F824003146002009F0B7FA0134FC
:10E2A000DAE70C23012053432C4C00FA01F1E0582B
:10E2B0000843E0502F48FFF719FF23E703F080FFE2
:10E2C000F8E7284601AA2F4909F0A0FA00242D4EAC
:10E2D00002AD78B1082C02D103F072FF12E709F009
:10E2E00039FA01AA45F824003146002009F08EFAD7
:10E2F0000134EEE7082CEFD1029B0F2BECD8DDF8B0
:10E300000CC0BCF1070FE7D8049F0D2FE4D8059E81
:10E3100006F16402C82ADFD8069DFF2DDCD80798D5
:10E320006428D9D808996429D6D88842D4DA099CB7
:10E33000032CD1D8DFF81CE0C3EBC3020EEB0203C1
:10E340000EF802C05F709E70DD70187159719C717B
:10E3500028E700BF862B002053CD0108F82B0020B2
:10E3600059CD01086FC60108D4A901085ECD010886
:10E370007FDC010868CD010893CC010870CD01084D
:10E3800075CD010879CD0108ACA60108F5CE0108CC
:10E3900053CE010832C1010810B50E2200210446F7
:10E3A0000BF031FE0A23238000236381A381A38025
:10E3B000E380238110BD03788B4286BF024B33F884
:10E3C00011000020704700BFCC260020034B187EB0
:10E3D00010B1002201201A76704700BFCC26002021
:10E3E0007FB5284E28493288284CB2F5805F284BEB
:10E3F000284A096826D31B78C4F8191092F82020FF
:10E4000094F82110E37794F822306177A27784F8AA
:10E410002030532006F0CAFDD4F81900FDF7DCF9CE
:10E42000607FFDF7D9F9A37F01A80193E37F0293F1
:10E4300094F82030039306F0E1FD0023012033809F
:10E4400004B070BD1B7892F82020019194F821103F
:10E450008DF80A3004F1190594F822308DF808106F
:10E460008DF809202946082201A88DF80B300BF001
:10E47000A1FD0028E4D001AB03CBC4F81900C4F817
:10E480001D10C6E754230020E4240020CC260020E1
:10E49000A5350020103600202DE9F04188460024E3
:10E4A0000C4B93E8E000054406440744444501DB77
:10E4B000BDE8F08137F9142036F9143035F914002D
:10E4C0001344022293FBF2F3C01A06F026FE013435
:10E4D000ECE700BF782200202DE9F04F102285B034
:10E4E0000021B3480BF08FFD00263D23B14C2320C3
:10E4F00084F84D30E66103F022F904AB03F80B6DAC
:10E500000122752104F11800FAF78EFC04F11805B8
:10E51000002841D0A84B01222365A84B31466365F2
:10E520004323284684F85C300DF10603FAF77CFC9F
:10E530009DF8063003F07E038DF80630002840F089
:10E54000FD809DF8053003F07E03682B8DF80530C3
:10E5500040F0198106220223114684F84B30266DC3
:10E5600002AB9748B0479DF80D309DF80B209B00FB
:10E57000520002F0020203F0040313439DF8092045
:10E5800002F00102134300F0EF80012B40F0E08025
:10E59000002384F84C3039E08A4BE069A36110B95C
:10E5A0002C2003F069F9884EE06196F8232082B9A7
:10E5B00010B11C23C2718371132103F083F9E06948
:10E5C00003F0E9F90221A069FDF704FE012386F8B2
:10E5D0002330E06903F0DAF9F521A069FDF747FE81
:10E5E0000123002202A9A069FDF713FEE06903F0F0
:10E5F000D2F99DF80830712B00F0918000F28780ED
:10E60000122B00F09780702B00F03D82002384F8DD
:10E610004A3094F84B30022B40F039826B4A22602A
:10E620006B4A62606B4AE2606B4A2262012284F8A4
:10E630004A20073B052B88BF0023684E684F32688D
:10E6400097F8039042F00102326088BFFB71B9F184
:10E65000000F03D0B9F1070F40F0F280FB79B878D2
:10E66000002B00F0E7800323DFF890A184F8473007
:10E67000431E84F8483008F0B7F9514608F008FA0C
:10E6800008F008FCDFF828812368C8F8000084F847
:10E690004690484898473B780BB184F84A304FF091
:10E6A00000094FF0010BCA464E4C06F0BDFE442255
:10E6B00000212046D8F800700BF0A5FC95E8030077
:10E6C000494D04F1080304F1200E83E8030095E8A6
:10E6D0000F008EE80F0035F8053C3B4DA4F81B30C9
:10E6E00095F8278084F81A90B8F10C0F00F2E481B5
:10E6F000DFE818F0B000E201B000DC00EB00000140
:10E70000DC00120112011201120112011201AC2BE4
:10E7100000F0BB81AF2B0FD0732B7FF477AF0623B4
:10E7200084F84B30432384F85C30304B2365304B06
:10E7300063656BE70823F3E70923F1E7682B7FF4B0
:10E7400000AF012384F84B301D2384F85C305DE773
:10E75000022B01D101231CE703F00303032BF9D0A3
:10E76000032003F0AAF951E70DF10703266D0122FA
:10E770000C211348B0479DF8073013F00F03EFD07A
:10E78000042BE7D104E7702B04BF042384F84B303B
:10E790003CE7184A84F84A3022600D4A042362603C
:10E7A000154AA2600B4AE2600B4A226241E700BFB1
:10E7B00020410020CC3B0020298E0008B18D0008AC
:10E7C000E43B002000380040CC2600209DD000080B
:10E7D000458C0008358C000890C1793D1825002033
:10E7E000BA3B0020A82200201C3C0020A7C2000841
:10E7F000D7C200080D8D00088FCF00080000FC4133
:10E80000B84A2260B84A6260B84A063BDBB2E260AE
:10E81000B74A032B226296BFB64A0723D35C012274
:10E8200084F84A20002B00F0408102E7B24A2260BF
:10E83000B24AE8E70223DFF814A384F8473017E769
:10E840000023DFF80CA384F84730012010E74FF0D5
:10E85000000847E704AB03F808AD0122002153206C
:10E8600006F0FAFC10B39DF80830E52B1ED1A44B3E
:10E8700085F832A02360A34B63600423A37633683A
:10E88000A14843F0020333604FF48073238223686E
:10E8900098474FF47A732363AB8E002B4CD195F8D5
:10E8A0002630002B00F00C81A37609E1E37E022BD9
:10E8B0000BD1964B2360964B6360237F002B0CBFDC
:10E8C0006F236E2323760123D8E704AB03F8089D5A
:10E8D00001220D211C2006F0BFFC58B19DF8083024
:10E8E0002A2B01D01A2B05D18A4B23608A4B6360F7
:10E8F0000223C3E704AB03F8089D0122002118207E
:10E9000006F0AAFC40B19DF80830FB2B04D1834BE4
:10E910002360834B6360D6E7E37E042B40F0C9801D
:10E92000804B23607A4BF5E70BFA03F313F4587F1F
:10E9300000F0C2807C4BF4E70027DFF81882A88E35
:10E9400008F04EF8226B014608EB07002C37FEF763
:10E95000FDFC842FF3D1A2E70A2002F0F0FE0DF1B6
:10E9600007030122A021772006F076FC0446002848
:10E9700052D0002701221E21772006F01DFC4FF403
:10E980002F6002F0D1FEB846DFF8CC91A7F160010C
:10E9900002AB0222C9B277208DF808808DF8098079
:10E9A00006F05AFC9DF808209DF8093043EA02233E
:10E9B00027F809300237102FE8D100231946B5F89F
:10E9C000D22002F00F0702F47F42A5F8D22021F0F6
:10E9D00001002844B0F8C400002818BF002411F03A
:10E9E000010F1ABFC0B2434083EA1023082013F47A
:10E9F000004F18BF83F4C05301384FEA4303F6D1E8
:10EA000001311029E3D13A43A5F8D22024B9C3F348
:10EA100003339F4200F0A28095F8D44074BB1420C9
:10EA200002F08DFE414B0122D021762006F014FC2D
:10EA300095F8D530582B01D0012037E03C4B1822F7
:10EA40008821762006F008FC3122F421762006F099
:10EA5000B3FB0123374A85F8D430374B9A60374AE5
:10EA60001C805A6045F6D8125A80354ADA60354A19
:10EA70001A61354A5A6101E0012BDDD0336843F059
:10EA800004033360D8E705234AE6072348E6012B51
:10EA90003FF47FAE042B3FF4B3AE092B05D801221F
:10EAA0009A4012F4587F7FF4C1AE002005B0BDE853
:10EAB000F08F092B7FF638AFB8F1010F3FF6C7AEE4
:10EAC00095F8BC30042BD7D801A252F823F000BF30
:10EAD00059E9000839EA000859E9000859E900082D
:10EAE00019EA00080DD10008458C0008358C000893
:10EAF00090C1793D3FAB0108CBD100085F8D000884
:10EB0000D78D0008CF8E0008A822002077CF0008FC
:10EB1000898C0008958F00082F8E0008B78D00089B
:10EB2000898E000867CF00086FCF0008A12700205A
:10EB3000A427002065CF0008242300200BCC000868
:10EB4000FDCF000851D00008ADCD00080000FA420A
:10EB500000007A44042700209027002042F210721F
:10EB6000064B1A805A80064A5A60064A9A60064A3C
:10EB7000DA60064A1A61064A7CE700BF24230020B7
:10EB8000F3CF000841D00008E9CF00082FD00008DB
:10EB90000DCC0008064B1A684FF47A73B3FBF2F3FE
:10EBA000C3EB431203EB8203DB000380704700BF1B
:10EBB0002041002002392DE9F843426804460368E9
:10EBC000806806290DD8DFE801F0040873767B7EA3
:10EBD000810022605B42636003E05B42524223603B
:10EBE00062603C4B1B78002B60D1206807F0FCFE74
:10EBF0008046606807F0F8FE0746A06807F0F4FE5C
:10EC0000354D0646D5F8F410404607F041FFD5F8DB
:10EC100000118146384607F03BFF0146484607F0A1
:10EC20002FFED5F80C118146304607F031FF014622
:10EC3000484607F025FE08F01BFFD5F8F8102060C5
:10EC4000404607F025FFD5F804118146384607F005
:10EC50001FFF0146484607F013FED5F81011814604
:10EC6000304607F015FF0146484607F009FE08F058
:10EC7000FFFED5F8FC106060404607F009FFD5F8AC
:10EC800008118046384607F003FF0146404607F06A
:10EC9000F7FDD5F814110746304607F0F9FE014696
:10ECA000384607F0EDFD08F0E3FEA060BDE8F8830C
:10ECB000524222608FE75B4223604042A06090E7AF
:10ECC00022606360F9E752426260F6E752422260D6
:10ECD0005B42F6E71D040020CC26002003680A7A78
:10ECE000591C01601A70704738B50546064C2068FB
:10ECF00000B938BD4368EB1A002BFADB8368236048
:10ED000003689847F3E700BF602A002000231A46F3
:10ED100030B5084C037219198D79AD0742BF0979D6
:10ED200081540132D02B03D0072A03F11003F2DD06
:10ED300030BD00BF08BE0108002210B5064C04EB30
:10ED400002118B7913F0010302D00B79037010BD0F
:10ED500001320E2AF3D1F9E708BE0108142201237B
:10ED60004270152203708371C27103712122837076
:10ED700011234271C370704738B54D680446284668
:10ED800007F0C2F8294602462046FDF714FD236825
:10ED90005A1C22603B221A7038BD08B50B4B182054
:10EDA000197800231D460A4C8B4207DB40F2DC50E9
:10EDB00002F0BAFC074A084BDA60FEE700FB03F2F8
:10EDC000125902B115800133EEE700BFF422002092
:10EDD000802500200400FA0500ED00E030B5002297
:10EDE0000C25074905FB02F46318645C844201D1D9
:10EDF000184630BD0132242AF4D1002030BD00BFB6
:10EE00009CAE01082DE9F84F002480469146254626
:10EE10004E01DFF834A006F12007214650465FFA84
:10EE200084FBFEF7D8FA50B1AE4207D8AF4205D9FD
:10EE30005846FFF7D3FF01464046C8470135013425
:10EE4000242CEAD1BDE8F88FCC0C002080B501213C
:10EE5000022002F0DBFD144B1B7803F00503052BA9
:10EE600012D1124B0024186807F0EEFF104B114F1F
:10EE70001D7806B2AC4210DB0F4B1B780BB103F0D0
:10EE800055FD322002F05BFC0021012002F0BEFDA6
:10EE90000021084602F0BAFDFEE7304607F0A4FD67
:10EEA00047F824000134E5E7E50A0020C8260020E1
:10EEB000F4220020F822002058120020022828BF47
:10EEC0000220064B064A18704A2303FB0023054A1A
:10EED0000130C0B21360F9F795BE00BF08160020DC
:10EEE000AA320020102500202DE9F04F8DB001F04E
:10EEF00055FB0326DFF84C914D4FA7EB090718226D
:10EF000000210DEB02000BF07EF84A4B4A4ACDF887
:10EF1000189007975A6002F188325A6001228DF8E2
:10EF20002C203422DA60454B04A918689A889B7912
:10EF30000490ADF8142006A807228DF81630FDF7CE
:10EF4000ADFA072204A94FF6FF70FDF765FD4FF0FB
:10EF5000000A80463A4CDFF8F0B05C4536D3002515
:10EF60000CAC24F82C5D0222214606A8FDF796FA87
:10EF7000022221464046FDF74FFD40BAC04302221F
:10EF8000ADF8080002A906A8FDF788FA099860B153
:10EF900008ABC0F10402294618440BF034F8089974
:10EFA00006A8FDF70DFA09950A909DF82C300A9AEB
:10EFB00023B120490B6943F080030B61013E2DD042
:10EFC000002A9CD1FDF73EFD50B32CE0658806A8D1
:10EFD000C5F30B05AA1DADF8082022888DF80DA0F9
:10EFE000C2F30B01120BADF80A108DF80C2002A928
:10EFF0000622FDF753FA062202A94046FDF70CFD52
:10F00000804661682A4606A8FDF748FA61684046CE
:10F010002A46FDF701FD143480469EE7002AD1D030
:10F02000052002F04AFD01F0A1FA0DB0BDE8F08F15
:10F0300000000208002002402301674544AB01089C
:10F04000C0E1010800F801086CE501082DE9F8436A
:10F05000344B354D5A899989914228BF0022198A2B
:10F0600028BF5A81DA89914224BF0022DA81DA78F6
:10F07000002A50D0072A4ED001222A709A7000220E
:10F080002A4CDA71D9799A78002946D0102A38BFEB
:10F090001022274C9A70987807F0A6FC214607F0BA
:10F0A000F7FC814695F80080224C404607F09CFC16
:10F0B000494607F0EDFCA6780146022E97BF1E4B8D
:10F0C0001B4F03EB86039F68384607F09DFE80B117
:10F0D0004946384607F090FD07F0B6FE1028A8BF55
:10F0E00010200128B8BF0120C0B2404528BF4046CB
:10F0F000287023796BB1013E032E0AD839464FF0B0
:10F100007E5007F079FD08F0B3FC2388984238BFA1
:10F110002080BDE8F883094CB4E7032A38BF0322F6
:10F120009A70B8E7BA3B0020582C00206F12833A3F
:10F130006F1203386823002044AB01086F120339B3
:10F140002DE9F84301F02AFAAC4CAD4FDFF84883C3
:10F15000BC422DD2AB4D00E015462E88002E00F0AB
:10F16000AA81AA19424580F0A681052E40F2A3810A
:10F1700023886988C3F30B039942EDD16B799B0710
:10F18000EAD16168204695F80490FDF7A0F923883C
:10F19000B9EB133F0AD16388B21FC3F30B039A4242
:10F1A000A8BF1A46A91D606808F0FCFA1434CFE71E
:10F1B000954B5A78022A84BF00225A705A78022A44
:10F1C00005D80C20914900FB021291490A601A7877
:10F1D000904E022A84BF00221A701878022806D89E
:10F1E0004A228D4B02FB0030306001F033FA8B4A2B
:10F1F0001178A1F11703022B12D9894BC80013F81B
:10F20000314024B11C1864680CB9172414700344ED
:10F210005B782BB1834B13F831300BB91823137083
:10F22000814B9A78042A40F0DD809A8AB2F57A7F81
:10F2300002D24FF47A729A827C4C7D4A23681A403B
:10F2400012B943F0010323602368DD0702D5794832
:10F25000FDF774F92368580402D57748FDF76EF975
:10F260002368190702D57548FDF768F923689A01E4
:10F2700003D546F20900FDF761F923689B040FD519
:10F280006F48FDF75BF94FF40040FDF757F96D4B00
:10F2900040205A79012A04BF00225A71FDF74EF925
:10F2A000336800259A8CD98C674F914224BF002285
:10F2B0009A84FFF7CBFE2C46B9464FF0FF08EA5B75
:10F2C000530803F07733900800F03330D31A1B1A39
:10F2D000D00800F011301B1A03EB231303F00F3397
:10F2E00093FBF8F012F00101C0EB002018BF0134CD
:10F2F000A3EB000318BFE4B2012B0DDD022B40F09D
:10F30000DF8011B112F42F7F06D109EB050005F063
:10F310004FFB002800F0D4800835202DCFD1013CD0
:10F32000022C00F2CD80494B1B78012B05D8484BAD
:10F33000DA78022A04BF0122DA7003F0D1F8302211
:10F34000002144480AF05FFE002003F03FF8424BE2
:10F3500080F0010034681870404B414A1C60414BFA
:10F360000024197864234B43C83353609460D460FD
:10F37000146154619461D46182F8204082F8214084
:10F3800039493A4A3A4D0A603A4E32F8042C286B11
:10F390003280002840F08280374D384B28881E8804
:10F3A00007F022FB364907F073FB364C6060688833
:10F3B00007F01AFB324907F06BFB6B79324A237274
:10F3C0002B7920606372314B30461A6007F00CFBDA
:10F3D00001462F4807F010FC2E4B1860BDE8F8439B
:10F3E00001F0C4B8002A7FF427AF1A88B2F5F07F85
:10F3F00084BF4FF4F0721A801EE700BFC0E101081D
:10F400006CE5010807F801080816002040110020EB
:10F41000AC2D002010250020AA3200201C25002041
:10F4200088AB0108D4A901086823002068180020CF
:10F430000960000208600002092000020160000269
:10F4400009400002FE35002032410020E40A00207D
:10F45000F0260020D0140020000000200415002019
:10F4600010360020B8310020F8330020F4260020A8
:10F47000A822002000270020FA270020B810002032
:10F4800017B7D138743100203661023DA031002019
:10F49000C0C9FB48BC100020000002080A4F308899
:10F4A00007F09EFA2A6B014638192C34FDF74EFFFF
:10F4B000842CF4D170E761682046FDF708F875E602
:10F4C0000248F8F77DFF2EE7042700203241002094
:10F4D00008B5FFF709FDFFF733FEBDE8084001203E
:10F4E000F9F790BB38B50E4C0E4DAC4211D3002548
:10F4F000FDF77EFF0C4C0D4B0D482570186001F098
:10F50000A9F80C4B0C4A65701A60BDE8384005F04C
:10F51000FDBA61682046FCF7DAFF1434E5E700BF66
:10F52000C0E101086CE50108081600201025002044
:10F53000AA320020AC2D00204011002070B50C290B
:10F5400048D8DFE801F0074747474847474784471F
:10F550004747BE00038C158823F001031B041B0CD6
:10F560000384038C8488018B23F0020321F0730150
:10F570000904090C2943568815891B0435431B0CC3
:10F580002B43674DA4B2A8429BB20FD005F500658E
:10F59000A8420BD005F54065A84207D005F5806567
:10F5A000A84203D005F58065A8420ED1558923F005
:10F5B00008032B43958823F004032B43D6899589B0
:10F5C00024F4407435432C43A4B2D2888480018350
:10F5D0008286038470BD038C148823F010031B04FF
:10F5E0001B0C0384038C8588018B23F0200321F4FA
:10F5F000E6410904090C41EA0421568814891B04D8
:10F6000034431B0C43EA0413454CADB2A04289B20B
:10F610009BB203D004F50064A04213D1548923F0B7
:10F62000800343EA04134FF6BF741C409388D689C5
:10F6300044EA0313948925F44065344345EA84057C
:10F640009BB2ADB2D288858001830287C1E7038C6B
:10F65000148823F480731B041B0C0384038C85889B
:10F66000818B23F4007321F073010904090C2143F9
:10F67000568814891B0434431B0C43EA0423284C8A
:10F68000ADB2A0429BB203D004F50064A04213D1F6
:10F69000548923F4006343EA04234FF6FF341C40EB
:10F6A0009388D68944EA0323948925F4405534434A
:10F6B00045EA04159BB2ADB2D288858081838287EA
:10F6C00087E7038C158823F480531B041B0C0384E9
:10F6D000038C8488818B23F4005321F4E6410904D0
:10F6E000090C41EA0521568815891B0435431B0C7A
:10F6F00043EA05330A4DA4B2A84289B29BB203D0B3
:10F7000005F50065A84205D1958924F4804444EAB2
:10F710008514A4B2D28884808183A0F8402058E761
:10F72000002C014030B598B10A4B00221C461D79CF
:10F73000854207D19D79294202D004EB021030BDE9
:10F740000029FAD001320E2A03F11003EFD1002074
:10F7500030BD00BF08BE01080149024801F090BE5B
:10F76000701C0020000800400149024801F088BEDA
:10F77000481C00200004004002494FF0804001F086
:10F780007FBE00BF201C00200149024801F078BE66
:10F79000F81B0020002C0140FFF7F6BFF0B5002554
:10F7A00041F221072B4624490A78961EECB2B44256
:10F7B00019DB0244941E013A0C440A4464785278DE
:10F7C00002EB042292B293420CD100244FF4AF67B3
:10F7D00091F82450194E0130E3B29D4217D801220E
:10F7E000174B1A70F0BD04440C44647883EA042378
:10F7F000082413F4004F04F1FF344FEA430318BF09
:10F800007B4014F0FF049BB2F3D10135CEE700EB4F
:10F810004303DAB28B1801320A4493F801E05378BB
:10F8200003EB0E239BB27B431B1303F5487326F8AF
:10F8300014300134D0E700BF0C280020CC26002073
:10F84000E426002007298FBF0020034B03EB810132
:10F85000886A80B2704700BF0C2800202DE9F04173
:10F86000174D95F8482012B90020BDE8F08100221C
:10F8700085F8482095F84920A82AF5D195F85C40EC
:10F88000002CF1D10F4F104E05F14908283508EB37
:10F890000403D8781B7903EB002007F0A1F8394660
:10F8A00007F0F6F8314606F0E9FF07F0F3FA45F8FD
:10F8B00014000234102CEAD10120BDE8F08100BF11
:10F8C0000C2800200000203E0080BB43034B03EBCC
:10F8D0004101B1F85E00C008704700BF0C2800204D
:10F8E0001F4BF0B593F87E2019460AB90020F0BDF1
:10F8F000002093F87F40B3F8806003EB440595F84F
:10F90000857095F8862083F87E0042EA07229642A9
:10F91000ECD193F88330012B02D0812B14D0F0BDB1
:10F920001846102C88BF10234FF0000288BF81F8C2
:10F930007F300C4B91F87F40A3F12705D1B28C4268
:10F9400003F1020302D8F0BD0320EAE713F8026CCA
:10F9500013F8011C41EA062125F812100132EDE7E7
:10F960000C2800209128002003788B420CD9074BEB
:10F97000890093F8A7200B44D3F8A80002B14008EF
:10F9800000F5777080B27047002070470C28002087
:10F99000054B03EB8101D1F8D80000EB8000C008D3
:10F9A00000F55C7080B270470C2800205E4B10B5EB
:10F9B00093F82001002800F0B680002293F823413C
:10F9C00093F8240183F8202193F8222104F0070101
:10F9D00042EA012200F03F01490141EAD401C3F8A3
:10F9E000D82093F82521C3F8DC1093F82611920053
:10F9F00093F8274142EA901201F0010042EA802286
:10FA0000C3F8E02093F8280104F00F02D20142EA83
:10FA1000510200F07F01C3F8E420090193F8292185
:10FA200041EA141193F82A415200C3F8E81042EA5F
:10FA3000D01204F0030193F82B0142EA4122C3F8EB
:10FA4000EC2093F82C2100F01F018901D20041EA3B
:10FA5000940142EA501293F82E4193F82F01C3F813
:10FA6000F42093F82D21C3F8F01004F0070142EAC6
:10FA7000012200F03F01490141EAD401C3F8F82016
:10FA800093F83021C3F8FC1093F83111920093F8E9
:10FA9000324142EA901201F0010042EA8022C3F8AA
:10FAA000002193F8330104F00F02D20142EA51021F
:10FAB00000F07F01090141EA1411C3F80811C3F8ED
:10FAC000042193F8342193F83541520004F00301E6
:10FAD00042EAD01242EA4122C3F80C2193F83721BE
:10FAE00093F83601D20042EA501200F01F01C3F829
:10FAF000142193F83821890141EA9401D407C3F80D
:10FB000010114CBF40F21471AD21C3F818119107C8
:10FB10004CBF40F21471AD2112F0080F14BF032046
:10FB20000120C3F81C1110BD0C28002008B5084B9B
:10FB300003EB8101D1F83C0106F052FF054906F0C4
:10FB4000A7FF054906F09CFE07F0A4F980B208BDA6
:10FB50000C28002001F11F3F00405C446B4B30B586
:10FB600093F87C210AB9002030BD002283F87C2163
:10FB700093F87F21162AF6D1082112F0800F4FEA60
:10FB8000420218BF82F0D5020139D2B2F5D193F802
:10FB90007E015F4D02388142C0F2A78093F8961132
:10FBA0009142E0D1182293F8814193F8820183F8C1
:10FBB0007E2193F8802104F0070142EA012200F03F
:10FBC0003F014901C3F83C2141EAD40193F8832164
:10FBD000C3F8401193F88411920093F8854142EAEA
:10FBE000901201F0010042EA8022C3F8442193F808
:10FBF000860104F00F02D20142EA510200F07F01B7
:10FC0000C3F84821090193F8872141EA141193F8B8
:10FC100088415200C3F84C1142EAD01204F00301AB
:10FC200093F8890142EA4122C3F8502193F88A21CE
:10FC300000F01F018901D20041EA940142EA50120A
:10FC400093F88C4193F88D01C3F8582193F88B21D8
:10FC5000C3F8541104F0070142EA012200F03F0109
:10FC60004901C3F85C2141EAD40193F88E21C3F81D
:10FC7000601193F88F11920093F8904142EA90122C
:10FC800001F0010042EA8022C3F8642193F8910157
:10FC900004F00F02D20142EA510200F07F01090193
:10FCA00041EA1411C3F86C11C3F8682193F892214A
:10FCB00093F89341520004F0030142EAD01242EA61
:10FCC000412293F89401C3F8702193F8952100F034
:10FCD0001F018901D20042EA501241EA9401C3F89F
:10FCE0007411C3F87821012030BD6C18E4786240AB
:10FCF000082412F0800F4FEA420218BF82F0D502AA
:10FD0000013CD2B2F5D1013145E700BF0C280020FB
:10FD10008929002070B5304E054633782F4C3BB111
:10FD2000D4F8A43183429EBF0023337084F8A831F5
:10FD30002B4B1B6813F001021CD094F8A92194F8F6
:10FD4000AA3193420CD00123002184F8A831254B1D
:10FD500084F8AA211970D4F8AC312B44C4F8A4312A
:10FD600094F8C83173BBD4F8D801854234BF002061
:10FD7000012070BD13F4005308D013461A4A32F81C
:10FD8000131009BB01330C2BF9D1E9E784F8C83112
:10FD9000D4F8D4319847C307E2D5012300F002001C
:10FDA000002814BF1A46002284F8C8310D4B5A703F
:10FDB0000CBF012300233370D4F8AC312B44C4F8BA
:10FDC000A431CDE7012070BD0123002284F8A831C1
:10FDD000044B1A70F0E700BFA53500200C28002066
:10FDE0000C36002020040020BC2900200020704791
:10FDF000002070470023032BCCBF012200220CBF40
:10FE000005211E2100F8132000EB43020133122BC1
:10FE10005170F0D1704710B500234FF47A744FF44D
:10FE2000FA61C452C2180433102B5180F9D110BDAD
:10FE3000024B03EB4101B1F8B00170470C280020E0
:10FE4000024B03EB4101B1F8B00170470C280020D0
:10FE5000044B93F8DC0118B10022012083F8DC2167
:10FE6000704700BF0C280020024B03EB4101B1F8A2
:10FE7000DE0170470C280020024B03EB8101B1F832
:10FE8000040270470C280020034610B500F16004FE
:10FE9000064A0C3303CA43F80C0C106843F8081CDC
:10FEA00043F8040CA342F3D110BD00BF58AB0108C6
:10FEB00040F2DC5303803223438001230422837306
:10FEC0000023C2731A4630B5084C838119198D7905
:10FED0002D0741BF0D7981180D710132D02B03D050
:10FEE000072A03F11003F1DD30BD00BF08BE010891
:10FEF00070B5054601F0D0FB324CD4F83C32C4F862
:10FF00003C02C31AB3F5FA5F82BF002384F8403283
:10FF100084F8413294F8403233B9A12D1ED1012228
:10FF200084F841221B22227094F841222AB1E2185F
:10FF3000EDB20133557084F8403294F84052237882
:10FF4000AB420AD194F84232052B0ED0062B0FD0CB
:10FF5000002384F8413284F8403270BDA22DE3D1F1
:10FF6000012284F841222322DDE70020FFF716FC5E
:10FF7000A3781E2BECD100200246013DC3B2AB4258
:10FF800007DB25446B789A42E2D10320FFF706FC99
:10FF9000DEE7082123445B78DBB282EA030616F031
:10FFA000010F4FEA530301F1FF310CBFDBB283F0C5
:10FFB0008C0311F0FF01C2F34702EED101301A4663
:10FFC000DCE700BF0C28002010B5044601F064FBFC
:10FFD00041F288310D4BD3F84422C3F84402821A0F
:10FFE0008A4284BF002283F8482293F84822142AC8
:10FFF00003EB02010CBF0122013281F8494014BF1A
:020000040801F1
:1000000083F8482283F8482010BD00BF0C28002048
:1000100010B5044601F040FB254BD3F84C22C3F841
:100020004C02821AB2F57A6F84BF002283F8502204
:1000300093F850224AB9A82C38D183F87E20A3F82F
:100040008020991881F8824006E0022A02D183F8C4
:100050007F40F6E7242AF4D993F87F100132023169
:10006000D2B249008A4283F8502216DA082241F2BD
:100070002101B3F88000E4B280EA042010F4004FBC
:1000800002F1FF324FEA400018BF484012F0FF0271
:1000900080B2F3D1A3F8800010BD01318A4201BFC4
:1000A000002283F85022012283F87E2010BD00BF79
:1000B0000C280020F8B5434C94F85802002859D079
:1000C000002384F8583294F8593294F85A5205EBC8
:1000D000032501F0E1FA3C4BADB2B0FBF3F0D4F8EC
:1000E0006C32002B47D1A4F87052C4F86C02032282
:1000F000D4F8743294F873521E7894F8720294F81B
:100100007872511E631893F859322B4103F00F0394
:10011000B34212D20B2B10D808B183420DD0214428
:1001200091F859E2A11891F859120EEA070E04EB62
:10013000830301EB0E21C3F8A8100232112AE0D18B
:1001400094F87932ABB194F87A3293B194F85B3287
:100150001B060ED501F0A0FAD4F854321B496430C6
:100160001BB15A68121A002A28DB194AD3600432DC
:100170000A600120F8BD9842B9D0C31A012BB2D150
:1001800094F87222002AAED0B4F8703294F8A71016
:1001900092002244EB1A49B16FF01301DB0293FB8A
:1001A000F1F303F50063C2F8A8309CE76FF0130188
:1001B0009B0293FBF1F303F58063F4E703F108017D
:1001C0009B68CDE70C28002020A10700602A0020B2
:1001D0002004002010B5044601F05EFA41F2883197
:1001E0000E4BD3F87C22C3F87C02821A8A4284BF69
:1001F000002283F8802293F880220F2A0DD8511C08
:10020000C9B21A441029E4B282F8594214BF00223C
:10021000012283F8801283F8582210BD0C28002098
:1002200010B5044601F038FA40F6AC51104BD3F843
:100230008422821A8A42C4BF002283F8882293F85B
:1002400088228AB90F2C11D1C3F88402511CC9B27B
:100250001A44192982F8214114BF0022012283F88F
:10026000881283F8202101E0182AEFD910BD00BFC1
:100270000C28002010B5044601F00EFA124BD3F8FA
:100280008C2202F57A72904284BF002283F8902279
:1002900093F8901219B9C3F88C02052204E00229E0
:1002A000FBD993F87E2102328A420CDD481CC0B291
:1002B0008242CCBF00220122194483F8900281F8C7
:1002C0007D4183F87C2110BD0C28002010B5044628
:1002D00001F0E2F9284AD2F89432C31AB3F5FA7F52
:1002E000134628D9002283F8982283F8992293F89C
:1002F0009822C3F8940292B9E1B2042901D02029CE
:1003000021D183F89B1283F89C120221002083F8EC
:100310009D124FF6FF7183F89A02A3F89E12991866
:1003200081F8A04293F89C1201398A4220D101221F
:1003300083F8C02210BD92F899120029D7D0013954
:1003400082F8991210BD93F89B1271B9552C0CD1FB
:1003500001211F2083F89A1283F89B4283F89C02A4
:10036000A3F89E2283F89D12D9E78C42D7D010BD06
:10037000013283F89822FAE70C28002010B5074CC8
:1003800094F87A2242B104F2C121D4F8D80201F0E3
:1003900045FA002384F87A3210BD00BF0C280020F3
:1003A000F8B52A4E96F8C03234460BB90020F8BD95
:1003B000002596F89A3286F8C052012B96F89C12C6
:1003C00032D1314491F89F3291F89E22B6F89E02C4
:1003D00002EB032296F89D3292B203F11C05EDB2B6
:1003E000E61896F8A17296F8A012023301EB0721E5
:1003F000DBB20144AB4288B2F2D18242D6D10022B4
:1004000094F89D52124905EB4203DBB2234493F862
:10041000A10293F8A03203EB002341F8223001320D
:100420000E2AF0D10120F8BD06F52870FAF7BBF9C5
:100430000028BBD096F89B32202BE0D006F5287020
:10044000FAF7CCF986F89902B0E700BF0C28002033
:10045000102A00202DE9F04105460F460446094EBA
:1004600006F10808217809B9BDE8F081054809F0CE
:10047000FFFD20B140453EBF801B631B3B54013450
:10048000F0E700BF64AB010810B500212C22044640
:1004900009F0B9FD0123637223751E23A37540F291
:1004A000DC53238340F24C43638340F26C73A38399
:1004B0000223A377132384F82030062384F8223004
:1004C00040F24653A38440F27533E38440F643037D
:1004D000214623850148BDE81040BBE77BCD0108DC
:1004E000094A92F8DC325BB9084B92F8CC1193F8C8
:1004F00022300433DBB28B4228BF0B4682F8DC3259
:1005000092F8DC02704700BF0C280020383600202B
:10051000124B03EB400393F8DD222AB1022A12D0DA
:100520000F4B33F810007047022809D90328F7D180
:100530000C4B1B6813F4805F0B4B02D1D88C7047B7
:10054000094B188B704793F8DE0200EB800000EB3C
:10055000800000F2EE2080B2704700BF0C2800201F
:10056000CC3500200C3600203836002008B501F0CC
:1005700093F80222064B83F80823C3F80403054BC3
:100580001A68054B9A60012283F8212008BD00BF3C
:100590000C280020801B00201036002008B501F038
:1005A0007BF80222074B00F5B71083F80823064AB0
:1005B00000F55870C3F80403936803F2DC539360AA
:1005C00008BD00BF0C2800201036002070B50024A4
:1005D000114D2146702205F20A3085F8094309F0D1
:1005E00012FD214605F27A34A4F17000631893F9E4
:1005F00002207AB11E680A180E509E889B79073136
:10060000937195F80933702903F10103968085F8F9
:100610000933EBD170BD00BF0C2800200C230B4A1E
:1006200003FB002393F8F7331146FF2B07D092F812
:10063000CC219A4203D9064A32F9130070470C23A1
:1006400003FB0010B0F9F403704700BF0C28002032
:10065000CC35002038B5134A134C054694F84C3479
:1006600010685843114B186006F0BAF9104906F0AB
:100670000FFAC4F85004284602F06EF8284601F03C
:10068000ADFF688D06F0B0F90A4906F001FAC4F82A
:100690005404A88D06F0A8F9064906F0F9F9C4F843
:1006A000580438BD204100200C280020F8240020E8
:1006B000BD3786356F12833A2DE9F04F85B0044679
:1006C00001F049FA064620B101F07AFD05B0BDE817
:1006D000F08F204603AA5E4907F098F83446054695
:1006E000B0464FF0FF37DFF89491DFF894A1DFF8C0
:1006F00094B1BDB90C2639465648FCF76DF9564BF6
:1007000078B206FB05F2D118D256824200F08680FC
:100710000135042DF5D1B8F1000F33D14F48FCF766
:100720005BF9D3E7012E0ED0022E11D01EB9284658
:1007300007F010F8074603AA4549002007F066F8BD
:1007400001360546D5E7284607F004F88046F2E76B
:100750004946284609F0E8FC20B94149284609F0F5
:10076000E3FC08B144F001045146284609F0DCFCE2
:1007700028B95946284609F0D7FC0028DBD044F0B8
:100780000204D8E7002C08BF03240022E4B201923F
:10079000009443461146F8F70BF8054608B931486E
:1007A000BDE741463048FCF717F93048FCF714F92B
:1007B0002F4B1C682046F7F7A9FF2846F7F7A6FF3E
:1007C0000021084601F022F90021012001F01EF964
:1007D000204601F01DF870B10121002001F016F94A
:1007E000204601F012F80146284601F014F80021D5
:1007F000084601F00BF9284601F00AF80028E7D076
:100800000121002001F002F9284600F0FEFF014618
:10081000204601F000F800210846D7E74D68002D7A
:100820003FF479AF1348FCF7D7F854B169798C429B
:1008300007D022461048FCF7CFF8E1B2284600F076
:10084000DEFFEB6A002BB0D00023EB62ADE700BF08
:1008500079CD01088ACD01085841002093CD0108C7
:1008600072C70108ABCD0108C2CD010805CE010851
:100870007C250020D7CD0108E7CD010884CD0108F3
:1008800087CD010897CA01082DE9F04F80468946B7
:1008900016460D4614464FF0000ADFF810B189B035
:1008A000002E6FD06A6863689A4269D1AF68A36806
:1008B000FB1A5F425F4194F90B305A46049394F956
:1008C0000A3039460393B4F9083040460293B4F92C
:1008D00006300193B4F904300093534601F00EFB47
:1008E00095F90B305A46049395F90A30394603932B
:1008F000B5F9083040460293B5F906300C3401933F
:10090000B5F904300C35009353460AF1010A01F0A1
:100910000BFBBAF1080FC3D100242546DFF890A0E5
:1009200096B300270123325903FA07FB59F8043024
:1009300053403BEA030314BF0123002312EA0B0FC9
:10094000079306D000972B4652460799404601F080
:10095000D5FA59F804301BEA030F06D000972B464E
:1009600052460799404601F0DFFA01370E2FD9D1E0
:100970000135082D04F10C04D2D109B0BDE8F08F87
:10098000002798E73746ABE73746012359F804209C
:10099000BB40134206D000972B46524601214046E9
:1009A00001F0C2FA01370E2FEFD1E1E728CE01089E
:1009B00040CE01082DE9F04F054688461446002731
:1009C000DFF8E0A085B0062300267B430393039B5A
:1009D000334408EB030292F8C0B0002C5ED02344ED
:1009E00093F8C0305246ABEB0300D0F1000949EB5D
:1009F0000009019300963B464946284601F07EFADD
:100A00008DE840083B46524649462846013601F0EB
:100A10008BFA062EDBD10137062FD4D10026DFF862
:100A200084B008F1E40A1AF8019B002C38D0A3190D
:100A300093F8E4305A46A9EB03014F424F4101932A
:100A4000009606233946284601F058FA8DE8400200
:100A50000623144A39462846013601F065FA0B2E62
:100A6000E1D198F8F0606CB194F8F0302846F21AB1
:100A7000019300235442544100930A4A072321461C
:100A800001F03CFA002301960093064A0723214611
:100A9000284601F049FA05B0BDE8F08FA146AFE75E
:100AA0002746D3E755CE01087FB5054601F053F838
:100AB000044630B1002218490120FFF77BFF04B043
:100AC00070BD28466A46154906F0A0FE134E01ADDA
:100AD00078B1032C02D101F073FBF0E706F03AFE87
:100AE0006A4645F824003146002006F08FFE0134A6
:100AF000EEE7032CEFD101AC70CC32462946E0B2D0
:100B000003F084FF0028E6D033462A4621460448F5
:100B100001F032F9D3E700BF2434002079CD010879
:100B200055CE01082DE9FF47814690460E461546F1
:100B30000027DFF864A0B8F1000F2AD02B88328894
:100B40009A4224D174886A88A21A54425441EA789D
:100B500021460292AA7848460192009352463B46AB
:100B600001F0CCF9F37852460293B3782146019311
:100B700036F8043B484600933B46013701F0D4F970
:100B8000102F05F10405D6D104B0BDE8F08700248C
:100B9000DDE74446E6E700BF69CE01082DE9F041F4
:100BA000064600F0D8FF044628B1BDE8F041002217
:100BB00022490120B6E7304606F0CCFD0F28054655
:100BC0002EDC304600F0CFFF0646DFF87C801C4F5D
:100BD0002035304606F0BEFD38F81430984226DC49
:100BE000012C11D0022C13D027F8250030462C21DF
:100BF00009F03EFA064678B1012301360134B3B15B
:100C0000032CE6D1BDE8F08107EB85039870EDE792
:100C100007EB8503D870E9E7A21E53425341EDE785
:100C20002146BDE8F0410F22064801F0B2B800238A
:100C300047F82530BDE8F04101F0C2BAA4340020E5
:100C40002434002013C601087CAB01082DE9F04FC5
:100C500007468A46164600248FB0DFF860800DF103
:100C600024095AF82430494602A80293F9F70CFBEC
:100C700016B356F82430029D0393EB1A5D420DF132
:100C8000100B5D41594603A8F9F7FEFACDF800B004
:100C9000234642462946384601F030F92346CDF82E
:100CA0000090424629463846013401F03DF9202C97
:100CB000D7D10FB0BDE8F08F3546EFE77BCE010806
:100CC0002DE9F04F87B0054600F045FF044638B1E6
:100CD000002255490120FFF7B9FF07B0BDE8F08FAA
:100CE000284606F037FD1F28074600F39780284660
:100CF00000F039FFA0460646A246A1462546A34677
:100D0000494B009443F827400193484BE1B2E05C23
:100D100000230DF10C0CB64616F8012B1AB19042C7
:100D20000FD00A2B09D106AE33440026904203F8B7
:100D30000C6C08D001F044FACFE703F80C20013323
:100D4000E9E70246EFE701390EF10106032932D83F
:100D5000DFE801F04E1F025B4FF0010EDFF8DCC050
:100D60000DF10B0010F8011F49B30023304AD25C8B
:100D70008A4203D00133072BF8D15346002212F8E0
:100D80000CA08A453DD10EFA02F248EA02089A46C2
:100D9000E8E74FF0010C0DF10B0111F8012F72B1D2
:100DA0000023244813F800E0964526D10CFA03F3FB
:100DB00049EA0309F1E703A806F0CCFC83460134B5
:100DC000052CA2D1009B05F00F0545EA834545EAB5
:100DD000895949EA0A2A4FEA0B134AEA0838019A64
:100DE000DBB248EA030342F8273003F08FFE74E7D2
:100DF00003A806F0AFFC0546E1E70133062BD0D18E
:100E0000CBE70132062ABAD1C1E703A806F0A2FC5B
:100E100003460F28C8BF00230093D0E71F222146B6
:100E2000054800F0B6FF58E72434002082AB0108E3
:100E300006A9010800A9010813C601080DA90108A7
:100E40002DE9F34781460F46904602260024DFF83D
:100E500060A0B8F1000F28D037F8242038F82430EB
:100E60009A4238F806201ED1BD5BA91A4D424D4169
:100E700001920093524623462946484601F03EF827
:100E8000BB5B5246019337F824302946009348460D
:100E90002346013401F048F8042C06F10406D8D1A9
:100EA00002B0BDE8F0870025E2E74546E8E700BF6D
:100EB00085CE0108F8B5054600F04DFE064628B17E
:100EC000BDE8F840002226490120B9E72549284617
:100ED00009F0A1F868B94FF47A714FF4FA62204B27
:100EE00019805A809980DA8019815A819981DA8132
:100EF000F8BD284606F02EFC0328044628D82846CC
:100F000000F031FE064658B106F024FC01270546E4
:100F1000304600F028FE30B9BDE8F84001F050B985
:100F200005460746F4E706F015FC002FF4D040F222
:100F3000DC53A5F2EE229A42EED8A0F2EE229A42BB
:100F4000EAD8074B23F8245003EB84035880F8BDFC
:100F50003146BDE8F8400322034800F01ABF00BF45
:100F60006C2D002053CD01080FD501082DE9F04F5D
:100F70000E461546002797B008900992D6F80080D3
:100F80000021404605F018FF0446002869D1736827
:100F90000493B3680593F3680693099B002B3DD037
:100FA000D5F800B0EB6859464046D5F804A0D5F80E
:100FB0000890079305F000FF80B15146049805F0B2
:100FC000FBFE58B14946059805F0F6FE30B1079989
:100FD000069805F0F1FE041C18BF012413A9584619
:100FE000FBF750FB10A983465046FBF74BFB0DA9BE
:100FF00082464846FBF746FB0AA981460798FBF75D
:1010000041FBCDF808900390CDF804A0CDF800B0D6
:101010003B46154A2146089800F070FF13A9404648
:10102000FBF730FB10A904460498FBF72BFB0DA936
:1010300080460598FBF726FB0AA981460698FBF730
:1010400021FB3B4603908DE81003074A00210898D6
:10105000013700F069FF082F06F1100605F11005B1
:101060008CD117B0BDE8F08F96CE01082DE9F84F6E
:1010700007460026534D384600F06DFD804628B1E6
:101080000022BDE8F84F4F4901206FE705224E4985
:10109000384608F0FBFF38B900224A4BC2501030E6
:1010A0008028FBD1BDE8F88F04224849384608F073
:1010B000EDFF04463846002C3FD100F054FD814638
:1010C00000287CD004F020FFDFF818A15FFA80FB35
:1010D0005AF82480B8F1000F04D13D48BDE8F84F1C
:1010E00001F068B85A464146484608F0CFFF01343F
:1010F00007460028ECD1374B2E6003EBC404D4F82C
:1011000010E02E612E622E632E642E652E662E67F1
:10111000BEF1000F03D094F80CC0674505DB4146D3
:101120002D4800F029FE2D4FA5E73B01EC18734434
:101130000FCB013784E80F00EFE706F00BFB072821
:10114000054635D8384600F00EFD064628B3FBF7B5
:10115000FDF901241B4A2B01D050304600F003FD5D
:10116000064630B1FBF7F2F9164B013403EB0513D9
:101170005860304600F0F7FC064630B1FBF7E6F960
:10118000104B013403EB05139860304600F0EBFC84
:1011900028B9BDE8F84F01F013B80446DDE7FBF7C6
:1011A000D5F9084B032C03EB0515E860F1D167E78F
:1011B0004146BDE8F84F0722094800F0EABDBDE806
:1011C000F88F00BF6417002053CD010859CD0108E6
:1011D0006FC601087CAB01085ECD01087FDC010809
:1011E00013C60108ACA601082DE9F04F81469046D0
:1011F0000C46154600261927DFF8B0A087B0B8F1D5
:10120000000F51D023782A7893422B794AD1607805
:101210006978884246D1A078A978884242D1E0789E
:10122000E97888423ED1217999423BD16179687948
:10123000081A414241410593EB7848460493AB7844
:101240008B467B4303F5617303936B7801927B4379
:1012500003F5617302936B7952460093334600F0B5
:101260004DFE237952460593E37859460493A378BB
:1012700048467B4303F561730393637806357B43EC
:1012800003F56173029323780634019314F8013C4B
:1012900000933346013600F047FE0F2EAFD107B062
:1012A000BDE8F08F0021C6E7C346DAE7AACE010801
:1012B000F7B5074600F04FFC044630B1002236492E
:1012C0000120FFF791FF03B0F0BD384606F042FA67
:1012D0000E28054659DC06264643781C8DF8074043
:1012E00000F041FC2C4C074650B106F033FA0328BD
:1012F00006D8A31958719DF8073001338DF80730CF
:10130000384600F030FC074658B106F023FA0D28A5
:1013100007D806236B43E0549DF8073001338DF85E
:101320000730711C0DF107022144384600F027FCFC
:1013300000F019FC074660B106F00CFA182808D82E
:10134000062303FB0543D8709DF8073001338DF861
:101350000730384600F007FC60B106F0FBF90D28B5
:1013600008D8062303FB05459DF807302871013393
:101370008DF807309DF80730062BA4D00023A21962
:10138000A351938000F01CFF9DE70E2221460348E5
:1013900000F0FFFC97E700BF1C19002013C60108EE
:1013A00010B5046B0346C168406944B11A6C8C1ACD
:1013B000013A08BF0A46005D1A64C0B210BD1A6A3D
:1013C000805C01328A4228BF2246C0B21A6210BD38
:1013D000436B13B190F844007047836A406A1B1A4C
:1013E000584258417047416A836A0269994238BF3E
:1013F0008918CB1A416B21B149680B44511E8B42AD
:1014000002D2501EC01A704700207047036B4BB1C8
:10141000026C5B689342A3EB02032EBF1846C068C0
:10142000C0187047C269036A9A422FBFD01AC068B9
:101430008018C01A70470A4B30B503F1100493F9B5
:1014400000205D78072AC8BF143A81180D739D7873
:101450000433855413F8012CA3420A76EFD130BD32
:1014600080AE01082323037024234370002383707C
:10147000C37070474171F7F7AFBE8160F7F7ACBE3C
:101480002DE9F047064689464FF000474FF0000827
:10149000038A8589ADB21D400DB9BDE8F087B5FA64
:1014A00085F327FA03F2D2431B3B91B231821540F8
:1014B000042BF1D8DFE803F02925211A0300D9F81D
:1014C000244084B1013CA4B2C9F82480D9F820A0FA
:1014D000BAF1000FE0D0DAF80030504621469847C4
:1014E000DAF804A0F4E7B48DA4B2EFE7D9F800006D
:1014F000B18E036889B29847CEE7D9F80400318FDE
:10150000F7E7D9F80800B18FF3E7D9F80C00B6F87F
:101510004010EEE71FB50023ADF80A30ADF80630F5
:101520008DF80C30074B01391B68ADF80810B3FB80
:10153000F2F204A9013A21F80C2D03F006FF05B0E0
:101540005DF804FB1000002073B504460068FFF747
:10155000E1FF2268174913889BB243F0010313800F
:10156000002351F8334001EBC300A2421DD145795D
:101570000124002601A88DF804508DF805408DF84F
:1015800006608DF8074003F0F9FD1B2D0BD11923E0
:1015900001A88DF804308DF805408DF806608DF8AF
:1015A000074003F0EBFD02B070BD0133042BD8D12E
:1015B0000025DDE778A101080B4B800A98420FD087
:1015C00004D8B0F5801F09D0FE207047074B984221
:1015D00008D049339842F7D1002070470120704766
:1015E0000220704703207047010010000200100025
:1015F000F8B5046805462046FFF7DEFF032841D80A
:101600006B794FEA930E39B975460227A689AF4028
:10161000B6B226EA0706A6810A2505FB00E51D4E9F
:1016200046F82510043546F82520324631B1990890
:101630000223A5898B402B439BB2A38128234343DC
:1016400003F120011144EFF31286502585F312882F
:101650000425103313441F6817B10F601968043153
:10166000013D03F10403F6D10D60F3B283F3118859
:10167000282303FB0020036A2BB1A3899BB243F00C
:101680000103A381F8BDA38923F001031B041B0CF4
:10169000F7E700BFF81B00201E4B30B55B681E4A01
:1016A000C3F308039BB9EFF3128383B91B49106896
:1016B0008C6800BF13689842F9D14FF47A72184BC6
:1016C000196802FB01F31B1BB3FBF1F31EE0EFF300
:1016D0001281102383F31288104CA568236813F439
:1016E000803F18BF01200F4B1CBF1860A56814680D
:1016F0001868CAB282F311884FF47A72084B2044FA
:10170000196802FB01F35B1BB3FBF1F302FB003032
:1017100030BD00BF00ED00E0801B002010E000E0C5
:10172000E00A0020A02D002038B50446FFF7B4FFE2
:101730000546FFF7B1FF401BA042FAD338BD10B5F4
:10174000044604B910BD4FF47A70FFF7EDFF013C79
:10175000F7E7EFF31283102282F312880649DBB217
:101760000A6801320A600021044A1160044A1268C2
:1017700083F31188704700BF801B0020A02D00203C
:1017800010E000E0014B5868F7F7F4BC400B002074
:10179000014B1868F7F7EEBC400B0020836A8169A3
:1017A000426B1944D160416A8B4229BF0169CB1A4F
:1017B000CB1A53602ABF0023536083624FF00003AB
:1017C00080F84430136838BF816243F0010313602E
:1017D0007047436A8269D154436A02690133934274
:1017E00028BF00234362436B1BB11B68DB0705D492
:1017F000D4E7026DD36843F08003D3607047036879
:101800009B69184703685B6918470368DB681847DA
:1018100003685B68184703681B68184703682DE96D
:10182000F041DB6904460E46174693B90D467B1B13
:101830003344002B01DCBDE8F081236820469B681F
:1018400098470028F9D015F8011B2046FFF7E3FF61
:10185000EDE7BDE8F0411847E0E7064B53F82020DC
:1018600032B193881268D1680B4218BF1B04136110
:10187000704700BFEC0A002010B50409013C022C9F
:1018800000F00F0215D80C4B33F8141041FA02F394
:1018900013F001000ED0012090400138084005F0FF
:1018A00069FB064B1C44237C0344054800EBC30042
:1018B00010BD002010BD00BF70A1010880AE01085E
:1018C000341600202DE9F0410C460746002851D07F
:1018D00003682D4A03F14043A3F5843302EB9323BD
:1018E000D87C03F02DFCBD88E20654BF04F00C0147
:1018F00004F00F0115F0FF0F04F07C063B681AD0CE
:1019000000204FF0010E4FF00F0C1A680EFA00F78E
:1019100037EA05040BD184000CFA04F822EA080225
:1019200001FA04F4282E42EA040225D15F61013055
:101930000828EBD11A60FF2D1CD900204FF0010EB2
:101940004FF00F0C5A6800F108040EFA04F434EA60
:1019500005070BD187000CFA07F822EA080201FA02
:1019600007F7282E42EA07020AD15C6101300828F5
:10197000E9D15A60BDE8F081482E08BF1F61D6E763
:10198000482E08BF1C61F1E780AE010810B1036862
:1019900082885A61704710B1036882881A61704763
:1019A00038B1002914BF00211021838802688B40C0
:1019B000136170470F4B01461B883BB90E4B1868EB
:1019C0000E4B1B780BB981F00101E9E70C4B5A690A
:1019D00072B150B10B4A196810880B4A92FBF0F2B1
:1019E00092B20A8001225A7470471A6810805874A3
:1019F000704700BF400C0020440C0020480C002021
:101A00004C0C0020640C002020A107000123084A90
:101A1000834012781340074A52F8200019B1191C6C
:101A200018BF0121BCE7B3FA83F14909FAE700BF07
:101A3000E60A0020EC0A002038B50D4601210446D4
:101A40000846FFF7E3FF00210846FFF7DFFF04B970
:101A500038BD0120FFF701FF0020FFF7FEFE012047
:101A6000FFF7A8FF2846FFF76AFE0120FFF7F5FE03
:101A70000020FFF7F2FE0020FFF79CFF013C284604
:101A8000FFF75DFEE4B2E2E738B50D460130C4B2BF
:101A900005B938BD05203221FFF7CEFF4FF4FA70AB
:101AA000FFF74DFE1CB1FA212046FFF7C5FF4FF4AA
:101AB0007A70FFF744FE013DEAE708B50A21FFF717
:101AC000E3FF024A024BDA6008BD00BF0400FA05DA
:101AD00000ED00E0FAF760BBFAF75EBBFAF75CBB1B
:101AE000FAF75ABBFAF758BBFAF756BBFAF754BBEA
:101AF000037903F00C03042B05D0082B0FD0BBB9DE
:101B0000B0F80B0070470B4BB0F80B001B7803EBE1
:101B1000C30203EB820300EB430080B27047054B26
:101B2000B0F80B005B7803EB430300EB8300F4E7B2
:101B3000002070470816002010B4447A631CDBB202
:101B400004444372A172027A9A4202D810BCFAF796
:101B50002BBC10BC704720B10078B0FA80F040096F
:101B600070470120704708B5202108F081FA03462C
:101B700018461BB102780133202AF9D008BD2DE99F
:101B8000F8430D4616468146002440F634074FF0D0
:101B900019084846FFF7E7FF814690B105F0DAFDE6
:101BA000B842A8BF3846B0F5617FB8BF4FF4617046
:101BB000A0F5617090FBF8F04CB9287033780133D0
:101BC00033700134022CE4D14846BDE8F8836870D4
:101BD000F4E710B50446B0F80900FAF79DFC014699
:101BE0002046FFF785FF4B68184410BD38B5054601
:101BF0000C46FFF7EEFF2B7903F00303012B00D017
